:100000000C9455470C9476470C948DD10C947647FC
:100010000C9476470C9476470C9476470C9476476C
:100020000C9476470C9476470C9476470C94B8D38E
:100030000C9476470C9476470C941BB40C9476473A
:100040000C9476470C9476470C9476470C9476473C
:100050000C9476470C9476470C9476470C9476472C
:100060000C9476470C94A7D10C9436D10C94764717
:100070000C940DCB0C94AFCA0C94EBCA0C9476473D
:100080000C9458D20C9476470C9476470C9476478F
:100090000C9476470C9476470C9476470C947647EC
:1000A0000C9476470C9476470C9476470C94F6BAE9
:1000B0000C949ABB0C9476470C9476470C940CB62F
:1000C0000C9476470C9476470C9476470C947647BC
:1000D0000C9476470C9476470C9476470C947647AC
:1000E0000C9491A50C9476470C9476470C94764723
:1000F0000C9476470C9476470C9476470C9476478C
:100100000C94CDBA0C9471BB0C94A4BA0C9448BB5B
:100110000C9476470C9476470C9476470C9476476B
:100120000C9476470C9476470C9476470C9476475B
:100130000C9476470C9470B50C9476470C947647E3
:100140000C9476470C9476470C9476470C9476473B
:100150000C9476470C9476470C9487A50C947647BC
:100160000C9476470C9476470C9476470C9476471B
:100170000C9476470C9476470C9476470C9476470B
:100180000C9476470C9476470C9476470C947647FB
:100190000C9476470C9476470C9476470C947647EB
:1001A0000C941FBB0C94C3BB0C9476470C947647FD
:1001B0000C94BEB50C9476470C9476470C94764715
:1001C0000C9476470C9476470C9476470C947647BB
:1001D0000C9476470C9476470C9476470C947647AB
:1001E0000C9476470C9476471C71267130713A71E5
:1001F00045714B774B774B774B774B774B714B7701
:100200004B774B774B774B774B774D7157716171CC
:100210006B7175714B774B774B774B774B774B7790
:100220007F714B77D5714B774B774B774B774B770C
:100230004B774B7714724B7730754B774B774B7707
:100240004B774B774B774B774B7730754B774B77BB
:100250004B774172467250725A725C72667271725A
:100260004B777C724B774B77B9724B774B774B77E9
:100270004B774B774B774B774B774B774B774B776E
:100280004B774B774B774B77C3724B774B774B77EB
:100290004B774B774B774B774B774B77CD720A7316
:1002A000477390739A73B373B373BD73C773D1738A
:1002B000DB73E573EA73F473FE7349774977497723
:1002C000497749774977497749774977497749772E
:1002D000497749774977497749774977497749771E
:1002E0004977BD734977497749774977497749779E
:1002F00049774977497749774977497749774977FE
:10030000497749774977087412741C7426744977C1
:100310004977497749774977497749774977B37377
:10032000D67695769976A1767D76817689768D7664
:10033000AD76C276CA76CE76D2762E77A576A174C1
:10034000B274C3744B774B773B740D714B77D47495
:10035000E574F6743075A47318754B774C744B774D
:1003600007755D7430744B774B774B776E747F7481
:1003700090743DBA45BA4DBA55BA5DBA65BA6DBA10
:1003800075BA60BDC5BCCDBCD5BCDDBCE5BCEDBCA3
:10039000F5BCFDBC05BD0DBD15BD1DBD25BD2DBDEF
:1003A00045BD45BD45BD45BD45BD45BD45BD45BD3D
:1003B00045BD45BD45BD45BD45BD45BD45BD45BD2D
:1003C00045BD45BD45BD45BD45BD45BD45BD45BD1D
:1003D00045BD45BD45BD45BD45BD45BD45BD45BD0D
:1003E00045BD45BD45BD35BD3DBD084AD73B3BCEAE
:1003F000016E84BCBFFDC12F3D6C74319ABD568324
:100400003DDA3D00C77F11BED9E4BB4C3E916BAADB
:10041000AABE000000803F05A84CCDB2D44EB9382A
:1004200036A9020C50B9918688083CA6AAAA2ABE11
:10043000000000803F07634236B79BD8A71A39688F
:100440005618AEBAAB558C1D3CB7CC5763BD6DED9D
:10045000FD753EF6177231BF000000803F080000B6
:1004600000BE922449123EABAAAA2ABECDCCCC4CE7
:100470003E00000080BEABAAAAAA3E00000000BF5A
:10048000000000803F0000000000084178D3BB431B
:1004900087D1133D190E3CC3BD4282AD2B3E68ECA3
:1004A0008276BED98FE1A93E4C80EFFFBE01C4FF2A
:1004B0007F3F0000000000000C9447AD0C94D7561D
:1004C0000C943DBD0C94E9560C94A3630C941FC18D
:1004D0000C9449C70C94E6A60C9499760C945DC9CB
:1004E0000C9426740C94B6CD0C9475BA0C94975A4F
:1004F0000C9441720C94F0B90C9445BD0C94CA76DE
:100500000C94915B0C94D4740C946F5A0C94EF5629
:100510000C94ABCE0C94735A0C9457710C9414BA7F
:100520000C942DBD0C9418750C945D5B0C942E6886
:100530000C94EC5D0C9455BA0C948C470C941C7183
:100540000C944B770C940DBD0C9482470C9400577F
:100550000C9414C20C9493590C940B5F0C94A35AF2
:100560000C9487570C9495BC0C9478470C94405D80
:100570000C94F2A60C9461710C946B710C9460BD98
:100580000C9443AD0C94645D0C946F630C94BB5954
:100590000C94875A0C94CE630C94935A0C947D5B04
:1005A0000C94DD560C9435BD0C94FE730C941F57BF
:1005B0000C9407AD0C94C2760C9450CC0C94DB795F
:1005C0000C9408BA0C94746E0C94ED910C94907485
:1005D0000C9450720C94795B0C94D25A0C946DBAB2
:1005E0000C9440570C94E94A0C943A710C94EBC962
:1005F0000C948F5A0C9420580C945C720C94AD5946
:100600000C94CA560C949F5A0C94755B0C949C588D
:100610000C94FDBC0C9423AD0C940B570C943071CE
:100620000C94AB5E0C9421540C94E3560C940A6D1C
:100630000C94F6740C94A75A0C944C740C94A174FA
:100640000C9422CE0C941C630C94695B0C9410BA2D
:100650000C943E640C94F4B90C942E6B0C94FB78BF
:100660000C9459570C94F15A0C94B8830C942A5753
:100670000C94B35A0C94D6760C94147F0C94CB47FC
:100680000C943FAD0C94675A0C9483780C944DBA3B
:100690000C94E5740C94F6570C94DEA60C94F2AC12
:1006A0000C940A730C944D710C945DBA0C94B37352
:1006B0000C949FAE0C9412740C94E1670C9415BDCD
:1006C0000C94AEAB0C9445710C944BAD0C94AAAB4E
:1006D0000C94B66E0C9414630C947F710C9489582E
:1006E0000C94B2740C94F9B90C94F6A60C945B6853
:1006F0000C948FBC0C945A720C94A8AB0C94E859CF
:100700000C94366B0C9420630C9466720C94C37238
:100710000C947B5A0C94DDBC0C9470680C94AFB8AC
:100720000C94DAA60C94C2590C9495760C94E5734B
:100730000C94ED6D0C941DBD0C94BD730C9495B987
:100740000C94EEA60C94815B0C9485790C94186340
:100750000C94595B0C94C9590C9405BD0C9490737E
:100760000C94DC470C9441B90C941C5D0C94DB7325
:100770000C945D740C94D2760C94C25C0C94037946
:100780000C949A730C947D760C94D5BC0C94C45D37
:100790000C94837F0C94995B0C94825E0C94625948
:1007A0000C949D770C9446790C94D25E0C947571E0
:1007B0000C94955B0C94C65D0C94835A0C94C37492
:1007C0000C947C720C949B670C9404C70C949860F6
:1007D0000C9414720C9437C10C9476AE0C94817600
:1007E0000C940D710C948D760C945E810C94267192
:1007F0000C9449770C943B740C94DB780C941EC1D8
:100800000C94E1680C94075A0C9446720C948B5D1E
:100810000C9447730C948BCF0C94D1730C945B5E47
:100820000C94C7730C9407750C94A3B80C9427CF41
:100830000C946E740C942DB90C94115E0C94BF57EB
:100840000C94635A0C94185D0C9471720C9475623C
:100850000C94BDB90C941C740C946B5A0C946EAB34
:100860000C94A55B0C94775A0C9470AB0C94B05B11
:100870000C94E5BC0C9455630C94CE760C948B5A76
:100880000C9470C10C9459620C945BB90C943DBAF1
:100890000C94ECB90C94C3620C94365E0C94CDBCF1
:1008A0000C94AB5A0C9430740C9414570C94355728
:1008B0000C9445BA0C94AFBC0C94855B0C940A590B
:1008C0000C9424630C94CAC90C94D6780C940779C0
:1008D0000C94F5560C9418670C945CCA0C94B0797F
:1008E0000C9474CE0C949B5A0C9465BA0C94D6A6B6
:1008F0000C94C5BC0C94A5760C940CBA0C94D6D070
:100900000C94877F0C94F5BC0C94EA730C94086EDD
:100910000C94EAA60C94A4730C9425BD0C940B794A
:100920000C944ACA0C9430750C9406640C9422CD35
:100930000C9453C10C94624E0C948D5B0C94655BCB
:100940000C94145B0C947F5A0C948E590C94AF5AEF
:100950000C94EDBC0C946D5B0C94895B0C94B97297
:100960000C94F55A0C947F740C9489760C948963DA
:100970000C9470570C94AD760C94E2A60C94B3BC16
:100980000C94CD720C9410680C94A1760C944B715D
:100990000C94715B0C94615B0C948B7F0C94FF78CE
:1009A0000C94F4730C9472AB0C9459580C94087416
:1009B0000C948D770C94B4590C94D5710C9497B811
:1009C0000C94FAA60C942E770C94DFA75B25732564
:1009D000735D20257320257320706F736974696FB0
:1009E0006E2531382E336625730A005B2573257317
:1009F0005D202573202573206F666673657425322C
:100A0000302E336625730A005B257325735D202520
:100A100073207A65726F206261636B6F6666253141
:100A2000392E336625730A005B257325735D2025F7
:100A300073206C61746368206261636B6F66662506
:100A400031382E336625730A005B257325735D20CC
:100A50002573206C617463682076656C6F636974BC
:100A6000792531332E306625732F6D696E0A005B50
:100A7000257325735D20257320736561726368207B
:100A800076656C6F636974792531322E3066257313
:100A90002F6D696E0A005B257325735D2025732019
:100AA000737769746368206D617825313764205BE2
:100AB000303D6F66662C313D686F6D696E672C3214
:100AC0003D6C696D69742C333D6C696D69742B687C
:100AD0006F6D696E675D0A005B257325735D202568
:100AE0007320737769746368206D696E253137648C
:100AF000205B303D6F66662C313D686F6D696E67B7
:100B00002C323D6C696D69742C333D6C696D697470
:100B10002B686F6D696E675D0A005B257325735DD9
:100B2000202573207261646975732076616C756528
:100B30002532302E346625730A005B257325735DDC
:100B4000202573206A756E6374696F6E2064657604
:100B5000696174696F6E2531342E346625732028DF
:100B60006C61726765722069732066617374657267
:100B7000290A005B257325735D202573206A657241
:100B80006B20686F6D696E672531362E3066257370
:100B90002F6D696E5E33202A2031206D696C6C697F
:100BA0006F6E0A005B257325735D202573206A65CF
:100BB000726B206D6178696D756D2531352E3066EB
:100BC00025732F6D696E5E33202A2031206D696C8C
:100BD0006C696F6E0A005B257325735D2025732099
:100BE00074726176656C206D696E696D756D253105
:100BF000372E336625730A005B257325735D202528
:100C0000732074726176656C206D6178696D756DA5
:100C10002531372E336625730A005B257325735DF6
:100C20002025732076656C6F63697479206D617817
:100C3000696D756D2531312E306625732F6D696EA6
:100C40000A005B257325735D202573206665656446
:100C500072617465206D6178696D756D2531312E15
:100C6000306625732F6D696E0A005B257325735DF1
:100C70002025732061786973206D6F646525313894
:100C8000642025730A005B6D615D20206D696E2014
:100C9000617263207365676D656E742531382E331C
:100CA0006625730A005B736C5D2020736F66742089
:100CB0006C696D697420656E61626C6525313264A2
:100CC0000A005B63745D202063686F7264616C204E
:100CD000746F6C6572616E63652531372E346625DD
:100CE000730A005B6A615D20206A756E6374696FC8
:100CF0006E20616363656C65726174696F6E25381F
:100D00002E306625730A005B6764695D2064656642
:100D100061756C742067636F6465206469737461C6
:100D20006E6365206D6F6465253264205B303D47DE
:100D300039302C313D4739315D0A005B6770615DA8
:100D40002064656661756C742067636F64652070EC
:100D500061746820636F6E74726F6C253364205BFE
:100D6000303D4736312C313D4736312E312C323D26
:100D70004736345D0A005B67636F5D2064656661BA
:100D8000756C742067636F646520636F6F72642095
:100D900073797374656D253364205B312D3620289B
:100DA0004735342D473539295D0A005B67756E5D1F
:100DB0002064656661756C742067636F6465207577
:100DC0006E697473206D6F6465253564205B303DFA
:100DD0004732302C313D4732315D0A005B67706C21
:100DE0005D2064656661756C742067636F6465205F
:100DF000706C616E6525313064205B303D47313762
:100E00002C313D4731382C323D4731395D0A0025C0
:100E10006320776F726B206F66667365743A253155
:100E2000322E336625730A002563206D616368697D
:100E30006E6520706F736E3A2531312E33662573DF
:100E40000A00256320706F736974696F6E3A2531EB
:100E5000352E336625730A00546F6F6C206E756DE6
:100E60006265722020202020202020202025640A76
:100E700000466565642072617465206D6F64653A33
:100E800020202020202025730A0044697374616E9D
:100E90006365206D6F64653A202020202020202586
:100EA000730A0050617468204D6F64653A202020F9
:100EB000202020202020202025730A00506C616E05
:100EC000653A2020202020202020202020202020C3
:100ED0002025730A004D6F74696F6E206D6F646515
:100EE0003A20202020202020202025730A00436F54
:100EF0006F7264696E6174652073797374656D3A9D
:100F000020202025730A00556E6974733A20202032
:100F100020202020202020202020202025730A00AF
:100F2000486F6D696E672073746174653A20202084
:100F3000202020202025730A0046656564686F6CB8
:100F4000642073746174653A20202020202025736A
:100F50000A004D6F74696F6E2073746174653A2076
:100F60002020202020202025730A004379636C650F
:100F70002073746174653A202020202020202020D6
:100F800025730A00526177206D616368696E652080
:100F900073746174653A20202025730A004D6163E3
:100FA00068696E652073746174653A202020202082
:100FB000202025730A004C696E65206E756D626590
:100FC000723A2531302E30660A004665656420721B
:100FD0006174653A2531362E336625732F6D696E3F
:100FE0000A0056656C6F636974793A2531372E3380
:100FF0006625732F6D696E0A0050101F10FF0F4792
:101000003935202D20756E6974732D7065722D72BF
:1010100065766F6C7574696F6E206D6F64650047DF
:101020003934202D20756E6974732D7065722D6DA5
:10103000696E757465206D6F64652028692E652E54
:10104000206665656472617465206D6F6465290052
:10105000473933202D20696E766572736520746977
:101060006D65206D6F6465008C106C104739312000
:101070002D20696E6372656D656E74616C206469A4
:101080007374616E6365206D6F646500473930204D
:101090002D206162736F6C7574652064697374616F
:1010A0006E6365206D6F646500DD10C510AF10477D
:1010B0003634202D20636F6E74696E756F757320E2
:1010C0006D6F6465004736312E31202D20657861C3
:1010D00063742073746F70206D6F646500473631E0
:1010E000202D2065786163742070617468206D6FB5
:1010F00064650017110811F910473139202D205966
:101100005A20706C616E6500473138202D20585A86
:1011100020706C616E6500473137202D20585920B2
:10112000706C616E6500A311911178115711301127
:10113000473830202D2063616E63656C206D6F74BD
:10114000696F6E206D6F646520286E6F6E6520611B
:1011500063746976652900473320202D20636F75FD
:101160006E74657220636C6F636B77697365206161
:101170007263206665656400473220202D20636C11
:101180006F636B7769736520617263206665656460
:1011900000473120202D206C696E656172206665E4
:1011A000656400473020202D206C696E65617220D7
:1011B000747261766572736520287365656B2900AA
:1011C0006A12501236121C120212E811CE11473563
:1011D00039202D20636F6F7264696E6174652073AE
:1011E000797374656D203600473538202D20636F84
:1011F0006F7264696E6174652073797374656D20B4
:101200003500473537202D20636F6F7264696E613A
:1012100074652073797374656D203400473536200A
:101220002D20636F6F7264696E61746520737973CA
:1012300074656D203300473535202D20636F6F7244
:1012400064696E6174652073797374656D20320012
:10125000473534202D20636F6F7264696E61746549
:101260002073797374656D203100473533202D204C
:101270006D616368696E6520636F6F7264696E612A
:1012800074652073797374656D009D1297129012C6
:10129000486F6D696E6700486F6D6564004E6F74CE
:1012A00020486F6D656400D112CC12C712C112BC08
:1012B00012B312456E6420486F6C6400486F6C6412
:1012C00000446563656C00506C616E0053796E6319
:1012D000004F666600E412E012DB12486F6C640097
:1012E00052756E0053746F70000E130413FE12F7E4
:1012F00012F3124A6F6700486F6D696E6700507293
:101300006F6265004D616368696E696E67004F6664
:10131000660044133E13381333132F13291320137D
:1013200053687574646F776E004379636C6500452C
:101330006E640053746F7000416C61726D00526591
:1013400061647900496E697469616C697A696E6774
:1013500000A713A1139B13961392138E1389138363
:10136000137D1376137213691353687574646F7762
:101370006E004A6F6700486F6D696E67004379635E
:101380006C650050726F626500486F6C6400527546
:101390006E00456E640053746F7000416C61726D35
:1013A00000526561647900496E697469616C697A9B
:1013B000696E6700CE13B813473231202D206D6956
:1013C0006C6C696D65746572206D6F646500473281
:1013D00030202D20696E63686573206D6F64650031
:1013E0000814FD13F113E8135B7261646975735D92
:1013F000005B696E686962697465645D005B737443
:10140000616E646172645D005B64697361626C65E6
:10141000645D0022141E1419142064656700206D99
:101420006D0020696E002A2A2A204E4F54494345F8
:10143000202A2A2A20526573657474696E672062B7
:10144000617564207261746520746F202573005B80
:10145000626175645D20555342206261756420723B
:1014600061746525313564205B313D393630302C6F
:10147000323D31393230302C333D33383430302C3A
:10148000343D35373630302C353D31313532303022
:101490002C363D3233303430305D0A005B72786D6B
:1014A0005D2073657269616C205258206D6F6465B0
:1014B00025313564205B303D636861725F6D6F6418
:1014C000652C313D6C696E655F6D6F64655D0A000A
:1014D0005B65785D2020656E61626C6520666C6F6F
:1014E0007720636F6E74726F6C25313064205B30CF
:1014F0003D6F66662C313D584F4E2F584F46462C57
:10150000323D5254532F4354535D0A005B65655D71
:101510002020656E61626C65206563686F253138D7
:1015200064205B303D6F66662C313D6F6E5D0A0056
:101530005B65635D2020657870616E64204C462099
:10154000746F2043524C46206F6E205458253664E9
:10155000205B303D6F66662C313D6F6E5D0A0092F8
:10156000158D15871581157B1574156D1532333062
:1015700034303000313135323030003537363030AC
:1015800000333834303000313932303000393630C1
:1015900030003000737973006662000000000702BB
:1015A000FB788B5DC45DE039D723DC43737973002E
:1015B0006676000000000703FF788B5DC45DE439A8
:1015C000EC51783F737973006870000000000700E9
:1015D00003798B5DD25EEC390000803F7379730034
:1015E000687600000000070007798B5DDB78F03932
:1015F000000000417379730069640000000004007A
:101600000B798378C45DDC39000000000000000025
:101610006E00000000000100635A5957825E5B3281
:1016200000000000000000006C696E650000010011
:10163000635A7057825E5B320000000000000000B9
:1016400076656C0000000002C9598757C45DDC391B
:1016500000000000000000006665656400000002F4
:10166000E859BF57C45DDC390000000000000000ED
:101670007374617400000000675ACA56C45DDC3997
:1016800000000000000000006D61637300000000B6
:101690006B5AD756C45DDC39000000000000000022
:1016A00063796373000000006F5ADD56C45DDC3956
:1016B00000000000000000006D6F74730000000067
:1016C000735AE356C45DDC390000000000000000DE
:1016D000686F6C6400000000775AE956C45DDC391D
:1016E0000000000000000000756E6974000000003A
:1016F0007F5AF556C45DDC39000000000000000090
:10170000636F6F7200000000835A0057C45DDC39BC
:1017100000000000000000006D6F6D6F0000000011
:10172000875A0B57C45DDC39000000000000000040
:10173000706C616E000000008B5A1457C45DDC3978
:1017400000000000000000007061746800000000EC
:101750008F5A1F57C45DDC390000000000000000F4
:101760006469737400000000935A2A57C45DDC3921
:10177000000000000000000066726D6F00000000B5
:10178000975A3557C45DDC390000000000000000A6
:10179000746F6F6C000000009B5A4057C45DDC39C9
:1017A000000000006D706F006D706F780000000326
:1017B000A55B2058C45DDC39000000006D706F002F
:1017C0006D706F7900000003A55B2058C45DDC39A3
:1017D000000000006D706F006D706F7A00000003F4
:1017E000A55B2058C45DDC39000000006D706F00FF
:1017F0006D706F6100000003A55B2058C45DDC398B
:10180000000000006D706F006D706F6200000003DB
:10181000A55B2058C45DDC39000000006D706F00CE
:101820006D706F6300000003A55B2058C45DDC3958
:1018300000000000706F7300706F73780000000389
:10184000995BF657C45DDC3900000000706F7300CF
:10185000706F737900000003995BF657C45DDC3943
:1018600000000000706F7300706F737A0000000357
:10187000995BF657C45DDC3900000000706F73009F
:10188000706F736100000003995BF657C45DDC392B
:1018900000000000706F7300706F7362000000033F
:1018A000995BF657C45DDC3900000000706F73006F
:1018B000706F736300000003995BF657C45DDC39F9
:1018C000000000006F6673006F667378000000030D
:1018D000B05B5958C45DDC39000000006F667300CE
:1018E0006F66737900000003B05B5958C45DDC3942
:1018F000000000006F6673006F66737A00000003DB
:10190000B05B5958C45DDC39000000006F6673009D
:101910006F66736100000003B05B5958C45DDC3929
:10192000000000006F6673006F66736200000003C2
:10193000B05B5958C45DDC39000000006F6673006D
:101940006F66736300000003B05B5958C45DDC39F7
:1019500000000000686F6D00686F6D65000000009A
:101960007B5AEF569359DC3900000000686F6D0018
:10197000686F6D7800000000995B1C5DC45D3032BB
:1019800000000000686F6D00686F6D790000000056
:10199000995B1C5DC45D313200000000686F6D0012
:1019A000686F6D7A00000000995B1C5DC45D323287
:1019B00000000000686F6D00686F6D61000000003E
:1019C000995B1C5DC45D333200000000686F6D00E0
:1019D000686F6D6200000000995B1C5DC45D34326D
:1019E00000000000686F6D00686F6D63000000000C
:1019F000995B1C5DC45D35320000000070726200AE
:101A000070726265000000001EC11C5DC45D36324C
:101A100000000000707262007072627800000003C3
:101A20001EC18B5DC45D3732000000007072620021
:101A300070726279000000031EC18B5DC45D3B3291
:101A400000000000707262007072627A0000000391
:101A50001EC18B5DC45D3F320000000070726200E9
:101A600070726261000000031EC18B5DC45D433271
:101A70000000000070726200707262620000000379
:101A80001EC18B5DC45D47320000000070726200B1
:101A900070726263000000031EC18B5DC45D4B3237
:101AA000000000006A6F67006A6F6778000000003E
:101AB0001EC1185DAD595532000000006A6F670005
:101AC0006A6F6779000000001EC1185DB459553275
:101AD000000000006A6F67006A6F677A000000000C
:101AE0001EC1185DBB595532000000006A6F6700C7
:101AF0006A6F6761000000001EC1185DC25955324F
:101B000000000000707772007077723100000000F2
:101B100014BA41B9C45DDC3900000000707772006E
:101B2000707772320000000014BA41B9C45DDC392C
:101B300000000000707772007077723300000000C0
:101B400014BA41B9C45DDC3900000000707772003E
:101B5000707772340000000014BA41B9C45DDC39FA
:101B60000000000031000000316D61000000030042
:101B7000F0B91C5DC65D5E580000404031000000B9
:101B80003173610000000303F4B98B5D97B86958A5
:101B90006666E63F310000003174720000000B04FD
:101BA000F9B98B5DA3B86D580000B4433100000053
:101BB000316D69000000030008BA1C5DAFB85F58C2
:101BC000000000413100000031706F000000030090
:101BD0000CBA1C5DEC5D63580000803F31000000D2
:101BE00031706D000000030010BA1C5D2DB96458FF
:101BF0000000004032000000326D61000000030070
:101C0000F0B91C5DC65D7D58000000403200000048
:101C10003273610000000303F4B98B5D97B88858F4
:101C20006666E63F320000003274720000000B046A
:101C3000F9B98B5DA3B88C585C8F2241320000004B
:101C4000326D69000000030008BA1C5DAFB87E5811
:101C5000000000413200000032706F0000000300FD
:101C60000CBA1C5DEC5D82580000803F3200000021
:101C700032706D000000030010BA1C5D2DB983584E
:101C80000000004033000000336D610000000300DD
:101C9000F0B91C5DC65D9C580000803F3300000019
:101CA0003373610000000303F4B98B5D97B8A75844
:101CB0006666E63F330000003374720000000B04D8
:101CC000F9B98B5DA3B8AB585C8F2241330000009B
:101CD000336D69000000030008BA1C5DAFB89D5861
:101CE000000000413300000033706F00000003006B
:101CF0000CBA1C5DEC5DA1580000803F3300000071
:101D000033706D000000030010BA1C5D2DB9A2589D
:101D10000000004034000000346D6100000003004A
:101D2000F0B91C5DC65DBB58000000003400000027
:101D30003473610000000303F4B98B5D97B8C65893
:101D40006666E63F340000003474720000000B0445
:101D5000F9B98B5DA3B8CA585C8F224134000000EA
:101D6000346D69000000030008BA1C5DAFB8BC58B0
:101D7000000000413400000034706F0000000300D8
:101D80000CBA1C5DEC5DC05800000000340000007F
:101D900034706D000000030010BA1C5D2DB9C158ED
:101DA000000000407800000078616D000000030032
:101DB000145B89589C58EC300000803F780000008C
:101DC00078766D0000000B005D5B8B5DC362F130C7
:101DD0000080BB44780000007866720000000B00B1
:101DE000595B8B5DC362ED300080BB44780000001E
:101DF00078746E0000000B03655B8B5DC362F93085
:101E0000000000007800000078746D0000000B03F3
:101E1000615B8B5DC362F53000000A43780000000F
:101E2000786A6D0000000B00695B8B5D0A59FD301C
:101E30000000FA4378000000786A680000000B0098
:101E40006D5B8B5D6259013100007A4478000000BF
:101E5000786A640000000B04715B8B5DC36209311A
:101E60000AD7233C7800000078736E00000003005E
:101E7000795B1C5D95BC10300000803F780000004D
:101E800078737800000003007D5B1C5D95BC113009
:101E900000000000780000007873760000000B005E
:101EA000815B8B5DC36211310000FA437800000052
:101EB000786C760000000B00855B8B5DC36215318A
:101EC0000000C84178000000786C620000000B033D
:101ED000895B8B5DC36219310000A040780000006F
:101EE000787A620000000B038D5B8B5DC3621D314D
:101EF000000000007900000079616D00000003001F
:101F0000145B89589C5821310000803F7900000003
:101F100079766D0000000B005D5B8B5DC36226313E
:101F20000080BB44790000007966720000000B005D
:101F3000595B8B5DC36222310080BB447900000095
:101F400079746E0000000B03655B8B5DC3622E31FC
:101F5000000000007900000079746D0000000B03A0
:101F6000615B8B5DC3622A310000E64279000000AC
:101F7000796A6D0000000B00695B8B5D0A59323194
:101F80000000FA4379000000796A680000000B0045
:101F90006D5B8B5D6259363100007A447900000038
:101FA000796A640000000B04715B8B5DC3623E3193
:101FB0000AD7233C7900000079736E00000003000B
:101FC000795B1C5D95BC12300000803F79000000F9
:101FD00079737800000003007D5B1C5D95BC1330B5
:101FE00000000000790000007973760000000B000B
:101FF000815B8B5DC36246310000FA4379000000CB
:10200000796C760000000B00855B8B5DC3624A3102
:102010000000C84179000000796C620000000B03E9
:10202000895B8B5DC3624E310000A04079000000E7
:10203000797A620000000B038D5B8B5DC3625231C5
:10204000000040407A0000007A616D00000003004B
:10205000145B89589C5856310000803F7A0000007C
:102060007A766D0000000B005D5B8B5DC3625B31B7
:102070000080BB447A0000007A66720000000B000A
:10208000595B8B5DC36257310080BB447A0000000E
:102090007A746E0000000B03655B8B5DC362633175
:1020A00000008CC27A0000007A746D0000000B03FF
:1020B000615B8B5DC3625F31000000007A0000004D
:1020C0007A6A6D0000000B00695B8B5D0A5967310D
:1020D0000000FA437A0000007A6A680000000B00F2
:1020E0006D5B8B5D62596B3100007A447A000000B1
:1020F0007A6A640000000B04715B8B5DC36273310C
:102100000AD7233C7A0000007A736E0000000300B7
:10211000795B1C5D95BC1430000000007A00000063
:102120007A737800000003007D5B1C5D95BC153060
:102130000000803F7A0000007A73760000000B00F8
:10214000815B8B5DC3627B310000FA437A00000043
:102150007A6C760000000B00855B8B5DC3627F317B
:102160000000C8417A0000007A6C620000000B0396
:10217000895B8B5DC36283310000A0407A00000060
:102180007A7A620000000B038D5B8B5DC36287313E
:10219000000000006100000061616D0000000300AC
:1021A000145B89589C588B3100004040610000004E
:1021B00061766D00000003005D5B8B5DD25E903147
:1021C0000000B4446100000061667200000003007A
:1021D000595B8B5DD25E8C310000B444610000001D
:1021E00061746E0000000303655B8B5DC362983110
:1021F000000080BF6100000061746D0000000303F7
:10220000615B8B5DD25E9431000080BF6100000095
:10221000616A6D0000000300695B8B5D0A599C31A7
:102220000000FA4361000000616A680000000300DA
:102230006D5B8B5D6259A0310000FA4361000000C4
:10224000616A640000000304715B8B5DD25EA8319B
:102250000AD7233C610000006172610000000B039B
:10226000755B8B5DD25EAC31CF2E654261000000A4
:1022700061736E0000000300795B1C5D95BC163035
:102280000000803F610000006173780000000300DF
:102290007D5B1C5D95BC17300000000061000000F4
:1022A0006173760000000300815B8B5DD25EB0310C
:1022B0000000164461000000616C7600000003001D
:1022C000855B8B5DD25EB4310000C84261000000C6
:1022D000616C620000000303895B8B5DD25EB831E4
:1022E0000000A04061000000617A6200000003036A
:1022F0008D5B8B5DD25EBC3100000040620000004F
:1023000062616D0000000300145B89589C58C03165
:10231000000000006200000062766D000000030013
:102320005D5B8B5DD25EC5310000B444620000008D
:102330006266720000000300595B8B5DD25EC131A2
:102340000000B4446200000062746E0000000303E9
:10235000655B8B5DC362CD31000080BF6200000011
:1023600062746D0000000303615B8B5DD25EC93156
:10237000000080BF62000000626A6D000000030080
:10238000695B8B5D0A59D1310000FA43620000009D
:10239000626A640000000300715B8B5DD25EDD3118
:1023A0000AD7233C620000006272610000000B0348
:1023B000755B8B5DD25EE131CF2E6542630000001C
:1023C00063616D0000000300145B89589C58F5316F
:1023D000000000006300000063766D000000030051
:1023E0005D5B8B5DD25EFA310000B4446300000097
:1023F0006366720000000300595B8B5DD25EF631AC
:102400000000B4446300000063746E000000030326
:10241000655B8B5DC3620232000080BF6300000019
:1024200063746D0000000303615B8B5DD25EFE315F
:10243000000080BF63000000636A6D0000000300BD
:10244000695B8B5D0A5906320000FA4363000000A5
:10245000636A640000000300715B8B5DD25E123220
:102460000AD7233C630000006372610000000B0385
:10247000755B8B5DD25E1632CF2E654270310000E7
:102480007031667271000300D6A68B5DD25E3A573A
:102490000000C84270310000703163736C000300AB
:1024A000DAA68B5DD25E3E5700E0F6457031000043
:1024B0007031637368000300DEA68B5DD25E425705
:1024C0000000484670310000703163706C000303F7
:1024D000E2A68B5DD25E4657B81E053E7031000005
:1024E0007031637068000303E6A68B5DD25E4A57C5
:1024F0007B142E3E70310000703177736C00030046
:10250000EAA68B5DD25E4E570000000070310000DD
:102510007031777368000300EEA68B5DD25E525770
:102520000000000070310000703177706C00030310
:10253000F2A68B5DD25E5657CDCCCC3D70310000FB
:102540007031777068000303F6A68B5DD25E5A5730
:10255000CDCCCC3D703100007031706F660003034C
:10256000FAA68B5DD25E5E57CDCCCC3D673534008C
:102570006735347800000B03915B8B5DC3625C3080
:1025800000000000673534006735347900000B0324
:10259000915B8B5DC36260300000000067353400E2
:1025A0006735347A00000B03915B8B5DC362643046
:1025B00000000000673534006735346100000B030C
:1025C000915B8B5DC36268300000000067353400AA
:1025D0006735346200000B03915B8B5DC3626C3026
:1025E00000000000673534006735346300000B03DA
:1025F000915B8B5DC3627030000000006735350071
:102600006735357800000B03915B8B5DC3627430D6
:1026100000000000673535006735357900000B0391
:10262000915B8B5DC3627830000000006735350038
:102630006735357A00000B03915B8B5DC3627C309C
:1026400000000000673535006735356100000B0379
:10265000915B8B5DC3628030000000006735350000
:102660006735356200000B03915B8B5DC36284307C
:1026700000000000673535006735356300000B0347
:10268000915B8B5DC36288300000A0C16735360066
:102690006735367800000B03915B8B5DC3628C302D
:1026A00000000000673536006735367900000B03FF
:1026B000915B8B5DC362903000000000673536008F
:1026C0006735367A00000B03915B8B5DC3629430F3
:1026D00000000000673536006735366100000B03E7
:1026E000915B8B5DC3629830000000006735360057
:1026F0006735366200000B03915B8B5DC3629C30D3
:1027000000000000673536006735366300000B03B4
:10271000915B8B5DC362A03000000000673537001D
:102720006735377800000B03915B8B5DC362A43083
:1027300000000000673537006735377900000B036C
:10274000915B8B5DC362A8300000000067353700E5
:102750006735377A00000B03915B8B5DC362AC3049
:1027600000000000673537006735376100000B0354
:10277000915B8B5DC362B0300000000067353700AD
:102780006735376200000B03915B8B5DC362B43029
:1027900000000000673537006735376300000B0322
:1027A000915B8B5DC362B830000000006735380074
:1027B0006735387800000B03915B8B5DC362BC30DA
:1027C00000000000673538006735387900000B03DA
:1027D000915B8B5DC362C03000000000673538003C
:1027E0006735387A00000B03915B8B5DC362C430A0
:1027F00000000000673538006735386100000B03C2
:10280000915B8B5DC362C830000000006735380003
:102810006735386200000B03915B8B5DC362CC307F
:1028200000000000673538006735386300000B038F
:10283000915B8B5DC362D0300000000067353900CA
:102840006735397800000B03915B8B5DC362D43030
:1028500000000000673539006735397900000B0347
:10286000915B8B5DC362D830000000006735390092
:102870006735397A00000B03915B8B5DC362DC30F6
:1028800000000000673539006735396100000B032F
:10289000915B8B5DC362E03000000000673539005A
:1028A0006735396200000B03915B8B5DC362E430D6
:1028B00000000000673539006735396300000B03FD
:1028C000915B8B5DC362E830000000006739320025
:1028D0006739327800000103915B8B5DC45DCD32B6
:1028E00000000000673932006739327900000103C7
:1028F000915B8B5DC45DD13200000000673932000E
:102900006739327A00000103915B8B5DC45DD5327B
:1029100000000000673932006739326100000103AE
:10292000915B8B5DC45DD9320000000067393200D5
:102930006739326200000103915B8B5DC45DDD325B
:10294000000000006739320067393263000001037C
:10295000915B8B5DC45DE13200000000673238009E
:102960006732387800000103955B8B5DC45DE5320A
:102970000000000067323800673238790000010338
:10298000955B8B5DC45DE932000000006732380062
:102990006732387A00000103955B8B5DC45DED32D0
:1029A0000000000067323800673238610000010320
:1029B000955B8B5DC45DF13200000000673238002A
:1029C0006732386200000103955B8B5DC45DF532B0
:1029D00000000000673238006732386300000103EE
:1029E000955B8B5DC45DF9320000000067333000F9
:1029F0006733307800000103955B8B5DC45DFD3269
:102A000000000000673330006733307900000103B5
:102A1000955B8B5DC45D01330000000067333000BF
:102A20006733307A00000103955B8B5DC45D05332D
:102A3000000000006733300067333061000001039D
:102A4000955B8B5DC45D0933000000006733300087
:102A50006733306200000103955B8B5DC45D0D330D
:102A6000000000006733300067333063000001036B
:102A7000955B8B5DC45D1133000000006A696400E2
:102A80006A696461000000001EC1645DAB5E063AC5
:102A9000000000006A6964006A6964620000000066
:102AA0001EC1645DAB5E0A3A000000006A69640002
:102AB0006A696463000000001EC1645DAB5E0E3A8B
:102AC000000000006A6964006A6964640000000034
:102AD0001EC1645DAB5E123A0000000073797300A2
:102AE0006A61000000000F00B35A8B5DC3622A3098
:102AF0000050C347737973006374000000000F0433
:102B0000D25A8B5DC3622E300AD7233C737973008F
:102B1000736C000000000700F15A1C5DC65D323086
:102B20000000000073797300737400000000070058
:102B3000AFBC1C5D8FBC05300000803F7379730013
:102B40006D74000000000702ECB98B5D5BB95A5848
:102B500000000040000000006D6500000000000063
:102B60001FC1BDB9BDB9DC39000000000000000084
:102B70006D640000000000001FC195B995B9DC39F3
:102B80000000000073797300656A00000000070010
:102B9000837F1C5DEC5DF8390000803F7379730022
:102BA0006A76000000000700877F1C5D147FCC3C24
:102BB00000004040737973006A7300000000070052
:102BC0008B7F1C5DEC5DCE3C0000803F7379730011
:102BD000747600000000070014C21C5DEC5DCD5946
:102BE0000000803F737973007176000000000700D9
:102BF0004BAD1C5D365E9357000000007379730087
:102C00007376000000000700AEAB1C5D115EA0579C
:102C10000000803F737973007369000000000700B3
:102C2000AAAB405D72ABA15700007A437379730081
:102C3000656300000000070014631C5DCE63E22F93
:102C40000000000073797300656500000000070054
:102C500018631C5D3E64E32F00000000737973006D
:102C600065780000000007001C631C5D0664E42F0B
:102C7000000000407379730072786D000000070057
:102C800020631C5DEC5DE52F0000803F73797300CD
:102C9000626175640000040024631C5D7562E02FAE
:102CA0000000A0400000000073720000000000005F
:102CB000A8AB6EAB70ABDC39000000000000000078
:102CC00071720000000000003FADF2ACC45DDC3961
:102CD000000000000000000071690000000000001A
:102CE00043AD07ADC45DDC3900000000000000000A
:102CF000716F00000000000047AD23ADC45DDC39FA
:102D000000000000000000006572000000000000EC
:102D10001EC1DFA7C45DDC39000000000000000018
:102D200071660000000000001EC1185D8E59DC397C
:102D300000000000000000007278000000000000A9
:102D400053C15962C45DDC3900000000000000007E
:102D50006D736700000000001FC1185DC45DDC39A1
:102D60000000000000000000636C6561720000005C
:102D70001EC1624E624EDC390000000000000000FF
:102D800074657374000000001EC18579B3BCDC3922
:102D900000000000000000006465666100000000A3
:102DA0001EC1B079C25CDC390000000000000000E8
:102DB000626F6F74000000001EC1DB79D678DC39C9
:102DC000000000000000000068656C70000000005A
:102DD0001EC14679C45DDC3900000000000000001F
:102DE00068000000000000001EC14679C45DDC39A7
:102DF000000000007379730067706C00000007002A
:102E00009F5A1C5D115E4030000000007379730012
:102E100067756E0000000700A35A1C5DEC5D413031
:102E20000000803F7379730067636F000000070044
:102E3000A75A1C5DC65D3F300000004073797300E7
:102E40006770610000000700AB5A1C5D115E4230E4
:102E50000000004073797300676469000000070098
:102E6000AF5A1C5DEC5D4330000000000000000024
:102E700067630000000000001EC18D779D77DC397C
:102E800000000000000000006D61000000000B0465
:102E9000F55A8B5DC3623730CDCCCC3D00000000CD
:102EA000666400000000030037C11C5DEC5DCD3C92
:102EB000000000007564610075646130000003006B
:102EC00053C1645DAB5E9839000000007564610019
:102ED000756461310000030053C1645DAB5E9C39D1
:102EE0000000000075646100756461320000030039
:102EF00053C1645DAB5EA0390000000075646100E1
:102F0000756461330000030053C1645DAB5EA43996
:102F10000000000075646200756462300000030008
:102F200053C1645DAB5EA8390000000075646200A7
:102F3000756462310000030053C1645DAB5EAC395F
:102F400000000000756462007564623200000300D6
:102F500053C1645DAB5EB03900000000756462006F
:102F6000756462330000030053C1645DAB5EB43925
:102F700000000000756463007564633000000300A6
:102F800053C1645DAB5EB839000000007564630036
:102F9000756463310000030053C1645DAB5EBC39EE
:102FA0000000000075646300756463320000030074
:102FB00053C1645DAB5EC0390000000075646300FE
:102FC000756463330000030053C1645DAB5EC439B4
:102FD0000000000075646400756464300000030044
:102FE00053C1645DAB5EC8390000000075646400C5
:102FF000756464310000030053C1645DAB5ECC397D
:103000000000000075646400756464320000030011
:1030100053C1645DAB5ED03900000000756464008C
:10302000756464330000030053C1645DAB5ED43942
:10303000000000005F7465005F74657800000002A6
:1030400070C18B5DC45D0355000000005F746500B6
:103050005F7465790000000270C18B5DC45D075527
:10306000000000005F7465005F74657A0000000274
:1030700070C18B5DC45D0B55000000005F7465007E
:103080005F7465610000000270C18B5DC45D0F5507
:10309000000000005F7465005F746562000000025C
:1030A00070C18B5DC45D1355000000005F74650046
:1030B0005F7465630000000270C18B5DC45D1755CD
:1030C000000000005F7472005F74727800000002FC
:1030D00070C18B5DC45D2856000000005F747200F3
:1030E0005F7472790000000270C18B5DC45D2C5664
:1030F000000000005F7472005F74727A00000002CA
:1031000070C18B5DC45D3056000000005F747200BA
:103110005F7472610000000270C18B5DC45D345643
:10312000000000005F7472005F74726200000002B1
:1031300070C18B5DC45D3856000000005F74720082
:103140005F7472630000000270C18B5DC45D3C5609
:10315000000000005F7473005F74733100000002B0
:1031600070C18B5DC45D9355000000005F707300FB
:103170005F7073310000000270C18B5DC45DA355A8
:10318000000000005F6373005F63733100000002A2
:1031900070C18B5DC45DB355000000005F657300B6
:1031A0005F6573310000000270C18B5DC45DC35563
:1031B000000000005F7873005F7873310000000248
:1031C00070C18B5DC45DF558000000005F6665004E
:1031D0005F6665310000000270C18B5DC45DD35530
:1031E000000000005F7473005F747332000000021F
:1031F00070C18B5DC45D9755000000005F70730067
:103200005F7073320000000270C18B5DC45DA75512
:10321000000000005F6373005F6373320000000210
:1032200070C18B5DC45DB755000000005F65730021
:103230005F6573320000000270C18B5DC45DC755CD
:10324000000000005F7873005F78733200000002B6
:1032500070C18B5DC45D0D59000000005F666500A4
:103260005F6665320000000270C18B5DC45DD7559A
:10327000000000005F7473005F747333000000028D
:1032800070C18B5DC45D9B55000000005F707300D2
:103290005F7073330000000270C18B5DC45DAB557D
:1032A000000000005F6373005F637333000000027F
:1032B00070C18B5DC45DBB55000000005F6573008D
:1032C0005F6573330000000270C18B5DC45DCB5538
:1032D000000000005F7873005F7873330000000225
:1032E00070C18B5DC45D2559000000005F666500FC
:1032F0005F6665330000000270C18B5DC45DDB5505
:10330000000000005F7473005F74733400000002FB
:1033100070C18B5DC45D9F55000000005F7073003D
:103320005F7073340000000270C18B5DC45DAF55E7
:10333000000000005F6373005F63733400000002ED
:1033400070C18B5DC45DBF55000000005F657300F8
:103350005F6573340000000270C18B5DC45DCF55A2
:10336000000000005F7873005F7873340000000293
:1033700070C18B5DC45D3D59000000005F66650053
:103380005F6665340000000270C18B5DC45DDF556F
:1033900000000000000000005F64616D000000009C
:1033A0001EC1075A075ADC39000000000000000067
:1033B00073653030000002001EC1405D5B5EAC579B
:1033C00000000000000000007365303100000200C2
:1033D0001EC1405D5B5EAE570000000000000000B3
:1033E00073653032000002001EC1405D5B5EB05765
:1033F0000000000000000000736530330000020090
:103400001EC1405D5B5EB25700000000000000007E
:1034100073653034000002001EC1405D5B5EB4572E
:10342000000000000000000073653035000002005D
:103430001EC1405D5B5EB65700000000000000004A
:1034400073653036000002001EC1405D5B5EB857F8
:10345000000000000000000073653037000002002B
:103460001EC1405D5B5EBA57000000000000000016
:1034700073653038000002001EC1405D5B5EBC57C2
:1034800000000000000000007365303900000200F9
:103490001EC1405D5B5EBE570000000000000000E2
:1034A00073653130000002001EC1405D5B5EC05795
:1034B00000000000000000007365313100000200D0
:1034C0001EC1405D5B5EC2570000000000000000AE
:1034D00073653132000002001EC1405D5B5EC4575F
:1034E000000000000000000073653133000002009E
:1034F0001EC1405D5B5EC65700000000000000007A
:1035000073653134000002001EC1405D5B5EC85728
:10351000000000000000000073653135000002006B
:103520001EC1405D5B5ECA57000000000000000045
:1035300073653136000002001EC1405D5B5ECC57F2
:103540000000000000000000736531370000020039
:103550001EC1405D5B5ECE57000000000000000011
:1035600073653138000002001EC1405D5B5ED057BC
:103570000000000000000000736531390000020007
:103580001EC1405D5B5ED2570000000000000000DD
:1035900073653230000002001EC1405D5B5ED4578F
:1035A00000000000000000007365323100000200DE
:1035B0001EC1405D5B5ED6570000000000000000A9
:1035C00073653232000002001EC1405D5B5ED85759
:1035D00000000000000000007365323300000200AC
:1035E0001EC1405D5B5EDA57000000000000000075
:1035F00073653234000002001EC1405D5B5EDC5723
:103600000000000000000000736532350000020079
:103610001EC1405D5B5EDE57000000000000000040
:1036200073653236000002001EC1405D5B5EE057EC
:103630000000000000000000736532370000020047
:103640001EC1405D5B5EE25700000000000000000C
:1036500073653238000002001EC1405D5B5EE457B6
:103660000000000000000000736532390000020015
:103670001EC1405D5B5EE6570000000000000000D8
:1036800073797300000000001EC198600B5FDC3985
:103690000000000000000000703100000000000089
:1036A0001EC198600B5FDC390000000000000000C4
:1036B00031000000000000001EC198600B5FDC3983
:1036C00000000000000000003200000000000000C8
:1036D0001EC198600B5FDC39000000000000000094
:1036E00033000000000000001EC198600B5FDC3951
:1036F0000000000000000000340000000000000096
:103700001EC198600B5FDC39000000000000000063
:1037100078000000000000001EC198600B5FDC39DB
:103720000000000000000000790000000000000020
:103730001EC198600B5FDC39000000000000000033
:103740007A000000000000001EC198600B5FDC39A9
:103750000000000000000000610000000000000008
:103760001EC198600B5FDC39000000000000000003
:1037700062000000000000001EC198600B5FDC3991
:1037800000000000000000006300000000000000D6
:103790001EC198600B5FDC390000000000000000D3
:1037A00067353400000000001EC198600B5FDC39F3
:1037B0000000000000000000673535000000000038
:1037C0001EC198600B5FDC390000000000000000A3
:1037D00067353600000000001EC198600B5FDC39C1
:1037E0000000000000000000673537000000000006
:1037F0001EC198600B5FDC39000000000000000073
:1038000067353800000000001EC198600B5FDC398E
:1038100000000000000000006735390000000000D3
:103820001EC198600B5FDC39000000000000000042
:1038300067393200000000001EC198600B5FDC3960
:1038400000000000000000006732380000000000A7
:103850001EC198600B5FDC39000000000000000012
:1038600067333000000000001EC198600B5FDC3938
:1038700000000000000000006D706F0000000000FC
:103880001EC198600B5FDC390000000000000000E2
:10389000706F7300000000001EC198600B5FDC3980
:1038A00000000000000000006F66730000000000D0
:1038B0001EC198600B5FDC390000000000000000B2
:1038C000686F6D00000000001EC198600B5FDC395E
:1038D00000000000000000007072620000000000A4
:1038E0001EC198600B5FDC39000000000000000082
:1038F00070777200000000001EC198600B5FDC3919
:1039000000000000000000006A6F67000000000077
:103910001EC198600B5FDC39000000000000000051
:103920006A696400000000001EC198600B5FDC390A
:10393000000000000000000075646100000000004D
:103940001EC198600B5FDC39000000000000000021
:1039500075646200000000001EC198600B5FDC39D6
:10396000000000000000000075646300000000001B
:103970001EC198600B5FDC390000000000000000F1
:1039800075646400000000001EC198600B5FDC39A4
:1039900000000000000000005F74650000000000EF
:1039A0001EC198600B5FDC390000000000000000C1
:1039B0005F747200000000001EC198600B5FDC396C
:1039C00000000000000000005F74730000000000B1
:1039D0001EC198600B5FDC39000000000000000091
:1039E0005F707300000000001EC198600B5FDC393F
:1039F00000000000000000005F6373000000000092
:103A00001EC198600B5FDC39000000000000000060
:103A10005F657300000000001EC198600B5FDC3919
:103A200000000000000000005F787300000000004C
:103A30001EC198600B5FDC39000000000000000030
:103A40005F666500000000001EC198600B5FDC39F6
:103A500000000000000000006D00000000000000F9
:103A60001EC18963C45DDC39000000000000000055
:103A700071000000000000001EC16F63C45DDC39EE
:103A800000000000000000006F00000000000000C7
:103A90001EC15563C45DDC39000000000000000059
:103AA00024000000000000001EC1A363C45DDC39D7
:103AB00000000000486F6D696E67206572726F725A
:103AC000202D2025632061786973207365747469E3
:103AD0006E6773206D6973636F6E66696775726573
:103AE000640050726F62696E67206572726F722037
:103AF0002D20256320617869732063616E6E6F7479
:103B0000206D6F766520647572696E672070726FC4
:103B100062696E67005B69645D202054696E794755
:103B2000204944253330730A005B68765D202068A5
:103B3000617264776172652076657273696F6E2554
:103B400031362E32660A005B68705D202068617233
:103B5000647761726520706C6174666F726D253177
:103B6000352E32660A005B66765D20206669726DCE
:103B7000776172652076657273696F6E2531362EB6
:103B800032660A005B66625D20206669726D77614D
:103B90007265206275696C642531382E32660A00C0
:103BA000456E7465722024626F6F743D3120746FAE
:103BB00020656E7465722074686520626F6F742072
:103BC0006C6F616465722E0A000A0A0A232323209F
:103BD00054696E794720424F4F54204C4F41444521
:103BE000522048656C70202323230A00456E7465BB
:103BF000722024646566613D3120746F20726573A4
:103C00006574207468652073797374656D20746FB2
:103C10002074686520666163746F727920646566DC
:103C200061756C742076616C7565732E0A546869D1
:103C3000732077696C6C206F766572777269746532
:103C400020616E79206368616E67657320796F7596
:103C50002068617665206D6164652E0A000A0A0A93
:103C60002323232054696E794720524553544F52E1
:103C7000452044454641554C54532048656C7020BE
:103C80002323230A00496E766F6B652073656C668B
:103C9000207465737420627920656E746572696E34
:103CA000672024746573743D4E20776865726520C3
:103CB0004E206973206F6E65206F663A0A202024BB
:103CC000746573743D312020736D6F6B652074656E
:103CD00073740A202024746573743D322020686F49
:103CE0006D696E67207465737420202028796F7564
:103CF000206D757374207472697020686F6D696EC1
:103D000067207377697463686573290A20202474B7
:103D10006573743D3320207371756172652074651D
:103D20007374202020286120736572696573206F89
:103D3000662073717561726573290A202024746589
:103D400073743D3420206172632074657374202085
:103D50002020202028736F6D65206C6172676520BC
:103D6000636972636C6573290A2020247465737417
:103D70003D3520206477656C6C2074657374202059
:103D80002020286D6F7665732073706163656420F1
:103D900062792031207365636F6E64206477656C8F
:103DA0006C73290A202024746573743D36202066C4
:103DB000656564686F6C6420746573742028656E33
:103DC000746572202120616E64207E20746F2068EB
:103DD0006F6C6420616E6420726573746172742C00
:103DE00020726573706563746976656C79290A2041
:103DF0002024746573743D3720204D20636F646503
:103E00007320746573742020284D20636F6465737C
:103E100020696E7465726D696E676C656420776980
:103E20007468206D6F766573290A20202474657389
:103E3000743D3820204A534F4E20746573742020FF
:103E4000202020286D6F74696F6E20746573742054
:103E500072756E207573696E67204A534F4E2063EA
:103E60006F6D6D616E6473290A202024746573740C
:103E70003D392020696E76657273652074696D65C1
:103E800020746573740A202024746573743D313086
:103E900020726F74617279206D6F74696F6E207417
:103EA0006573740A202024746573743D3131207366
:103EB0006D616C6C206D6F76657320746573740A28
:103EC000202024746573743D313220736C6F772029
:103ED0006D6F76657320746573740A202024746591
:103EE00073743D313320636F6F7264696E61746502
:103EF0002073797374656D206F66667365742074C2
:103F000065737420284739322C204735342D4735C6
:103F100039290A0A546573747320617373756D656A
:103F200020612063656E7465726564205859206F46
:103F3000726967696E20616E64206174206C6561CE
:103F400073742038306D6D20636C656172616E63CF
:103F50006520696E20616C6C2064697265637469A8
:103F60006F6E730A546573747320617373756D6536
:103F7000205A20686173206174206C65617374201D
:103F800034306D6D20706F73696974697665206374
:103F90006C656172616E63650A5465737473207336
:103FA00074617274207769746820612047302058EA
:103FB00030205930205A30206D6F76650A486F6D79
:103FC000696E672069732074686520657863657021
:103FD00074696F6E2E204E6F20696E697469616C12
:103FE00020706F736974696F6E206F7220636C65E7
:103FF0006172616E636520697320617373756D65AD
:10400000640A000A0A0A2323232054696E79472090
:1040100053454C4620544553542048656C7020232A
:1040200023230A0045616368202420636F6D6D615E
:104030006E642061626F766520616C736F206469C5
:1040400073706C6179732074686520746F6B656E32
:1040500020666F7220656163682073657474696E91
:104060006720696E205B205D20627261636B6574FE
:10407000730A546F20766965772073657474696E6E
:10408000677320656E746572206120746F6B656E56
:104090003A0A0A2020243C746F6B656E3E0A0A4679
:1040A0006F72206578616D706C652024796672206E
:1040B000746F20646973706C61792074686520592D
:1040C000206D6178206665656420726174650A0AF6
:1040D000546F207570646174652073657474696EC3
:1040E000677320656E74657220746F6B656E2065F2
:1040F0007175616C732076616C75653A0A0A2020CF
:10410000243C746F6B656E3E3D3C76616C75653E1C
:104110000A0A466F72206578616D706C652024799B
:1041200066723D38303020746F2073657420746877
:10413000652059206D617820666565642072617420
:104140006520746F20383030206D6D2F6D696E756D
:1041500074650A466F7220636F6E66696775726177
:1041600074696F6E2064657461696C732073656532
:104170003A2068747470733A2F2F67697468756297
:104180002E636F6D2F73796E746865746F732F541F
:10419000696E79472F77696B692F54696E79472D5E
:1041A000436F6E66696775726174696F6E0A005459
:1041B0006865736520636F6D6D616E6473206172F5
:1041C000652061637469766520666F7220636F6E27
:1041D00066696775726174696F6E3A0A202024738C
:1041E00079732053686F772073797374656D202815
:1041F00067656E6572616C292073657474696E679A
:10420000730A2020243120202053686F77206D6F9F
:10421000746F7220312073657474696E677320281F
:104220006F72207768617465766572206D6F746F48
:104230007220796F752077616E7420312C322C33A7
:104240002C34290A2020247820202053686F7720DE
:104250005820617869732073657474696E67732080
:10426000286F72207768617465766572206178695D
:104270007320796F752077616E7420782C792C7A91
:104280002C612C622C63290A2020246D20202053CD
:10429000686F7720616C6C206D6F746F722073652E
:1042A0007474696E67730A2020247120202053687B
:1042B0006F7720616C6C206178697320736574740A
:1042C000696E67730A2020246F20202053686F775F
:1042D00020616C6C206F66667365742073657474FE
:1042E000696E67730A2020242420202053686F778A
:1042F00020616C6C2073657474696E67730A20208A
:10430000246820202053686F7720746869732068C0
:10431000656C702073637265656E0A0A000A0A0A8A
:104320002323232054696E794720434F4E46494743
:1043300055524154494F4E2048656C702023232329
:104340000A000A466F722064657461696C656420B6
:1043500054696E794720696E666F207365653A20EF
:1043600068747470733A2F2F6769746875622E636E
:104370006F6D2F73796E746865746F732F54696EE7
:1043800079472F77696B692F0A466F7220746865C9
:10439000206C6174657374206669726D77617265F3
:1043A000207365653A2068747470733A2F2F6769BB
:1043B000746875622E636F6D2F73796E746865749F
:1043C0006F732F54696E79470A506C65617365206D
:1043D0006C6F6720616E79206973737565732061F6
:1043E0007420687474703A2F2F7777772E73796EF4
:1043F000746865746F732E636F6D2F666F72756D61
:10440000730A486176652066756E0A000A4E6F74FD
:10441000653A2054696E79472067656E65726174EC
:104420006573206175746F6D617469632073746165
:10443000747573207265706F727473206279206472
:10444000656661756C740A546869732063616E20D7
:1044500062652064697361626C65642062792065BD
:104460006E746572696E67202473763D300A5365F9
:1044700065207468652077696B692062656C6F7769
:1044800020666F72206D6F72652064657461696C5F
:10449000732E0A00546865736520636F6D6D616EDD
:1044A0006473206172652061637469766520667249
:1044B0006F6D2074686520636F6D6D616E64206C34
:1044C000696E653A0A205E78202020202020202076
:1044D000202020202052657365742028636F6E743D
:1044E000726F6C207829202D20736F66747761724B
:1044F000652072657365740A20203F2020202020EB
:1045000020202020202020204D616368696E6520D6
:10451000706F736974696F6E20616E642067636F7A
:104520006465206D6F64656C2073746174650A2026
:104530002024202020202020202020202020205344
:10454000686F7720616E642073657420636F6E6698
:10455000696775726174696F6E2073657474696ED2
:1045600067730A20202120202020202020202020C6
:1045700020202046656564686F6C64202D2073746C
:104580006F70206D6F74696F6E20776974686F75D6
:1045900074206C6F73696E6720706F736974696FD4
:1045A0006E0A20207E202020202020202020202075
:1045B00020204379636C65205374617274202D2030
:1045C000726573746172742066726F6D20666565C2
:1045D00064686F6C640A202068202020202020203E
:1045E00020202020202053686F7720746869732072
:1045F00068656C702073637265656E0A202024689C
:1046000020202020202020202020202053686F7789
:1046100020636F6E66696775726174696F6E20687A
:10462000656C702073637265656E0A202024746562
:1046300073742020202020202020204C69737420B7
:1046400073656C662D74657374730A202024746519
:1046500073743D4E2020202020202052756E207340
:10466000656C662D74657374204E0A202024686F73
:104670006D653D312020202020202052756E206164
:1046800020686F6D696E67206379636C650A20200E
:1046900024646566613D3120202020202020526561
:1046A00073746F726520616C6C2073657474696ECD
:1046B000677320746F2022666163746F72792220A1
:1046C00064656661756C74730A000A0A0A23232301
:1046D0002054696E79472048656C70202323230A93
:1046E000005B6A735D20206A736F6E207365726968
:1046F000616C697A65207374796C65253964205B17
:10470000303D72656C617865642C313D73747269FB
:1047100063745D0A005B6A765D20206A736F6E20A9
:10472000766572626F7369747925313564205B3008
:104730003D73696C656E742C313D666F6F74657284
:104740002C323D6D657373616765732C333D636F08
:104750006E666967732C343D6C696E656E756D2C81
:10476000353D766572626F73655D0A005B656A5DF3
:104770002020656E61626C65206A736F6E206D6FBC
:10478000646525313364205B303D746578742C3169
:104790003D4A534F4E5D0A00C958C358BC58B758DC
:1047A000AE58A35898588C58805872585B584C583B
:1047B0003F5833581F581258FD57E957E657E357EB
:1047C000D457BF57AA579B578B57795762574557AE
:1047D00028570F57F956E856D656C956B7569D561C
:1047E0009A569756945691568E568B56885685569D
:1047F00082567F567C5679567656735670566D564D
:104800006A566756645661565E565B5658565556FC
:1048100052564F564C5649564656435640563D56AC
:104820003A563756345631562E562B56285625565C
:1048300022561F561C5619561656135610560D560C
:104840000A56075604560156FE55D755B35593558B
:1048500079555F55455521550455EC54D654BC54F3
:1048600098547B546954495432541954F753DE53C5
:10487000C053A4538C537A535C53475343533F5311
:104880003B53375333532F532B53275323531F5328
:104890001B53175313530F530B530753ED52D3525C
:1048A000C052A45292527B525A5249522952095232
:1048B000EF51D551BE518B515E513E511C51F650B6
:1048C000CF50B35094507A5060503B501250FA4F32
:1048D000CF4FA34F6D4F384F264F144F054FF24E19
:1048E000D94EB74EA54E934E814E6F4E5D4E4B4EF8
:1048F000394E274E154E034EF14DDF4DCD4DBB4D7C
:10490000B74DB34DAF4DAB4DA74DA34D9F4D9B4DF7
:10491000974D934D8F4D8B4D874D834D7F4D7B4DE7
:10492000774D734D6F4D6B4D574D394D1D4DF24CBD
:10493000CD4CA84CA44CA04C9C4C984C944C904C06
:104940008C4C884C844C804C7C4C784C744C704C17
:104950005C4C404C244C084CEC4BD04BB44B984B2B
:104960007C4B604B444B284B0C4B084B044B004B8F
:10497000FC4AF84AF44AF04ADC4AB44A8D4A674A8B
:104980003A4A144AE749E349DF49DB49C849A7499C
:1049900092494A6F6767696E67206379636C652027
:1049A0006661696C65640050726F626520656E6453
:1049B000706F696E74206973207374617274696EAC
:1049C0006720706F696E740050726F626520637942
:1049D000636C65206661696C65640032343900324D
:1049E00034380032343700486F6D696E6720457285
:1049F000726F72202D20486F6D696E672073776922
:104A00007463686573206D6973636F6E666967753B
:104A100072656400486F6D696E67204572726F72CF
:104A2000202D204E65676174697665206C61746322
:104A300068206261636B6F666600486F6D696E67C0
:104A4000204572726F72202D2054726176656C2041
:104A50006D696E2026206D61782061726520746812
:104A6000652073616D6500486F6D696E67204572E2
:104A7000726F72202D204C617463682076656C6FB4
:104A800063697479206973207A65726F00486F6D6D
:104A9000696E67204572726F72202D2053656172B6
:104AA00063682076656C6F63697479206973207A16
:104AB00065726F00486F6D696E67204572726F7224
:104AC000202D20426164206F72206E6F2061786912
:104AD000732073706563696669656400486F6D690A
:104AE0006E67206379636C65206661696C6564003C
:104AF0003233390032333800323337003233360044
:104B0000323335003233340032333300536F66743E
:104B1000206C696D697420657863656564656420DF
:104B20002D2043206D617800536F6674206C696D91
:104B30006974206578636565646564202D20432071
:104B40006D696E00536F6674206C696D69742065C1
:104B500078636565646564202D2042206D6178006E
:104B6000536F6674206C696D697420657863656540
:104B7000646564202D2042206D696E00536F667459
:104B8000206C696D6974206578636565646564206F
:104B90002D2041206D617800536F6674206C696D23
:104BA0006974206578636565646564202D20412003
:104BB0006D696E00536F6674206C696D6974206551
:104BC00078636565646564202D205A206D617800E6
:104BD000536F6674206C696D6974206578636565D0
:104BE000646564202D205A206D696E00536F6674D1
:104BF000206C696D697420657863656564656420FF
:104C00002D2059206D617800536F6674206C696D9A
:104C10006974206578636565646564202D2059207A
:104C20006D696E00536F6674206C696D69742065E0
:104C300078636565646564202D2058206D61780077
:104C4000536F6674206C696D69742065786365655F
:104C5000646564202D2058206D696E00536F667462
:104C6000206C696D697420657863656564656400AE
:104C700032313900323138003231370032313600CA
:104C800032313500323134003231330032313200CA
:104C900032313100323130003230390032303800B8
:104CA000323037003230360054726170657A6F6985
:104CB0006420706C616E6E6572206661696C6564FB
:104CC00020746F20636F6E7665726765004C696D46
:104CD00069742073776974636820686974202D2073
:104CE00053687574646F776E206F63637572726555
:104CF00064004D616368696E6520697320616C6151
:104D0000726D6564202D20436F6D6D616E64206E41
:104D10006F742070726F636573736564004D6F7696
:104D200065206C657373207468616E206D696E69AF
:104D30006D756D2074696D65004D6F7665206C65CD
:104D40007373207468616E206D696E696D756D2076
:104D50006C656E6774680047656E657269632054A0
:104D6000696E7947206572726F720031393900318E
:104D700039380031393700313936003139350031B1
:104D800039340031393300313932003139310031B1
:104D90003930003138390031383800313837003196
:104DA000383600313835003138340031383300318D
:104DB00038320031383100313830005420776F728A
:104DC0006420697320696E76616C69640054207791
:104DD0006F7264206973206D697373696E67005226
:104DE00020776F726420697320696E76616C6964E4
:104DF000005220776F7264206973206D6973736944
:104E00006E67005120776F726420697320696E7637
:104E1000616C6964005120776F7264206973206D42
:104E2000697373696E67004C20776F7264206973D1
:104E300020696E76616C6964004C20776F72642023
:104E40006973206D697373696E67004820776F72AC
:104E50006420697320696E76616C6964004820770C
:104E60006F7264206973206D697373696E670045A2
:104E700020776F726420697320696E76616C696453
:104E8000004520776F7264206973206D69737369C0
:104E90006E67004420776F726420697320696E76B4
:104EA000616C6964004420776F7264206973206DBF
:104EB000697373696E67005020776F72642069733D
:104EC000206E6F7420612076616C696420746F6F4E
:104ED0006C206E756D626572005020776F72642071
:104EE0006973206E6F7420616E20696E74656765EA
:104EF00072005020776F7264206973206E6567615D
:104F000074697665005020776F7264206973207A27
:104F100065726F005020776F726420697320696E2C
:104F200076616C6964005020776F72642069732029
:104F30006D697373696E6700417263207370656396
:104F4000696669636174696F6E206572726F722041
:104F50002D20656E64706F696E74206973207374A0
:104F6000617274696E6720706F696E74004172635C
:104F70002073706563696669636174696F6E20652B
:104F800072726F72202D2072616469757320617274
:104F900063206F7574206F6620746F6C6572616E2C
:104FA000636500417263207370656369666963615C
:104FB00074696F6E206572726F72202D206D697337
:104FC00073696E67206F6666736574287329004184
:104FD00072632073706563696669636174696F6E7B
:104FE000206572726F72202D206D697373696E6710
:104FF000206178697328657329004172632073709A
:105000006563696669636174696F6E206572726F4A
:1050100072005370696E646C65206D7573742062E4
:1050200065207475726E696E6720666F7220746891
:10503000697320636F6D6D616E64005370696E6497
:105040006C65206D757374206265206F66662066DE
:105050006F72207468697320636F6D6D616E640098
:105060005370696E646C65205320776F7264206999
:105070007320696E76616C6964005370696E646C4C
:1050800065205320776F7264206973206D69737394
:10509000696E67005370696E646C65207370656536
:1050A00064206578636565646564206D6178696D09
:1050B000756D005370696E646C652073706565640E
:1050C0002062656C6F77206D696E696D756D00503B
:1050D000726F6772616D6D656420706F696E7420A8
:1050E00073616D652061732063757272656E7420E3
:1050F000706F696E740043757474657220636F6DB0
:1051000070656E736174696F6E2063616E6E6F742B
:1051100020626520656E61626C6564005265717520
:1051200065737465642076656C6F63697479206556
:10513000786365656473206C696D697473004730CA
:10514000206F72204731206D757374206265206175
:10515000637469766520666F722047353300526F3D
:105160007461727920617865732063616E6E6F740B
:10517000206265207573656420776974682074689F
:10518000697320636F6D6D616E6400496E76657240
:1051900073652074696D65206D6F64652063616E51
:1051A0006E6F74206265207573656420776974681A
:1051B000207468697320636F6D6D616E640046656D
:1051C000656472617465206E6F74207370656369C5
:1051D000666965640053656C656374656420706C12
:1051E000616E6520697320696E76616C6964005335
:1051F000656C656374656420706C616E65206973AD
:10520000206D697373696E670041786973207461FA
:105210007267657420706F736974696F6E2069734B
:1052200020696E76616C69640041786973207461ED
:105230007267657420706F736974696F6E2069732B
:10524000206D697373696E670041786973206973B3
:105250002064697361626C656400417869732069D8
:105260007320696E76616C696420666F7220746861
:10527000697320636F6D6D616E640041786973209E
:1052800063616E6E6F742062652070726573656E07
:1052900074004178697320776F7264206D6973734D
:1052A000696E670047636F6465206D6F64616C2091
:1052B00067726F75702076696F6C6174696F6E00CC
:1052C0004D20636F646520756E737570706F7274B6
:1052D00065640047636F646520636F6D6D616E6424
:1052E00020756E737570706F727465640047656EBB
:1052F000657269632047636F646520696E707574B9
:10530000206572726F7200313239003132380031EB
:10531000323700313236003132350031323400312B
:10532000323300313232003132310031323000312B
:105330003139003131380031313700313136003107
:10534000313500313134004A534F4E207374726945
:105350006E6720746F6F206C6F6E67004A534F4EFC
:1053600020696E7075742068617320746F6F206D92
:10537000616E79207061697273004A534F4E2073D9
:10538000796E746178206572726F7200496E707503
:10539000742076616C75652072616E676520657238
:1053A000726F7200496E707574206578636565640C
:1053B00073206D6178696D756D2076616C7565001F
:1053C000496E707574206C657373207468616E200B
:1053D0006D696E696D756D2076616C756500496EDD
:1053E0007075742065786365656473206D617820DD
:1053F0006C656E67746800436F6D6D616E64206EDE
:105400006F742061636365707465642061742074D7
:105410006869732074696D6500506172616D6574AF
:1054200065722063616E6E6F7420626520726561C3
:105430006400506172616D657465722069732072D9
:105440006561642D6F6E6C7900556E737570706F49
:1054500072746564206E756D626572206F72204A89
:10546000534F4E207479706500426164206E756DF3
:1054700062657220666F726D617400496E76616C50
:105480006964206F72206D616C666F726D65642057
:10549000636F6D6D616E6400556E7265636F676EEC
:1054A000697A656420636F6D6D616E64206F722030
:1054B000636F6E666967206E616D650047656E6536
:1054C00072696320617373657274696F6E206661BF
:1054D000696C757265004D656D6F727920666175D6
:1054E0006C742064657465637465640053746163EF
:1054F0006B206F766572666C6F7720646574656388
:1055000074656400436F6E74726F6C6C65722061B9
:105510007373657274696F6E206661696C7572650C
:105520000043616E6F6E6963616C206D61636869D1
:105530006E6520617373657274696F6E2066616950
:105540006C75726500506C616E6E6572206173736C
:10555000657274696F6E206661696C75726500535F
:1055600074657070657220617373657274696F6EB3
:10557000206661696C75726500456E636F64657263
:1055800020617373657274696F6E206661696C75F2
:10559000726500494F207375622D73797374656D60
:1055A00020617373657274696F6E206661696C75D2
:1055B000726500436F6E666967207375622D73793B
:1055C0007374656D20617373657274696F6E2066A4
:1055D00061696C75726500494F206D656D6F7279F8
:1055E00020616C6C6F636174696F6E2061737365A9
:1055F0007274696F6E206661696C75726500383807
:105600000038370038360038350038340038330079
:105610003832003831003830003739003738003739
:10562000370037360037350037340037330037322C
:105630000037310037300036390036380036370051
:105640003636003635003634003633003632003612
:105650003100363000353900353800353700353601
:105660000035350035340035330035320035310032
:1056700035300034390034380034370034360034E3
:1056800035003434003433003432003431003430E7
:105690000033390033380033370033360042616459
:1056A00020737461747573207265706F72742073E7
:1056B000657474696E670050657273697374656EA2
:1056C0006365206572726F7200466C6F6174206949
:1056D00073204E414E00466C6F61742069732069DF
:1056E0006E66696E697465004D6F76652074696DCC
:1056F00065206973204E414E004D6F7665207469B8
:105700006D6520697320696E66696E69746500470E
:10571000656E6572696320657863657074696F6E24
:10572000207265706F7274004661696C65642074E4
:105730006F2067657420706C616E6E657220627593
:10574000666665720053797374656D20616C617271
:105750006D202D207368757474696E6720646F778F
:105760006E00496E697469616C697A6174696F6E03
:10577000206661696C75726500526561642D6F6E9B
:105780006C79206164647265737300496E76616C34
:105790006964204164647265737300446976696466
:1057A00065206279207A65726F00466C6F6174695A
:1057B0006E6720706F696E74206572726F72004937
:1057C0006E7465726E616C2072616E6765206572C1
:1057D000726F7200496E7465726E616C20657272D0
:1057E0006F720031390031380046756E6374696F2D
:1057F0006E206973207374756262656400456E740F
:105800006572696E6720626F6F74206C6F6164658A
:105810007200496E697469616C697A696E670042E9
:1058200075666665722066756C6C202D20666174E5
:10583000616C004275666665722066756C6C00422C
:10584000756666657220656D707479004E6F2073A1
:1058500075636820646576696365004D61782066CC
:10586000696C652073697A65206578636565646530
:10587000640046696C65206E6F74206F70656E0001
:10588000456E64206F662066696C6500456E642015
:105890006F66206C696E6500486172642072657382
:1058A0006574005465726D696E6174656400436F60
:1058B0006D706C657465004E6F6F70004561676157
:1058C000696E004572726F72004F4B005B703170F1
:1058D0006F665D2070776D207068617365206F66FC
:1058E000662020202531352E3366205B302E2E3168
:1058F0005D0A005B70317770685D2070776D2063A2
:1059000063772070686173652068692531352E33AF
:1059100066205B302E2E315D0A005B703177706C33
:105920005D2070776D2063637720706861736520F8
:105930006C6F2531352E3366205B302E2E315D0A9B
:10594000005B70317773685D2070776D20636377DB
:105950002073706565642068692531352E306620B6
:1059600052504D0A005B703177736C5D2070776D1B
:1059700020636377207370656564206C6F25313513
:105980002E30662052504D0A005B70316370685DA6
:105990002070776D20637720706861736520686977
:1059A000202531352E3366205B302E2E315D0A00E6
:1059B0005B703163706C5D2070776D206377207051
:1059C00068617365206C6F202531352E3366205B4E
:1059D000302E2E315D0A005B70316373685D20707C
:1059E000776D206377207370656564206869202572
:1059F00031352E30662052504D0A005B7031637392
:105A00006C5D2070776D206377207370656564200E
:105A10006C6F202531352E30662052504D0A005BC8
:105A200070316672715D2070776D20667265717578
:105A3000656E63792020202531352E306620487A26
:105A40000A0053595354454D205245414459004C86
:105A50006F6164696E6720636F6E66696773206645
:105A6000726F6D20454550524F4D00496E69746903
:105A7000616C697A696E6720636F6E66696773200F
:105A8000746F204F4D43204F746865724D696C6C84
:105A90002073657474696E6773007B226572223AA5
:105AA0007B226662223A25302E32662C22737422C3
:105AB0003A25642C226D7367223A222573227D7D5C
:105AC0000A007B65723A7B66623A25302E32662C7C
:105AD00073743A25642C6D73673A222573227D7D99
:105AE0000A005B71765D20207175657565207265B1
:105AF000706F727420766572626F7369747925377E
:105B000064205B303D6F66662C313D73696E676C57
:105B1000652C323D747269706C655D0A00716F3A74
:105B200025640A0071693A25640A0071723A256495
:105B30000A005B73765D2020737461747573207244
:105B400065706F727420766572626F7369747925FF
:105B50003664205B303D6F66662C313D66696C743F
:105B6000657265642C323D766572626F73655D0A9D
:105B7000005B73695D202073746174757320696EB6
:105B800074657276616C2531342E3066206D730A2F
:105B9000004D6F746F7220256320706F77657220DF
:105BA000656E61626C65642073746174653A253258
:105BB0002E30660A005B257325735D206D257320EA
:105BC000706F776572206D616E6167656D656E746B
:105BD00025313064205B303D64697361626C6564BB
:105BE0002C313D616C77617973206F6E2C323D6989
:105BF0006E206379636C652C333D7768656E206D2C
:105C00006F76696E675D0A005B257325735D206D95
:105C1000257320706F6C6172697479253138642046
:105C20005B303D6E6F726D616C2C313D72657665D7
:105C30007273655D0A005B257325735D206D2573A6
:105C4000206D6963726F73746570732531366420DB
:105C50005B312C322C342C385D0A005B25732573A4
:105C60005D206D25732074726176656C207065729D
:105C7000207265766F6C7574696F6E2531302E34C5
:105C80006625730A005B257325735D206D257320DF
:105C90007374657020616E676C652532302E3366D3
:105CA00025730A005B257325735D206D2573206DB8
:105CB000617020746F206178697325313564205BD1
:105CC000303D582C313D592C323D5A2E2E2E5D0A36
:105CD000005B6D745D20206D6F746F722069646C61
:105CE000652074696D656F75742531342E326620B8
:105CF0005365630A00045D005DFB5C20646567001A
:105D0000206D6D0020696E005B73745D20207377D9
:105D100069746368207479706525313864205B305C
:105D20003D4E4F2C313D4E435D0A00546573742047
:105D3000232564206E6F7420666F756E640A004EB2
:105D4000312054314D360A4E32204731370A4E3316
:105D5000204732310A4E382046313830300A4E3929
:105D60002047310A4E3130302047393220582D3209
:105D7000352E313737592D33342E303732205A2DC6
:105D8000312E303030202854454D502C2052454D76
:105D90004F5645204C41544552290A4E3334332046
:105DA000582D32352E353935592D33342E3334397B
:105DB0000A4E33343420582D32352E373031592D98
:105DC00033342E3433360A4E33343520582D3235A1
:105DD0002E373931592D33342E3532300A4E333483
:105DE0003620582D32352E383634592D33342E3650
:105DF00030310A4E33343720582D32352E39323077
:105E0000592D33342E3637390A4E33343820582D35
:105E100032352E393630592D33342E3735340A4E3B
:105E200033343920582D32352E393832592D333408
:105E30002E3832360A4E33353020582D32352E3931
:105E40003837592D33342E3839350A4E3335312011
:105E5000582D32352E393736592D33342E393631C7
:105E60000A4E33353220582D32352E393438592DDB
:105E700033352E3032330A4E33353320582D3235F8
:105E80002E393033592D33352E3038320A4E3335D2
:105E90003420582D32352E383431592D33352E31AA
:105EA00033380A4E33353520582D32352E373633B8
:105EB000592D33352E3139300A4E33353620582D91
:105EC00032352E363639592D33352E3233390A4E86
:105ED00033353720582D32352E353539592D333558
:105EE0002E3238340A4E33353820582D32352E3480
:105EF0003333592D33352E3332350A4E333539206D
:105F0000582D32352E323931592D33352E33363323
:105F10000A4E33363020582D32352E313334592D38
:105F200033352E3339370A4E33363120582D32343B
:105F30002E393633592D33352E3432380A4E333616
:105F40003220582D32342E373737592D33352E34F1
:105F500035350A4E33363320582D32342E35373707
:105F6000592D33352E3437370A4E33363420582DD9
:105F700032342E333637592D33352E3439360A4ED6
:105F800033363520582D32342E313434592D3335B3
:105F90002E3531310A4E33363620582D32332E39D4
:105FA0003039592D33352E3532320A4E33363720BB
:105FB000582D32332E363631592D33352E35323970
:105FC0000A4E33363820582D32332E343033592D83
:105FD00033352E3533320A4E33363920582D32338D
:105FE0002E313333592D33352E3533320A4E333774
:105FF0003020582D32322E383533592D33352E3549
:1060000032370A2F4E3235313820473058302E3350
:106010003237592D33332E3532315A2D312E30301F
:10602000300A4E32353139204D3330004E31204761
:1060300032300A4E3520473430204731370A4E314E
:1060400030205431204D30360A284E313520473922
:1060500030204730205830205930205A30290A4EFD
:106060003230205335303030204D3033200A4E321C
:10607000352058302E3036342059302E33323620E9
:106080005A300A4E343020473031204631362E30D7
:106090000A4E35302058302E3036342059302E33C9
:1060A00032360A4E35352058302E303630205930B1
:1060B0002E3239330A4E36302058302E30373720C2
:1060C00059302E3236370A4E36352058302E31317F
:1060D000312059302E3235370A4E37302058302E85
:1060E0003134392059302E3235320A4E3735205866
:1060F000302E3138382059302E3235350A4E38306E
:106100002058302E3232372059302E3236380A4E4F
:1061100038352058302E3235372059302E3237312D
:106120000A4E39302058302E3333352059302E3234
:1061300036350A4E39352058302E34313220593018
:106140002E3237310A4E3130302058302E34373429
:106150002059302E3238370A4E3130352058302E03
:106160003439312059302E3238390A4E313130200D
:1061700058302E3531372059302E3237330A4E31D0
:1061800031352058302E3534342059302E323633C4
:106190000A4E3132302058302E3538302059302ECA
:1061A0003236310A4E3132352058302E35393520CD
:1061B00059302E3236330A4E3133302058302E3695
:1061C00032312059302E3237340A4E31333520588F
:1061D000302E3635392059302E3330360A4E313490
:1061E000302058302E3637332059302E3333350A8D
:1061F0004E3134352058302E3637392059302E3331
:1062000036310A4E3135302058302E363738205945
:10621000302E3338390A4E3135352058302E363746
:10622000302059302E3432300A4E3136302058303A
:106230002E3637302059302E3434360A4E3136352A
:106240002058302E3638302059302E3437340A4E0C
:106250003137302058302E3730342059302E3439F1
:10626000370A4E3137352058302E373332205930E7
:106270002E3531350A4E3138302058302E373934EA
:106280002059302E3533350A4E3138352058302ECE
:106290003837322059302E3536370A4E31393020D2
:1062A00058302E3935302059302E3630340A4E31A0
:1062B00039352058312E3033312059302E3634378D
:1062C0000A4E3230302058312E3134392059302E98
:1062D0003732320A4E3230352058312E33303820A2
:1062E00059302E3835340A4E3231302058312E3460
:1062F00033302059302E3938340A4E323135205857
:10630000312E3434372059302E3938360A4E323255
:10631000302058312E3632382059302E3832320A59
:106320004E3232352058312E3733322059302E3705
:1063300031340A4E3233302058322E303039205921
:10634000302E3338310A4E3233352058322E313127
:10635000362059302E3236360A4E323430205832FA
:106360002E3232382059302E3135370A4E323435FC
:106370002058322E3238302059302E3132330A4EE6
:106380003235302058322E3333322059302E3039C6
:10639000340A4E3235352058322E343233205930BB
:1063A0002E3037300A4E3236302058322E343839BB
:1063B0002059302E3036350A4E3236352058322E9E
:1063C0003535372059302E3036360A4E32373020A8
:1063D00058322E3632372059302E3038340A4E3269
:1063E00037352058322E3639332059302E31303956
:1063F0000A4E3238302058322E3733302059302E62
:106400003133330A4E3238352058322E3830352069
:1064100059302E3139300A4E3239302058322E3828
:1064200032392059302E3231360A4E323935205821
:10643000322E3838302059302E3239310A4E33302E
:10644000302058322E3838342059302E3330300A2C
:106450004E3330352058322E3839382059302E33CB
:1064600033320A4E3331302058322E3930352059EC
:10647000302E3336370A4E3331352058322E3931EB
:10648000302059302E3430370A4E333230205832D3
:106490002E3930382059302E3434360A4E333235C6
:1064A0002058322E3930312059302E3439350A4EA9
:1064B0003333302058322E3839372059302E343982
:1064C000350A4E3333352058322E38393020593082
:1064D0002E3532340A4E3334302058322E3834328E
:1064E0002059302E3630340A4E3334352058322E6F
:1064F0003831342059302E3636350A4E3335302077
:1065000058322E3739342059302E3735300A4E3331
:1065100035352058322E3739312059302E3833381E
:106520000A4E3336302058322E3831392059302E29
:106530003937360A4E3336352058322E3833372025
:1065400059312E3034340A4E3337302058322E38F9
:1065500036322059312E3131320A4E3337352058F8
:10656000322E3837372059312E3134350A4E3338F0
:10657000302058322E3931322059312E3231370AFB
:106580004E3338352058322E3931372059312E329A
:1065900032360A4E3339302058322E3935312059AF
:1065A000312E3238310A4E3339352058322E3937B0
:1065B000302059312E3239350A4E3430302058329D
:1065C0002E3939362059312E3239350A4E3430358C
:1065D0002058332E3031332059312E3237350A4E80
:1065E0003431302058332E3032342059312E323568
:1065F000340A4E3431352058332E3037302059315B
:106600002E3135310A4E3432302058332E30373760
:106610002059312E3133340A4E3432352058332E3E
:106620003132352059312E3033390A4E343330204F
:1066300058332E3133382059312E3031390A4E3407
:1066400033352058332E3230352059302E393038FA
:106650000A4E3434302058332E3238322059302EFE
:106660003739370A4E3434352058332E33363120FB
:1066700059302E3639310A4E3435302058332E34C5
:1066800032362059302E3539320A4E3435352058BD
:10669000332E3435362059302E3534330A4E3436C5
:1066A000302058332E3437392059302E3439330ABC
:1066B0004E3436352058332E3439342059302E3468
:1066C00037320A4E3437302058332E353035205982
:1066D000302E3434360A4E3437352058332E353187
:1066E000382059302E3431370A4E34383020583360
:1066F0002E3533302059302E3339310A4E34383567
:106700002058332E3536342059302E3330300A4E4F
:106710003439302058332E3537372059302E323522
:10672000330A4E3439352058332E35363820593017
:106730002E3231320A4E3530302058332E35343433
:106740002059302E3137360A4E3530352058332E09
:106750003534312059302E3134360A4E353130201F
:1067600058332E3535332059302E3131390A4E35D4
:1067700031352058332E3537362059302E313036CA
:106780000A4E3532302058332E3539372059302EC5
:106790003130320A4E3532352058332E36313820DA
:1067A00059302E3130390A4E3533302058332E3699
:1067B00033392059302E3132390A4E35333520588D
:1067C000332E3635302059302E3135390A4E353496
:1067D000302058332E3636332059302E3137380A90
:1067E0004E3534352058332E3637382059302E3137
:1067F00039320A4E3535302058332E363939205942
:10680000302E3139370A4E3535352058332E373250
:10681000332059302E3139360A4E35363020583330
:106820002E3736342059302E3137390A4E35363529
:106830002058332E3830352059302E3136350A4E17
:106840003537302058332E3838342059302E3135F2
:10685000390A4E3537352058332E393439205930DE
:106860002E3136350A4E3538302058332E393636EB
:106870002059302E3137350A4E3538352058332ED1
:106880003937382059302E3139340A4E35393020D5
:1068900058332E3937382059302E3232330A4E359C
:1068A00039352058332E3936302059302E32343590
:1068B0000A4E3630302058332E3833342059302E9B
:1068C0003331310A4E3630352058332E37363220A8
:1068D00059302E3334350A4E3631302058332E3766
:1068E00032362059302E3338390A4E363135205859
:1068F000332E3730332059302E3435380A4E363265
:10690000302058332E3638322059302E3533300A65
:106910004E3632352058332E3637392059302E3501
:1069200033340A4E3633302058332E36323620591F
:10693000302E3638310A4E3633352058332E353620
:10694000382059302E3832380A4E363430205833F9
:106950002E3434342059312E3038300A4E36343506
:106960002058332E3430352059312E3136370A4EE7
:106970003635302058332E3430342059312E3136CC
:10698000370A4E3635352058332E333837205931B3
:106990002E3230380A4E3636302058332E333834C3
:1069A0002059312E3230380A4E3636352058332EA3
:1069B0003336352059312E3236350A4E36373020AF
:1069C00058332E3335352059312E3238350A4E366C
:1069D00037352058332E3334382059312E33303860
:1069E0000A4E3638302058332E3333332059312E67
:1069F0003335300A4E3638352058332E3332312075
:106A000059312E3339310A4E3639302058332E332E
:106A100031312059312E3432380A4E36393520582A
:106A2000332E3333392059312E3432330A4E373036
:106A3000302058332E3434302059312E3430360A39
:106A40004E3730352058332E3531302059312E34E1
:106A500030380A4E3731302058332E3538352059EA
:106A6000312E3432310A4E3731352058332E3631FB
:106A7000312059312E3433390A4E373230205833D1
:106A80002E3631312059312E3434310A4E373235D9
:106A90002058332E3631352059312E3434310A4EB8
:106AA0003733302058332E3633362059312E343890
:106AB000380A4E3733352058332E36333420593187
:106AC0002E3531370A4E3734302058332E36323295
:106AD0002059312E3534330A4E3734352058332E71
:106AE0003630352059312E3536330A4E3735302081
:106AF00058332E3537362059312E3537350A4E3733
:106B000035352058332E3534342059312E3538312F
:106B10000A4E3736302058332E3437392059312E2B
:106B20003539320A4E3736352058332E3435312038
:106B300059312E3539380A4E3737302058332E33F5
:106B400038372059312E3632360A4E3737352058ED
:106B5000332E3339302059312E3633360A4E3738FA
:106B6000302058332E3533322059312E3630320A08
:106B70004E3738352058332E3630312059312E35A6
:106B800039370A4E3739302058332E3636382059A7
:106B9000312E3539380A4E3739352058332E3738AB
:106BA000322059312E3631320A4E383030205833A7
:106BB0002E3739342059312E3631380A4E38303597
:106BC0002058332E3836382059312E3633360A4E77
:106BD0003831302058332E3931382059312E36355E
:106BE000350A4E3831352058332E39343520593155
:106BF0002E3636370A4E3832302058332E39363456
:106C00002059312E3638350A4E3832352058332E39
:106C10003936372059312E3638350A4E3833302040
:106C200058332E3937342059312E3639390A4E38F7
:106C300033352058332E3938342059312E373235F8
:106C40000A4E3834302058332E3938342059312EFA
:106C50003735380A4E3834352058332E39373020FE
:106C600059312E3739300A4E3835302058332E39C5
:106C700034352059312E3831370A4E3835352058C1
:106C8000332E3931382059312E3832360A4E3836C3
:106C9000302058332E3839312059312E3832370AC6
:106CA0004E3836352058332E3834322059312E386C
:106CB00030390A4E3837302058332E37393820597A
:106CC000312E3738340A4E3837352058332E373482
:106CD000362059312E3737320A4E38383020583363
:106CE0002E3639382059312E3736340A4E38383559
:106CF0002058332E3633352059312E3736360A4E4A
:106D00003839302058332E3535332059312E373825
:106D1000350A4E3839352058332E3437382059311A
:106D20002E3832300A4E3930302058332E34303934
:106D30002059312E3836340A4E3930352058332E0A
:106D40003334352059312E3931380A4E393130201B
:106D500058332E3236342059322E3032330A4E39DF
:106D600031352058332E3234382059322E303531D7
:106D70000A4E3932302058332E3234302059322ED8
:106D80003038310A4E3932352058332E33313620DF
:106D900059322E3038360A4E3933302058332E339C
:106DA00039302059322E3130340A4E39333520589B
:106DB000332E3431342059322E3132310A4E3934A7
:106DC000302058332E3433312059322E3135330AA6
:106DD0004E3934352058332E3433332059322E3146
:106DE00038300A4E3935302058332E343237205956
:106DF000322E3230350A4E3935352058332E343163
:106E0000332059322E3232340A4E3936302058333C
:106E10002E3339322059322E3234320A4E39363539
:106E20002058332E3333352059322E3234340A4E23
:106E30003937302058332E3237382059322E3233FA
:106E4000360A4E3937352058332E323536205932EE
:106E50002E3234320A4E3938302058332E323339FC
:106E60002059322E3235310A4E3938352058332EDA
:106E70003231312059322E3238300A4E39393020F1
:106E800058332E3137342059322E3335360A4E39A5
:106E900039352058332E3135392059322E33393790
:106EA0000A4E313030302058332E313530205932AF
:106EB0002E3433380A4E313030352058332E3134A9
:106EC000302059322E3438310A4E3130313020588A
:106ED000332E3133322059322E3531300A4E313093
:106EE00031352058332E3131382059322E35343354
:106EF0000A4E313032302058332E30393920593251
:106F00002E3537360A4E313032352058332E303553
:106F1000312059322E3633310A4E31303330205839
:106F2000332E3030332059322E3636360A4E313039
:106F300033352058322E3935372059322E363835F0
:106F40000A4E313034302058322E39303720593201
:106F50002E3639390A4E313034352058322E3836F3
:106F6000302059322E3731310A4E313035302058E9
:106F7000322E3831392059322E3732370A4E3130DD
:106F800035352058322E3736382059322E373435A1
:106F90000A4E313036302058322E373136205932B1
:106FA0002E3735370A4E313036352058322E3637A7
:106FB000352059322E3735370A4E31303730205888
:106FC000322E3537392059322E3733310A4E31308F
:106FD00037352058322E3537302059322E3732335C
:106FE0000A4E313038302058322E3535392059325A
:106FF0002E3732300A4E313038352058322E353364
:10700000302059322E3730310A4E31303930205845
:10701000322E3530312059322E3639330A4E313046
:1070200039352058322E3437312059322E36383304
:107030000A4E313130302058322E34343320593218
:107040002E3636380A4E313130352058322E33390B
:10705000362059322E3633340A4E313131302058F1
:10706000322E3335342059322E3539310A4E3131F2
:1070700031352058322E3335322059322E353931C0
:107080000A4E313132302058322E333235205932C7
:107090002E3534330A4E313132352058322E3331C9
:1070A000352059322E3532310A4E313133302058A5
:1070B000322E3330372059322E3439380A4E31319E
:1070C00033352058322E3239362059322E34363468
:1070D0000A4E313134302058322E32393320593271
:1070E0002E3432370A4E313134352058322E32396F
:1070F000352059322E3336360A4E3131353020584C
:10710000322E3332312059322E3330330A4E313160
:1071100035352058322E3335382059322E32343717
:107120000A4E313136302058322E3431392059321E
:107130002E3230330A4E313136352058322E34312A
:10714000392059322E3137390A4E313137302058F3
:10715000322E3430352059322E3135380A4E313105
:1071600037352058322E3336322059322E313233D1
:107170000A4E313138302058322E333534205932CE
:107180002E3130340A4E313138352058322E3335D5
:10719000342059322E3039310A4E313139302058AD
:1071A000322E3338302059322E3036350A4E3131B6
:1071B00039352058322E3431302059322E30353185
:1071C0000A4E313230302058322E3431302059328C
:1071D0002E3034370A4E313230352058322E34308A
:1071E000352059322E3032380A4E31323130205863
:1071F000322E3430382059322E3031300A4E31326E
:1072000031352058322E3431362059312E39393526
:107210000A4E313232302058322E34333320593135
:107220002E3938320A4E313232352058322E34332C
:10723000382059312E3936330A4E31323330205806
:10724000322E3434372059312E3934380A4E313207
:1072500033352058322E3436312059312E393338D7
:107260000A4E313234302058322E343830205931E1
:107270002E3933310A4E313234352058322E3437DC
:10728000382059312E3839390A4E313235302058AC
:10729000322E3438372059312E3837350A4E3132B4
:1072A00035352058322E3530342059312E3835348A
:1072B0000A4E313236302058322E3532372059318D
:1072C0002E3834380A4E313236352058322E353485
:1072D000392059312E3834390A4E3132373020585E
:1072E000322E3537372059312E3836310A4E313269
:1072F00037352058322E3630342059312E38363634
:107300000A4E313238302058322E3633312059313E
:107310002E3835340A4E313238352058322E363434
:10732000302059312E3832370A4E31323930205818
:10733000322E3634302059312E3739320A4E31321E
:1073400039352058322E3632392059312E373539D9
:107350000A4E313330302058322E363132205931F6
:107360002E3732370A4E313330352058322E3537EA
:10737000362059312E3639340A4E313331302058C7
:10738000322E3533362059312E3636320A4E3133CD
:1073900031352058322E3437302059312E3631369F
:1073A0000A4E313332302058322E333435205931A1
:1073B0002E3535310A4E313332352058322E3330A6
:1073C000372059312E3532310A4E3133333020587F
:1073D000322E3236302059312E3438320A4E313383
:1073E00033352058322E3234332059312E3437374A
:1073F0000A4E313334302058322E3232382059314F
:107400002E3436390A4E313334352058322E32324A
:10741000322059312E3434380A4E31333530205829
:10742000322E3232382059312E3432350A4E313331
:1074300035352058322E3235342059312E343035FE
:107440000A4E313336302058322E323638205931F8
:107450002E3337330A4E313336352058322E3237F9
:10746000392059312E3334320A4E313337302058D7
:10747000322E3330382059312E3238370A4E3133DC
:1074800037352058322E3334302059312E323534AE
:107490000A4E313338302058322E343037205931AB
:1074A0002E3230310A4E313338352058322E3434B2
:1074B000312059312E3135360A4E3133393020588A
:1074C000322E3435342059312E3133310A4E313396
:1074D00039352058322E3436302059312E3130365D
:1074E0000A4E313430302058322E3436342059315F
:1074F0002E3130320A4E313430352058322E343766
:10750000312059312E3033360A4E31343130205843
:10751000322E3436362059302E3937310A4E313436
:1075200031352058322E3435312059302E38393704
:107530000A4E313432302058322E34313520593011
:107540002E3739310A4E313432352058322E34300C
:10755000332059302E3736370A4E313433302058E5
:10756000322E3338382059302E3736350A4E3134E2
:1075700033352058322E3330362059302E383431BE
:107580000A4E313434302058322E323232205930C3
:107590002E3931310A4E313434352058322E3131C2
:1075A000342059302E3939350A4E3134353020588F
:1075B000322E3030322059312E3037360A4E3134A7
:1075C00035352058312E3930352059312E31333967
:1075D0000A4E313436302058312E37353420593167
:1075E0002E3232330A4E313436352058312E36336E
:1075F000372059312E3237380A4E3134373020583F
:10760000312E3538322059312E3330310A4E313453
:1076100037352058312E3535382059312E33313514
:107620000A4E313438302058312E3436302059311A
:107630002E3335320A4E313438352058312E333915
:10764000392059312E3336300A4E313439302058F2
:10765000312E3333382059312E3335340A4E3134FC
:1076600039352058312E3238372059312E333239BE
:107670000A4E313530302058312E323438205931CD
:107680002E3239340A4E313530352058312E3231D0
:10769000372059312E3235340A4E313531302058A9
:1076A000312E3231342059312E3235320A4E3135B5
:1076B00031352058312E3137322059312E3139357C
:1076C0000A4E313532302058312E3132382059317E
:1076D0002E3133390A4E313532352058312E313181
:1076E000302059312E3131370A4E31353330205860
:1076F000302E3935382059302E3934310A4E313553
:1077000033352058302E3839312059302E38373320
:107710000A4E313534302058302E38323520593029
:107720002E3830380A4E313534352058302E373522
:10773000352059302E3734370A4E31353530205800
:10774000302E3631392059302E3633330A4E31350A
:1077500035352058302E3437372059302E353236D3
:107760000A4E313536302058302E343737205930D4
:107770002E3532340A4E313536352058302E3431DC
:10778000312059302E3437360A4E313537302058B3
:10779000302E3333312059302E3435340A4E3135C2
:1077A00037352058302E3237382059302E34323782
:1077B0000A4E313538302058302E3233312059308E
:1077C0002E3339370A4E313538352058302E31387E
:1077D000332059302E3337390A4E3135393020585D
:1077E000302E3133352059302E3336350A4E31356F
:1077F00039352058302E3037362059302E33343139
:107800000A4E3136303520473030204633302E3066
:107810000A4E31363130204D3035200A4E31363166
:107820003520473930205830205930205A300A4E00
:1078300031363135204D33300A28456E64206F666D
:1078400020434E432050726F6772616D2900284DAE
:1078500053472A2A2A2A204D6963726F7374657010
:107860002054657374205B76315D202A2A2A2A29E8
:107870000A473030204731372047323120473430F3
:107880002047343920473830204739300A6730786C
:107890003079307A300A7B22316D69223A317D0AA3
:1078A0007B22326D69223A317D0A7B22336D692257
:1078B0003A317D0A7B22346D69223A317D0A673084
:1078C000207831300A7B22316D69223A327D0A7884
:1078D000300A7B22316D69223A347D0A7831300AD0
:1078E0007B22316D69223A387D0A78300A67302070
:1078F0007931300A7B22326D69223A327D0A793041
:107900000A7B22326D69223A347D0A7931300A7B52
:1079100022326D69223A387D0A79300A6730207A3E
:1079200031300A7B22336D69223A327D0A7A300A7D
:107930007B22336D69223A347D0A7A31300A7B2208
:10794000336D69223A387D0A7A300A673020613116
:10795000300A7B22346D69223A327D0A61300A7B1B
:1079600022346D69223A347D0A6131300A7B223437
:107970006D69223A387D0A61300A6D3200284D5314
:10798000472A2A2A2A20436F6F7264696E617465E0
:10799000206F6666736574732074657374205B76FC
:1079A000315D202A2A2A2A290A6730306731376751
:1079B00032316734306734396738306739300A67B5
:1079C00035340A673932783079307A300A663630A1
:1079D000300A284D53472A2A2A2A207465737420B6
:1079E000473932206F6666736574732A2A2A2A29FA
:1079F0000A286D73675374657020313A204D6F7695
:107A0000652066726F6D20302C3020746F2033300B
:107A10002C30206D6D20696E20706F7369746976EB
:107A200065205820646972656374696F6E290A283D
:107A30006D73675374657020323A205265736574B4
:107A4000206F726967696E20746F20302E30207548
:107A500073696E6720473932290A286D736753743A
:107A6000657020333A204D6F766520746F20323078
:107A70002C302E2053686F756C64206D6F766520F6
:107A80003230206D6D20696E20706F736974697675
:107A900065205820646972656374696F6E20616E39
:107AA0006420737461747573207265706F727420D2
:107AB00073686F756C642073746172742066726F82
:107AC0006D20302C30290A286D736753746570203F
:107AD000343A204D6F766520746F20302E30202090
:107AE0002053686F756C64206D6F7665203230208E
:107AF0006D6D20696E206E656761746976652058CA
:107B000020646972656374696F6E20616E642073AE
:107B10007461747573207265706F72742073686F0E
:107B2000756C642073746172742066726F6D20329C
:107B3000302C30290A67317833300A67393278308F
:107B40000A67317832300A6731783079300A247325
:107B5000720A67393278300A673470302E350A2855
:107B60004D53472A2A2A2A207465737420473535D5
:107B7000206F6666736574732A2A2A2A290A286D7B
:107B800073675374657020313A2053657420436FD6
:107B90006F7264696E6174652073797374656D20AA
:107BA00032205B6735355D20746F206F66667365C4
:107BB00074206F662035302C3530290A286D7367A4
:107BC0005374657020323A2053656C6563742047A6
:107BD000353520636F6F7264696E617465207379E7
:107BE0007374656D290A286D73675374657020334B
:107BF0003A204D6F766520746F20302C302E20484F
:107C00006561642073686F756C64206D6F766520A4
:107C1000646961676F6E616C6C7920696E202B58A6
:107C200020616E64202B5920616E6420737461742E
:107C30007573207265706F72742073686F756C64F1
:107C40002073746172742066726F6D20302C30293D
:107C50000A6731304C3270327835307935300A6706
:107C600035350A6730783079300A673470302E3510
:107C70000A284D53472A2A2A2A20746573742047FC
:107C80003533206162736F6C757465206F76657231
:107C90007269646573202A2A2A2A290A286D736763
:107CA0005374657020313A2052756E2061207371D3
:107CB0007561726520696E2047353520737973745C
:107CC000656D290A286D73675374657020323A20F8
:107CD00052756E20612073717561726520772F4730
:107CE0003533206F76657272696465290A6730786A
:107CF0003079300A673078323079300A673078323C
:107D0000307932300A673078307932300A6730782B
:107D10003079300A673470302E350A673533673072
:107D2000783079300A673533673078323079300A05
:107D300067353367307832307932300A67353367E8
:107D40003078307932300A673533673078307930BF
:107D50000A6730783079300A673470302E350A2857
:107D60004D53472A2A2A2A20746573742052657459
:107D700075726E20746F20686F6D65202A2A2A2A1A
:107D8000290A286D73675374657020313A20526553
:107D90007475726E20746F20686F6D6520757369DD
:107DA0006E6720473238290A286D736753746570EF
:107DB00020323A20526573657420746F2047353441
:107DC00020636F6F72642073797374656D290A671D
:107DD00032380A6735340A6D333000284D53472A4C
:107DE0002A2A2A2054657374206163637572616363
:107DF00079206F6620736C6F77206D6F76657320C6
:107E00005B76315D202A2A2A2A290A6735350A67D6
:107E100030783079300A673470302E350A67347024
:107E2000302E350A67317831306632320A673534A0
:107E30000A6730783079300A6D333000284D534767
:107E40002A2A2A2A20546573742076657279207351
:107E5000686F7274206D6F766573205B76315D207C
:107E60002A2A2A2A290A6730783079300A6734703A
:107E7000302E350A673178302E3166313030300A95
:107E800078300A78302E310A78300A78302E310A6C
:107E900078300A78302E310A78300A78302E310A5C
:107EA00078300A78302E310A78300A78302E310A4C
:107EB00078300A78302E310A78300A78302E310A3C
:107EC00078300A78302E310A78300A78302E310A2C
:107ED00078300A78302E310A78300A78302E310A1C
:107EE00078300A78302E310A78300A78302E310A0C
:107EF000673470302E350A78300A78302E30310AE7
:107F000078300A78302E30310A78300A78302E30C6
:107F1000310A78300A78302E30310A78300A7830D9
:107F20002E30310A78300A78302E30310A78300A13
:107F300078302E30310A78300A78302E30310A7895
:107F4000300A78302E30310A78300A78302E3031CD
:107F50000A78300A78302E30310A78300A78302E9C
:107F600030310A78300A78302E30310A78300A7889
:107F7000302E30310A6730783079300A6D3200287F
:107F80004D53472A2A2A2A20526F74617279204160
:107F9000786973204D6F74696F6E20546573742017
:107FA0005B76315D202A2A2A2A290A673030673118
:107FB0003767323167343067343967383067393082
:107FC0000A6730783079307A306130623063300A55
:107FD0006735350A6730783079300A6633363030A5
:107FE000300A6730613336300A623336300A633321
:107FF00036300A61300A62300A63300A6731613113
:108000003434300A62313434300A63313434300A63
:1080100061300A62300A63300A67316131343430CA
:1080200062373230633336300A783079307A3061F3
:1080300030623063300A6731783630613134343041
:1080400062373230633336300A783079307A3061D3
:1080500030623063300A67317836307935306131DB
:1080600034343062373230633336300A7830793026
:108070007A306130623063300A6731783630793572
:1080800030783235613134343062373230633336F0
:10809000300A783079307A306130623063300A6784
:1080A00035340A6730783079300A6D333000284D26
:1080B00053472A2A2A2A20496E766572736520540E
:1080C000696D65204D6F74696F6E205465737420FF
:1080D0005B76315D202A2A2A2A290A6730306731E7
:1080E0003767323167343067343967383067393051
:1080F0000A6735350A6730783079300A6739330ACC
:1081000066302E30310A67317831300A7931300AE1
:108110007A31300A6131300A78300A79300A7A309F
:108120000A61300A67317831307931307A2D313057
:108130006131300A6730783079307A3061300A66E0
:10814000302E310A6732783130792D31307A2D3244
:10815000306931300A6730783079307A300A6733E5
:10816000783130792D31307A2D32306931300A67EB
:1081700030783079307A300A673278323079307A34
:108180002D32306931300A6730783079307A300AF0
:10819000673378323079306931300A673078307936
:1081A000307A300A6732783079307A2D333069315D
:1081B000300A6733783079307A306931300A673085
:1081C000783079307A300A673278307930693230F5
:1081D0002028435720333630206465677265657305
:1081E000290A673378307930693230202843435781
:1081F000203336302064656772656573290A6739F4
:10820000340A6735340A6730783079300A6D333094
:10821000007B226763223A2267303067313767324A
:1082200031673430673439673830673930227D0A36
:108230007B226763223A22673535227D0A7B2267DB
:1082400063223A22673078307930227D0A7B2267B8
:1082500063223A2266353030227D0A7B2267632210
:108260003A22284D53477371756172657329227DD7
:108270000A7B226763223A226730783230227D0AF5
:108280007B226763223A22793230227D0A7B226781
:1082900063223A227830227D0A7B226763223A22C7
:1082A0007930227D0A7B226763223A226731783156
:1082B00030227D0A7B226763223A22793130227D87
:1082C0000A7B226763223A227830227D0A7B22676A
:1082D00063223A227930227D0A7B226763223A2286
:1082E000284D5347636972636C657329227D0A7B4D
:1082F000226763223A226732783130792D31306932
:108300003130227D0A7B226763223A22673078303F
:108310007930227D0A7B226763223A2267337831E3
:1083200030792D3130693130227D0A7B226763221A
:108330003A22673078307930227D0A7B22676322C7
:108340003A2267327832307930693130227D0A7BC7
:10835000226763223A22673078307930227D0A7BA7
:10836000226763223A2267337832307930693130BC
:10837000227D0A7B226763223A2267307830793087
:10838000227D0A7B226763223A2267327830793075
:10839000693130227D0A7B226763223A2267337873
:1083A000307930693130227D0A7B226763223A229C
:1083B000673534227D0A7B226763223A2267307850
:1083C000307930227D0A7B226763223A226D333076
:1083D000227D00284D53472A2A2A2A204D636F64A4
:1083E00065732074657374205B76315D202A2A2AB8
:1083F0002A290A6735350A6730783079300A6D33B3
:108400000A673470310A6D350A673470310A6D3489
:108410000A673470310A6D350A673470310A6D3776
:108420000A673470310A6D390A673470310A6D3861
:108430000A673470310A6D390A663530300A6730A0
:108440007832300A7932300A6D330A78300A6D3466
:108450000A79300A6D350A67317831300A6D370A8A
:108460007931300A6D380A78300A6D390A79300A64
:108470006732783130792D31306931300A6D330A05
:108480006730783079300A6D340A67337831307963
:108490002D31306931300A6D350A673078307930E6
:1084A0000A6D370A673278323079306931300A6DB7
:1084B000380A6730783079300A6D390A6733783294
:1084C0003079306931300A6730783079300A673274
:1084D000783079306931300A6733783079306931F2
:1084E000300A6735340A6730783079300A6D3330B6
:1084F00000284D53472A2A2A2A2046656564686F5A
:108500006C642054657374205B76315D202A2A2ABE
:108510002A290A284D53472A2A2A2A204D616E7596
:10852000616C6C7920656E746572202120616E64C7
:10853000207E20647572696E67206D6F76656D654B
:108540006E7420746F2074657374202A2A2A2A2975
:108550000A6735350A6730783079300A6734703306
:108560000A67303067313767323167343067343902
:108570006738306739300A663630300A673078310C
:1085800030307637362E3736350A783079300A670C
:1085900035340A6730783079300A6D333000284D31
:1085A00053472A2A2A2A204477656C6C2054657325
:1085B00074205B76315D202A2A2A2A290A67303006
:1085C0006731376732316739300A6735350A6730C6
:1085D000783079300A663530300A67307831300AC1
:1085E000673470310A67307832300A673470310A84
:1085F00067307831300A673470310A67307830304C
:108600000A673470310A79350A6735340A67307879
:108610003079300A6D330A673470310A6730783147
:10862000307931300A6D350A673470310A67307835
:1086300032307932300A6D340A673470310A67306B
:108640007833307933300A6D380A673470310A670D
:10865000307834307934300A6D390A673470310A31
:1086600067307835307935300A6730783079300ABC
:108670006D3330004E31206730306731376732312B
:108680006734306734396738306739300A4E3130F3
:10869000206730783079300A4E32302066353030FD
:1086A0000A4E3330206732783130792D31306931DC
:1086B0003020284357203237302064656772656563
:1086C00073290A4E3430206730783079300A4E35BD
:1086D00030206733783130792D31306931302028BE
:1086E0004343572039302064656772656573290AF2
:1086F0004E3630206730783079300A4E3830206777
:10870000327832307930693130202843572031387F
:10871000302064656772656573290A4E37302067BB
:1087200030783079300A4E383020673378323079FB
:108730003069313020284343572031383020646578
:108740006772656573290A4E393020673078307951
:10875000300A4E39392046313230300A4E3130300D
:1087600020673278307930693230202843572033FF
:1087700036302064656772656573290A4E31313081
:1087800020673278307930693230202843572033DF
:10879000363020616761696E290A4E3132302066B9
:1087A00037303020284368616E67652066656564F0
:1087B0002072617465207768696C6520696E204756
:1087C00032206D6F74696F6E206D6F6465290A4E7B
:1087D00031333020673278307930693230202843A5
:1087E0005720333630203372642074696D65290A4E
:1087F0004E31343020673278307930693230202879
:10880000435720333630203474682074696D6529ED
:108810000A4E31353020663530300A4E3136302040
:108820006733783079307A343069323020284343E6
:108830005720333630206465677265657320776929
:108840007468206C696E6561722074726176656C03
:10885000290A4E313730206733783079307A3069E1
:108860003230202843435720333630206167616916
:108870006E290A4E313830206637303020286D732B
:10888000672A2A2A2A4368616E67652066656564DF
:108890002072617465207768696C6520696E204775
:1088A00033206D6F74696F6E206D6F64652A2A2A9C
:1088B0002A290A4E313930206733783079306932CD
:1088C00030202843435720333630203372642074DD
:1088D000696D65290A4E323030206733783079303F
:1088E00069323020284343572033363020347468AF
:1088F0002074696D65290A4E32313020286D736706
:108900002A2A2A2A473138204576616C20746573FB
:10891000742A2A2A2A290A4E323230204731205816
:1089200033302E373037205A35302E373237204605
:108930003530300A4E32333020473138204730321C
:10894000205836372E373338205A32332E363137C7
:108950002052323520463235300A4E3234302067CC
:1089600038300A4E323530206730783079307A30FE
:108970000A4E323630206D333000284D53472A2AB4
:108980002A2A2053717561726573204D6F74696F67
:108990006E2054657374205B76315D202A2A2A2A62
:1089A000290A6730306731376732316734306734CE
:1089B000396738306739300A6730783079300A677C
:1089C0003078323020287472617665727365206168
:1089D0002032306D6D2073717561726520696E2073
:1089E0005820616E642059290A7932300A78300A99
:1089F00079300A673178313066353030202864723A
:108A0000617720612031306D6D2073717561726501
:108A100020696E205820616E6420592061742046C0
:108A2000353030290A7931300A78300A79300A67CE
:108A3000307A3230202874726176657273652061F5
:108A40002032306D6D2073717561726520696E2002
:108A50005820616E64205A290A7832300A7A300A26
:108A600078300A67317832307932307A3230663590
:108A7000303020286665656420612032306D6D20BD
:108A8000646961676F6E616C20696E20582C205993
:108A900020616E64205A290A783079307A300A7859
:108AA00034307934307A34302028747261766572CB
:108AB000736520612034306D6D20637562652069B7
:108AC0006E20582C205920616E64205A290A78346F
:108AD0003079307A300A78307934307A34300A7824
:108AE00034307934307A300A783079307A34300A58
:108AF00078307934307A300A78343079307A3430DA
:108B00000A783079307A300A6738300A673078303E
:108B100079300A673078310A673078300A6D33303F
:108B200000284D53472A2A2A2A20486F6D696E670C
:108B30002054657374205B76315D202A2A2A2A2905
:108B40000A6732382E32783079307A300A6D333015
:108B500000284D53472A2A2A2A20536D6F6B65201F
:108B600054657374205B76315D202A2A2A2A290AEB
:108B700047303020473137204732312047343020CA
:108B800047343920473830204739300A6D3367344D
:108B900070310A6D35673470310A6D346734703165
:108BA0000A6D33673470310A6D35673470310A6D80
:108BB00037673470310A6D39673470310A6D386740
:108BC0003470310A6D390A6730783079307A300A7A
:108BD000673030207832300A78300A7932300A79BA
:108BE000300A7A32300A7A300A6132300A61300A49
:108BF0004730302078323020793230207A323020BD
:108C00006132300A473030207830207930207A3095
:108C10002061300A473031206633302078322079A5
:108C200032207A322061320A7830207930207A304E
:108C30002061300A673078310A673078300A6D3247
:108C4000002C000A00257300256C750025312E309C
:108C500066002573002C000A0025733A2573002551
:108C6000733A256C750025733A25312E3066002540
:108C7000733A2573005B74765D20207465787420E8
:108C8000766572626F7369747925313564205B3063
:108C90003D73696C656E742C313D766572626F73DD
:108CA000655D0A0025660A00256C750A0025640AC0
:108CB0000025730A0074696E7967205B25735D2057
:108CC0006572723A2025733A202573200074696E0C
:108CD0007967205B25735D206F6B3E2000456E64D5
:108CE000206F6620636F6D6D616E642066696C65D0
:108CF0000A005DC904C7CAC9EBC94ACA49C722CD1F
:108D000004C7B6CD22CE50CC49C70000400640066D
:108D10001040B800B822CD04C7B6CD22CE50CC4901
:108D2000C70000400620060840B800B88BCF04C733
:108D3000ABCE27CFD6D074CEA008400605060901D9
:108D4000088BCF04C7ABCE27CF5CCA49C7B0084059
:108D5000060540B030800000000000F0E0D0C010F8
:108D60000100CF673322211F1B1301016E616E00CA
:108D7000696E66004E414E494E495459494E46CDA2
:108D8000CCCC3D0AD7233C17B7D13877CC2B3295C2
:108D900095E6241FB14F0A000020410000C84200A0
:108DA000401C4620BCBE4CCA1B0E5AAEC59D74006A
:108DB000407A10F35A00A0724E18090010A5D4E8AA
:108DC0000000E87648170000E40B54020000CA9A3D
:108DD0003B000000E1F5050000809698000000408F
:108DE000420F000000A086010000001027000000D4
:108DF00000E803000000006400000000000A00001A
:108E00000000000100000000002C76D888DC674FCD
:108E10000823DFC1DFAE59E1B1B796E5E3E453C6FD
:108E20003AE651997696E8E6C28426EB898C9B62F5
:108E3000ED407C6FFCEFBC9C9F40F2BAA56FA5F49F
:108E400090055A2AF75C936B6CF9676DC11BFCE0C7
:108E5000E40D47FEF520E6B500D0ED902E0300941A
:108E60003577050080841E080000204E0A000000AF
:108E7000C80C333333330F986E12831141EF8D21B9
:108E800014893BE65516CFFEE6DB18D1844B381B20
:108E9000F77C1D901DA4BBE424203284725E2281E5
:108EA00000C9F124ECA1E53D270011241FBECFEF3E
:108EB000CDBFDFE5DEBF00E00CBF13E2A0E0B0E213
:108EC000EAEAF8EC01E00BBF02C007900D92A63869
:108ED000B107D9F729E5A6E8B3E201C01D92A03E8B
:108EE000B207E1F70E942D800C9453E40C9400002B
:108EF000FC0160817181828193810E9424D66093FC
:108F0000AD320895FC0160817181828193810E945C
:108F100024D66093AC320895AF92BF92CF92DF9285
:108F2000EF92FF920F931F93CF93DF937B018C01FE
:108F300080E3C82E82E3D82EE601AA24A394BC2E97
:108F4000BC18F70161917191819191917F012CEA97
:108F500035EC47E257E30E94B3D718164CF4F801FA
:108F600040815181628173818B2D0E949B81A882F7
:108F70000C5F1F4F2196F2E3C633DF0701F7DF9145
:108F8000CF911F910F91FF90EF90DF90CF90BF9006
:108F9000AF900C94A681FC016081718182819381E4
:108FA0000E9424D66093AE32613019F481E00E94B1
:108FB000A27781E00C94C377CF93DF93CDB7DEB770
:108FC0006897CDBFDEBFFC01608171818281938192
:108FD0000E9424D66093AF3281E0613019F40E9480
:108FE000A2770CC00E94C377CE01019628E1FC0154
:108FF00011922A95E9F7BC010E94CB476896CDBF34
:10900000DEBFDF91CF9108950F931F93CF93DF932E
:10901000CDB7DEB72D97CDBFDEBF27E0E8EDF0E29C
:109020008E010F5F1F4FD80101900D922A95E1F735
:10903000BC01660F771F680F791F660F771F660FD9
:10904000771F660F771F68567A4E45E050E0CE01D5
:1090500008960E94C3E1688570E0C8010E94F1E1B2
:10906000009739F46B8570E0C8010E94F1E1009728
:1090700011F0801B01C08FEF2D96CDBFDEBFDF91B9
:10908000CF911F910F910895EF92FF920F931F932D
:10909000CF93DF938C01F62EE72EEC012D96FC0189
:1090A00061857285838594850E9424D61F926F9373
:1090B000DF93CF930F5E1F4F1F930F93DF93CF93D9
:1090C000EF92FF92ECEDF9E581818F9380818F9390
:1090D0000E948AE2EDB7FEB73C96EDBFFEBFDF917E
:1090E000CF911F910F91FF90EF9008950F931F93D1
:1090F000CF93DF93EC01162F072F8C819D810E9467
:10910000044883305CF58F3FA1F528C09E01235FA2
:109110003F4F9F938F938C858F938B858F938A85F9
:109120008F9389858F933F932F936196DF93CF938E
:109130003F932F930F931F938091DD598F938091CD
:10914000DC598F930E948AE28DB79EB740968DBFFF
:109150009EBFDF91CF911F910F910895E7E1F4E158
:10916000659174914FE450E084ED9CE30E94C3E16B
:10917000CDCFE091A632F0E0EE0FFF1FED5EFB4E8B
:10918000659174914FE450E084ED9CE30E94C3E14B
:10919000BDCF0F931F93CF93DF93EC01162F072FB3
:1091A0008C819D810E94044883307CF58F3FC1F5FE
:1091B0002CC0AE014F5E5F4F9E01235F3F4F9F93D8
:1091C0008F938C858F938B858F938A858F938985D9
:1091D0008F935F934F933F932F935F934F933F935F
:1091E0002F930F931F938091DD598F938091DC59BA
:1091F0008F930E948AE28DB79EB742968DBF9EBF25
:10920000DF91CF911F910F910895E7E1F4E165910E
:1092100074914FE450E084ED9CE30E94C3E1C9CF18
:10922000E091A632F0E0EE0FFF1FED5EFB4E659180
:1092300074914FE450E084ED9CE30E94C3E1B9CF08
:10924000DF92EF92FF920F931F93CF93DF93CDB7EF
:10925000DEB72897CDBFDEBF8B01E42ED52E37E0D9
:10926000EFEDF0E2DE01119601900D923A95E1F7F3
:1092700028870E940448F82E288582E08F1518F070
:10928000E22FF0E002C0E2E0F0E0EE0FFF1FED5E43
:10929000FB4E659174914FE450E084ED9CE30E9495
:1092A000C3E19F938F93F80183818F9382818F9382
:1092B00081818F9380818F93E1E0F0E0EC0FFD1FBF
:1092C000EF0DF11D80811F928F93DF92EF928091BD
:1092D000DD598F938091DC598F930E948AE2CDBF34
:1092E000DEBF2896CDBFDEBFDF91CF911F910F91DA
:1092F000FF90EF90DF9008954F925F926F927F9270
:10930000AF92BF92CF92DF92EF92FF920F931F9393
:10931000CF93DF93C0E3D2E305EF10E35C018991C3
:10932000813009F042C0F801C480D580E680F78022
:109330004080518062807380A3019201C701B60111
:109340000E9407D49F772CEA35EC47E257E30E944E
:10935000B0D587FD2AC020E034E244E759ECC701CC
:10936000B6010E94B3D718165CF4F5012081318153
:1093700042815381C701B6010E94B3D7181604F188
:1093800020E034E244E759ECC301B2010E94B3D7B4
:1093900018165CF4F5012081318142815381C301AB
:1093A000B2010E94B0D587FD0BC00B5C1F4FF4E0EB
:1093B000AF0EB11C82E3C633D80709F0B0CF02C0AC
:1093C0008CED01C080E0DF91CF911F910F91FF9054
:1093D000EF90DF90CF90BF90AF907F906F905F90B5
:1093E0004F90089580912C32811105C080912B32CD
:1093F00080932A3229C0823031F487E080932A3268
:1094000080912B3221C0833031F489E080932A325D
:1094100080912B3219C0843031F48AE080932A3253
:1094200080912B3211C080912D32813031F485E052
:1094300080932A3280912B3207C0823019F486E063
:1094400080932A3280912B32863019F080912A3213
:1094500008958BE080932A32089580912B320895ED
:1094600080932D32813059F018F0823041F0089508
:109470008BE592E38093593290935A32089583E2B8
:1094800096E58093593290935A320895FC01848175
:109490000895845B9F4FFC0180810895855B9F4FF9
:1094A000FC0180810895825B9F4FFC0180810895BB
:1094B000815B9F4FFC0180810895875B9F4FFC017A
:1094C000808108950C949C96CD96FC0160817181F9
:1094D000828193810895FC01648308958B5A9F4F84
:1094E000FC01608308958F5B9F4FFC014083518393
:1094F00062837383089560935B3270935C328093D0
:109500005D3290935E3280EE91E20C94E461BF9202
:10951000CF92DF92EF92FF920F931F93CF93DF933F
:10952000D090A8327C010DEC12E38091A73290E03C
:10953000EC01CC0FDD1FC80FD91FCC0FDD1FCC0FE6
:10954000DD1FCC0FDD1FCC5BDF4C81E0D816A9F00E
:10955000B881A981CA80BB8040912033413091F409
:10956000F80120813181428153816B2F7A2F8C2D1C
:109570009B2D0E9408D49B0109C020E030E080E0D0
:1095800090E004C02B2F3A2F8C2D9B2DA901BC01FC
:10959000F701458F568F678F70A3F4E0EF0EF11C33
:1095A0000C5F1F4F249682E3053E180771F6DF918A
:1095B000CF911F910F91FF90EF90DF90CF90BF90D0
:1095C0000895835B9F4FFC0160838BE592E30C94CD
:1095D000874A4F925F926F927F928F929F92AF9243
:1095E000BF92CF92DF92EF92FF920F931F93CF9390
:1095F000DF93CDB7DEB76897CDBFDEBF8C0160913A
:10960000203370E080E090E00E9452D62B013C01B4
:10961000F80160817181828193810E9424D670E07B
:109620005B01AA0CBB1CA60EB71EAA0CBB1CAA0C85
:10963000BB1CAA0CBB1CC5018C5B9F4C5C010DECD8
:1096400012E3FE0131964F01F501C190D190E190F6
:10965000F1905F01F80161917191819191918F0178
:10966000A30192010E9455D89B01AC01C701B6012C
:109670000E9408D4F40161937193819391934F01F7
:10968000F2E3053E1F0701F7CE0101960E947F9687
:109690008BE592E30E94874A6896CDBFDEBFDF91DB
:1096A000CF911F910F91FF90EF90DF90CF90BF90DF
:1096B000AF909F908F907F906F905F904F900895A4
:1096C0008B55924369F4E62FF0E0EE0FFF1FEE0F8B
:1096D000FF1FEB54FD4C608171818281938108955D
:1096E000862F0C947496CF92DF92EF92FF920F9395
:1096F0001F93CF93DF93EC0182E3CB35D80709F0BA
:109700004AC070E0FB01EE0FFF1FEE0FFF1FEB548E
:10971000FD4CC080D180E280F3808091A8328130FE
:1097200059F18091A73290E0FC01EE0FFF1FE80F86
:10973000F91FEE0FFF1FE60FF71FEE0FFF1FEE0FD3
:10974000FF1FEC5BFF4C00811181B281A38120914E
:1097500020332130B1F4FB01EE0FFF1FEE0FFF1F8E
:10976000E353FD4C2081318142815381B8018B2F1D
:109770009A2F0E9408D408C060E070E080E090E07A
:1097800003C0B8018B2F9A2F9B01AC01C701B60112
:109790000E9407D403C0862F0E948896C55BDF4FC6
:1097A0002881211106C023E333E34BEC51E40E94EE
:1097B000B7D5DF91CF911F910F91FF90EF90DF9080
:1097C000CF90089588E1E0E6F2E3A5EBB2E30190E3
:1097D0000D928A95E1F78091A43281110CC080919D
:1097E0005F32813041F41092983210929932109287
:1097F0009A3210929B3208954F925F926F927F92AD
:109800008F929F92AF92BF92CF92DF92EF92FF9290
:109810000F931F93CF93DF93CDB7DEB76997CDBF7B
:10982000DEBF80912C32811155C080915132813040
:1098300009F050C00E94A3C681114CC01092513251
:109840009CE5692E90E3792E26E3822E912C8E01E1
:109850000E5E1F4F36EEA32E30E2B32E33C0F7015B
:1098600081917F011F928F935F924F92BF92AF922F
:109870001F930F930E9455E3B80184E493E20E9482
:10988000495F8D839E83F60181919191A191B19160
:109890006F018A879B87AC87BD87CE0101960E94A6
:1098A000385CCDBFDEBF9EEDE91690E2F906B9F651
:1098B000E8E16E0E711CFFEF8F1A9F0A8CE3881689
:1098C000910441F0240189EDE82E80E2F82E630135
:1098D00088E7C8CF80E06996CDBFDEBFDF91CF912A
:1098E0001F910F91FF90EF90DF90CF90BF90AF90BE
:1098F0009F908F907F906F905F904F9008952F92E0
:109900003F924F925F926F927F928F929F92AF920F
:10991000BF92CF92DF92EF92FF920F931F93CF935C
:10992000DF93CDB7DEB72997CDBFDEBF4C015B011A
:109930004090AA325090A8322090A73260902033F5
:109940007090A6326B0180E692E3888799875CEE7F
:10995000E52E50E3F52E98E1299E10011124840193
:10996000D6016D917D918D919D916D012CEA35EC23
:1099700047E257E30E94B0D587FD80C0F7018081A0
:109980008150823008F07AC041104CC0F1E05F167F
:1099900009F1E885F985E20DF31DEC51F240808173
:1099A000898391819D83B281A381E1E06E1217C00A
:1099B000E885F985E359FF4F208131814281538148
:1099C000BC018B2F9A2F0E9408D469837D838E83DC
:1099D0009F8307C019821D821E821F8202C0BE8320
:1099E000AF8371100CC023E333E34BEC51E4D80197
:1099F0006D917D918D919C910E9455D805C0F80183
:109A0000608171818281938129813D814E815F8155
:109A10000E9408D4A885B9856D937D938D939C93FE
:109A200013972CC0A885B9858D919D910D90BC91FF
:109A3000A02D89839A83AB83BC8371100EC023E36E
:109A400033E34BEC51E4F8016081718182819381B1
:109A50000E9455D89B01AC0105C0D8012D913D91C4
:109A60004D915C9169817A818B819C810E9408D49F
:109A7000E885F985608371838283938388859985DE
:109A800004968887998795E3E90EF11C0C5F1F4FB8
:109A9000A885B985AC56B24309F062CF6090A63272
:109AA0007090AA32F091A832F983C090A732209129
:109AB00020332D838CE0A80EB11CABE8B1E3A8875E
:109AC000B9874CE6E42E42E3F42EB8E1CB9E600168
:109AD00011248401F50161917191819191915F014E
:109AE0002CEA35EC47E257E30E94B0D587FD8CC0E5
:109AF000A885B9858C91882309F486C0815082306D
:109B000030F4F80124843584468457843BC06110C6
:109B100016C023E333E34BEC51E4D8011C966D915E
:109B20007D918D919C911F970E9455D820E030E047
:109B300044EB53E40E9455D81B012C010DC020E0DA
:109B400030E044EB53E4F80164857585868597859C
:109B50000E9455D81B012C012BED3FE049EC50E44D
:109B6000A885B98591966D917D918D919C919497E1
:109B70000E9455D89B01AC01C201B1010E94B7D52A
:109B80001B012C01711031C0B981B130E1F0F70136
:109B9000EC0DFD1DEC51F240A081B18192808380DB
:109BA000ED81E130A1F4F701E359FF4F20813181CC
:109BB00042815381BD01892D982D0E9408D4DB017B
:109BC000982E892E04C0A0E0B0E0912C812CA20137
:109BD0009101BD01892D982D0E9408D4D7016D9364
:109BE0007D938D939C9313970FC0A2019101F70170
:109BF00060817181828193810E9408D4D7016D9325
:109C00007D938D939C931397E885F985F596E88766
:109C1000F987F4E0EF0EF11C0C5F1F4F88859985E2
:109C20008A52924309F056CF2996CDBFDEBFDF910D
:109C3000CF911F910F91FF90EF90DF90CF90BF9049
:109C4000AF909F908F907F906F905F904F903F90DC
:109C50002F90089580912830909129308F3E924125
:109C600011F08FE508958091DF339091E0338F3EBE
:109C70009241B9F78091B1329091B2328F3E9241C8
:109C800081F780912733909128338F3E924149F795
:109C900080917B5690917C568F3E924111F7809136
:109CA0003857909139578F3E9241D9F680E0089508
:109CB000CF93C82F0E949FA782E080932B328C2FD6
:109CC000CF91089580912C32811104C083E080935C
:109CD0002B3203C085E080932B3280E00895CF9330
:109CE000C82F0E9410B380E00E94B1AE8C2F0E945A
:109CF0009FA786E080932B328C2FCF91089580937D
:109D0000A53280E008958093A63280E00895809384
:109D1000AA3280E008954F925F926F927F929F9255
:109D2000AF92BF92CF92DF92EF92FF920F931F9369
:109D3000CF93DF93C82FB62E8A01F22ED32F8FEF49
:109D40008C0F863008F082C06091B33370E080E001
:109D500090E00E9452D62CEA35EC47E257E30E948D
:109D6000B0D587FD75C082E0B81619F0E4E1BE12E7
:109D700071C09090A632CF2CDD2E8C2F90E0EC019C
:109D8000CC0FDD1FC80FD91FCC0FDD1FCC0FDD1F7F
:109D9000CC0FDD1FCC5BDF4C780105EB12E3AA246E
:109DA000A394F60161917191819191916F012CEAD7
:109DB00035EC47E257E30E94B3D71816DCF5F2E022
:109DC000BF1214C091100CC023E333E34BEC51E4F9
:109DD000F70160817181828193810E9455D824C0EE
:109DE000F70160817181828193811EC0F8014080FA
:109DF00051806280738091100EC023E333E34BECFB
:109E000051E4F70160817181828193810E9455D86C
:109E10009B01AC0105C0F701208131814281538152
:109E2000C301B2010E9407D4688379838A839B832C
:109E3000A09251322496F4E0EF0EF11C0C5F1F4FFC
:109E400082E30D3C180709F0ACCF06C081EA05C0DB
:109E50008CEA03C08DEA01C080E0DF91CF911F91B1
:109E60000F91FF90EF90DF90CF90BF90AF909F90B9
:109E70007F906F905F904F900895CF93DF93CDB711
:109E8000DEB76897CDBFDEBF8093A732682F70E042
:109E900080E090E00E9450D669837A838B839C8314
:109EA0001D821E821F82188619861A861B861C86B2
:109EB0001D861E861F86188A198A1A8A1B8A1C8A82
:109EC0001D8A1E8A1F8A188EAE014F5F5F4FBA012E
:109ED00089EE9AE40E94DD8280E06896CDBFDEBF05
:109EE000DF91CF910895CF93DF93EBE5F2E386E521
:109EF000DF011D928A95E9F78BE5A9E2B3E3ED0155
:109F0000982F19929A95E9F7A4E8B3E3ED01199215
:109F10008A95E9F78FEE92E180932830909329306B
:109F20008093DF339093E0338093B1329093B232D9
:109F3000809327339093283380937B5690937C565D
:109F40008093385790933957E0935932F0935A32AF
:109F5000809141308093A63280913F300E943D4FE6
:109F6000809140308093A532809142308093A93215
:109F7000809143308093AA3281E08093A432809311
:109F8000213394E090935F32109252321092533208
:109F90001092543280932B3280932A320E944FAD1C
:109FA000DF91CF910C941F84CF92DF92EF92FF92BA
:109FB000CF93C82F6A017B01E82FF0E0DF01AA0FE1
:109FC000BB1FAA0FBB1FAB54BD4C4D935D936D934C
:109FD0007C931397EE0FFF1FEE0FFF1FE05AFD4C0F
:109FE00040835183628373838C2F0E949081B701D9
:109FF000A6018C2F0E949B81CF91FF90EF90DF9064
:10A00000CF900C94A6819F92AF92BF92CF92DF9295
:10A01000EF92FF920F931F93CF93DF93CDB7DEB7ED
:10A020006897CDBFDEBF962EA72EC62ED72E7C01F9
:10A0300000E010E0B12CF601619171918191919154
:10A040006F012CEA35EC47E257E30E94B3D71816AC
:10A05000A4F58091A63281110EC023E333E34BECCB
:10A0600051E4F70160817181828193810E9455D80A
:10A07000AB01BC0105C0F701408151816281738150
:10A08000E1E0F0E0EC0FFD1FE00FF11F4083518392
:10A0900062837383C801885D9F4CFC01E357FD4FC9
:10A0A0004083518362837383E555F1094083518373
:10A0B000628373838B2D0E949081B3940C5F1F4F3A
:10A0C000F4E0EF0EF11C0831110509F0B4CF492D71
:10A0D0005A2DBE016F5F7F4F8CE897E40E94DD82AE
:10A0E00080E06896CDBFDEBFDF91CF911F910F91C9
:10A0F000FF90EF90DF90CF90BF90AF909F9008952A
:10A100004F925F926F927F928F929F92AF92BF9287
:10A11000CF92DF92EF92FF920F931F93CF93DF9333
:10A12000CDB7DEB76897CDBFDEBF21E020932033E7
:10A130008090A7329090A6325B016C0105EB12E390
:10A14000882D90E07C01EE0CFF1CE80EF91EEE0C51
:10A15000FF1CEE0CFF1CEE0CFF1CC7018C5B9F4C20
:10A160007C01F50161917191819191915F012CEADE
:10A1700035EC47E257E30E94B3D7181664F5F701B0
:10A180002081318142815381F80160817181828116
:10A1900093810E9407D42B013C0191100EC023E350
:10A1A00033E34BEC51E4F60160817181828193814C
:10A1B0000E9455D89B01AC0105C0F6012081318178
:10A1C00042815381C301B2010E9407D4F801608F1C
:10A1D000718F828F938FF4E0CF0ED11C0C5F1F4FD5
:10A1E00084E0E80EF11C92E30D3C190709F0B9CFA9
:10A1F000682D70E080E090E00E9450D669837A83F9
:10A200008B839C831D821E821F82188619861A8664
:10A210001B861C861D861E861F86188A198A1A8A26
:10A220001B8A1C8A1D8A1E8A1F8A188EAE014F5FE8
:10A230005F4FBA0189EE9AE40E94DD8280E0689661
:10A24000CDBFDEBFDF91CF911F910F91FF90EF90B7
:10A25000DF90CF90BF90AF909F908F907F906F9046
:10A260005F904F900895CF93DF93CDB7DEB7689797
:10A27000CDBFDEBF109220331092CD321092CE327D
:10A280001092CF321092D0321092D1321092D2323C
:10A290001092D3321092D4321092D5321092D6321C
:10A2A0001092D7321092D8321092D9321092DA32FC
:10A2B0001092DB321092DC321092DD321092DE32DC
:10A2C0001092DF321092E0321092E1321092E232BC
:10A2D0001092E3321092E4326091A73270E080E095
:10A2E00090E00E9450D669837A838B839C831D8281
:10A2F0001E821F82188619861A861B861C861D865A
:10A300001E861F86188A198A1A8A1B8A1C8A1D8A29
:10A310001E8A1F8A188EAE014F5F5F4FBA0189EE09
:10A320009AE40E94DD8280E06896CDBFDEBFDF91B7
:10A33000CF910895CF93DF93CDB7DEB76897CDBFA8
:10A34000DEBF109220336091A73270E080E090E091
:10A350000E9450D669837A838B839C831D821E82E0
:10A360001F82188619861A861B861C861D861E86E5
:10A370001F86188A198A1A8A1B8A1C8A1D8A1E8AB5
:10A380001F8A188EAE014F5F5F4FBA0189EE9AE4C3
:10A390000E94DD8280E06896CDBFDEBFDF91CF9165
:10A3A0000895CF93DF93CDB7DEB76897CDBFDEBFFB
:10A3B00081E0809320336091A73270E080E090E0EC
:10A3C0000E9450D669837A838B839C831D821E8270
:10A3D0001F82188619861A861B861C861D861E8675
:10A3E0001F86188A198A1A8A1B8A1C8A1D8A1E8A45
:10A3F0001F8A188EAE014F5F5F4FBA0189EE9AE453
:10A400000E94DD8280E06896CDBFDEBFDF91CF91F4
:10A410000895CF9310925F320E947F4C809132302A
:10A42000813069F480E692E30E947C49C82F88233A
:10A4300031F00E949FA782E080932B3217C08BE5FA
:10A4400092E30E94874A85E080932B3280912C32E0
:10A45000811105C081E080932C320E94B2AB8BE564
:10A4600092E30E94A9960E94E24BC0E08C2FCF910C
:10A47000089588E1E5EBF2E3A5EEB2E301900D92D9
:10A480008A95E1F780E008950F931F93CF93DF93B0
:10A49000CDB7DEB76A97CDBFDEBF8C0181E0809378
:10A4A000A8328BE592E3698F7A8F0E94874A698D83
:10A4B0007A8DC8010E9409520E9417828823E1F315
:10A4C00088E1E0E0F0E2DE01119601900D928A95BC
:10A4D000E1F7BE016F5F7F4F85EE92E30E94095264
:10A4E0006A96CDBFDEBFDF91CF911F910F91089586
:10A4F00088E1E5EBF2E3ADEFB2E301900D928A95CE
:10A50000E1F780E008950F931F93CF93DF93CDB7CA
:10A51000DEB76A97CDBFDEBF8C0181E08093A832A1
:10A520008BE592E3698F7A8F0E94874A698D7A8DD5
:10A53000C8010E9409520E9417828823E1F388E132
:10A54000E0E0F0E2DE01119601900D928A95E1F7CC
:10A55000BE016F5F7F4F8DEF92E30E9409526A96B2
:10A56000CDBFDEBFDF91CF911F910F910895FB0109
:10A57000DC018091A432811111C09B01AD0160E02A
:10A5800070E080E89FE30E94B7D5609398327093A3
:10A59000993280939A3290939B3218C08091A63260
:10A5A000811109C023E333E34BEC51E4CD010E9458
:10A5B00055D8FB0101C0CD01AF01BC0140939832D9
:10A5C0005093993260939A3270939B3280E0089551
:10A5D0008093A43280E008958093A93280E00895AA
:10A5E0006093A0327093A1328093A2329093A332F1
:10A5F0000E94358380E008950F931F93CF93DF93DC
:10A60000EC018B018091A432882399F080919832DB
:10A6100090919932A0919A32B0919B32BC01CD01B8
:10A620009F772CEA35EC47E257E30E94B0D587FDCF
:10A6300030C081E080935F32B801CE010E947F4C30
:10A6400080913230813069F480E692E30E947C4947
:10A65000C82F882331F00E949FA782E080932B327D
:10A6600019C08BE592E30E94874A85E080932B32E4
:10A6700080912C32811105C081E080932C320E94A0
:10A68000B2AB8BE592E30E94A996C82F0E94E24BE1
:10A6900001C0CEE88C2FDF91CF911F910F910895CB
:10A6A000CF93DF93CDB7DEB76897CDBFDEBF682FFE
:10A6B00070E080E090E00E9450D669837A838B83BB
:10A6C0009C831D821E821F82188619861A861B860D
:10A6D0001C861D861E861F86188A198A1A8A1B8A5E
:10A6E0001C8A1D8A1E8A1F8A188EAE014F5F5F4F1B
:10A6F000BA0188E797E40E94DD8280E06896CDBFCA
:10A70000DEBFDF91CF910895CF93DF93CDB7DEB752
:10A710006897CDBFDEBF6091AD3270E080E090E021
:10A720000E9450D669837A838B839C831D821E820C
:10A730001F82188619861A861B861C861D861E8611
:10A740001F86188A198A1A8A1B8A1C8A1D8A1E8AE1
:10A750001F8A188EAE014F5F5F4FBA0182E897E4FF
:10A760000E94DD8280E06896CDBFDEBFDF91CF9191
:10A770000895CF93DF93CDB7DEB76897CDBFDEBF27
:10A78000682F70E080E090E00E9450D669837A8361
:10A790008B839C831D821E821F82188619861A86CF
:10A7A0001B861C861D861E861F86188A198A1A8A91
:10A7B0001B8A1C8A1D8A1E8A1F8A188EAE014F5F53
:10A7C0005F4FBA018BEC97E40E94DD8280E06896CF
:10A7D000CDBFDEBFDF91CF910895CF93DF93CDB78B
:10A7E000DEB76897CDBFDEBF682F70E080E090E0F5
:10A7F0000E9450D669837A838B839C831D821E823C
:10A800001F82188619861A861B861C861D861E8640
:10A810001F86188A198A1A8A1B8A1C8A1D8A1E8A10
:10A820001F8A188EAE014F5F5F4FBA018CED97E41F
:10A830000E94DD8280E06896CDBFDEBFDF91CF91C0
:10A840000895CF93FC0160817181828193810E9480
:10A8500024D660932B3210922D328BE592E38093B5
:10A86000593290935A3280912C32813011F41092E7
:10A870002C3210922E32109254320E946296C09165
:10A880002B32C430C9F40E94335180913F300E9472
:10A890003D4F809140308093A5328091433080932A
:10A8A000AA3280E00E94B1AE80E00E94ED5381E0C8
:10A8B0008093A432C0935F3281E0CF910C9476AA4A
:10A8C00080931D3380931E338093263380E0089558
:10A8D0002CEA35EC47E257E36091CB337091CC33EF
:10A8E0008091CD339091CE330E94B3D71816B4F433
:10A8F0008091703390917133A0917233B091733322
:10A90000BC01CD019F772CEA35EC47E257E30E946A
:10A91000B0D587FF03C010921D3303C081E0809340
:10A920001D3380E0089580931D33809170339091A2
:10A930007133A0917233B091733380931533909338
:10A940001633A0931733B093183380E008952CEAA0
:10A9500035EC47E257E36091CB337091CC33809173
:10A96000CD339091CE330E94B3D71816B4F48091B2
:10A97000703390917133A0917233B0917333BC01F5
:10A98000CD019F772CEA35EC47E257E30E94B0D522
:10A9900087FF03C010921E3303C081E080931E33F3
:10A9A00080E0089580931E338091703390917133CD
:10A9B000A0917233B09173338093193390931A330B
:10A9C000A0931B33B0931C3380E008952CEA35EC40
:10A9D00047E257E36091CB337091CC338091CD3314
:10A9E0009091CE330E94B3D71816B4F4809170338F
:10A9F00090917133A0917233B0917333BC01CD014A
:10AA00009F772CEA35EC47E257E30E94B0D587FFE9
:10AA100003C01092263303C081E08093263380E088
:10AA20000895809326338091703390917133A09173
:10AA30007233B09173338093223390932333A09376
:10AA40002433B093253380E00895BC018DEE90E26D
:10AA50000C94076281E080935232089581E08093E4
:10AA60005332089581E08093543208951F93CF9319
:10AA7000DF93CDB7DEB76897CDBFDEBF0E949C964F
:10AA80008130C9F10E944ED20E9452C90E949A821E
:10AA900080E00E94C7AB10E0812F0E947496AB014A
:10AAA000BC01812F0E94D44F1F5F1630A9F780E0B0
:10AAB00090E0A0E4B0E489839A83AB83BC831D82D9
:10AAC0001E821F82188619861A861B861C861D8682
:10AAD0001E861F86188A198A1A8A1B8A1C8A1D8A52
:10AAE0001E8A1F8A188EBE016F5F7F4FCB010E94A6
:10AAF000215480E001C08AE66896CDBFDEBFDF91B9
:10AB0000CF911F910895809152328130A9F4209104
:10AB10002D32213079F480912E3281110BC082E0E8
:10AB200080932D3283E296E58093593290935A3286
:10AB300020932E321092523280915332813091F410
:10AB400080912D32882331F0823061F490912E3241
:10AB5000943051F40E949C96811104C0109253329B
:10AB60000E94365590912E32809154328130C1F43A
:10AB700020915332211114C09150933088F01092DB
:10AB8000543295E090932E3290932B3290912C3248
:10AB9000911104C080932C320E94B2AB0E940E9F90
:10ABA00080E0089585E080932B3280912C328111D2
:10ABB00005C081E080932C320C94B2AB0895CF9302
:10ABC000DF93CDB7DEB76897CDBFDEBF80912C3263
:10ABD000882311F180E090E0A0E4B0E489839A83B7
:10ABE000AB83BC831D821E821F82188619861A863B
:10ABF0001B861C861D861E861F86188A198A1A8A3D
:10AC00001B8A1C8A1D8A1E8A1F8A188EBE016F5FCE
:10AC10007F4FCB010E9421546896CDBFDEBFDF91EC
:10AC2000CF910895CF93DF93CDB7DEB76897CDBFAF
:10AC3000DEBF80E090E0A0E4B0E489839A83AB8338
:10AC4000BC831D821E821F82188619861A861B8667
:10AC50001C861D861E861F86188A198A1A8A1B8AD8
:10AC60001C8A1D8A1E8A1F8A188EAE014F5F5F4F95
:10AC7000BA0181E294E50E94DD826896CDBFDEBF15
:10AC8000DF91CF910895CF93DF93CDB7DEB768976B
:10AC9000CDBFDEBF80E090E0A0E8B0E489839A8376
:10ACA000AB83BC831D821E821F82188619861A867A
:10ACB0001B861C861D861E861F86188A198A1A8A7C
:10ACC0001B8A1C8A1D8A1E8A1F8A188EAE014F5F3E
:10ACD0005F4FBA0181E294E50E94DD826896CDBFA4
:10ACE000DEBFDF91CF910895CF93DF93CDB7DEB76D
:10ACF0002797CDBFDEBF97E0EFEDF0E2DE011196C2
:10AD000001900D929A95E1F7873050F4E1E0F0E080
:10AD1000EC0FFD1FE80FF11D87FDFA95808101C042
:10AD200080E22796CDBFDEBFDF91CF910895EF92ED
:10AD3000FF920F931F93CF93DF931F92CDB7DEB790
:10AD40007C018B01642F70E080E090E049830E94D9
:10AD500050D6F701618772878387948782E0878363
:10AD60004981E42FF0E0EE0FFF1FE00FF11F659126
:10AD700074914FE450E084ED9CE30E94C3E1BC0178
:10AD8000C7010F90DF91CF911F910F91FF90EF902E
:10AD90000C94A961CF93DF93EC010E94F249482FF4
:10ADA00061E573E1CE01DF91CF910C94975640910C
:10ADB0002B3262E173E10C94975640912C3269EE8C
:10ADC00072E10C94975640912D3265ED72E10C942E
:10ADD000975640912E3267EA72E10C949756409153
:10ADE0002F326AE872E10C949756E0915932F09153
:10ADF0005A32E55BFF4F408164EB73E10C94975648
:10AE0000E0915932F0915A32E45BFF4F408160EC9F
:10AE100071E10C949756E0915932F0915A32448185
:10AE200066E271E10C949756E0915932F0915A32F2
:10AE3000E65BFF4F408163EF70E10C949756E09121
:10AE40005932F0915A32E25BFF4F408169EA70E17A
:10AE50000C949756E0915932F0915A32E15BFF4FD2
:10AE6000408168E670E10C949756E0915932F09178
:10AE70005A32E75BFF4F408169EF7FE00C949756B1
:10AE8000CF93DF93EC01E0915932F0915A32EF5AAF
:10AE9000FF4F608170E080E090E00E9450D66987AB
:10AEA0007A878B879C8782E08F8380E0DF91CF91C8
:10AEB0000895CF93DF93EC0160915B3270915C3227
:10AEC00080915D3290915E320E9450D669877A8778
:10AED0008B879C8782E08F8380E0DF91CF910895FC
:10AEE000CF93DF93EC01E0915932F0915A326081B7
:10AEF0007181828193810E9450D669877A878B877E
:10AF00009C8782E08F8380E0DF91CF910895CF937B
:10AF1000DF93EC0180912D32811105C019861A86CC
:10AF20001B861C8614C00E946B9669877A878B8764
:10AF30009C8720916E5621110AC025E832E441E237
:10AF40005DE30E9455D869877A878B879C878C81BF
:10AF50009D81FC01EE0FFF1FE80FF91FEE0FFF1F91
:10AF6000EE0FFF1FEE0FFF1FE156FA4E85919491F1
:10AF7000888784E08F8380E0DF91CF910895CF931D
:10AF8000DF93EC012091593230915A32F901FD964C
:10AF9000608171818281938169877A878B879C87A1
:10AFA0003E96208121110AC025E832E441E25DE3AA
:10AFB0000E9455D869877A878B879C878C819D8171
:10AFC000FC01EE0FFF1FE80FF91FEE0FFF1FEE0F42
:10AFD000FF1FEE0FFF1FE156FA4E8591949188876F
:10AFE00084E08F8380E0DF91CF910895CF93DF934A
:10AFF000EC018C819D810E940448682F8091593218
:10B0000090915A320E94734B69877A878B879C870D
:10B010008C819D81FC01EE0FFF1FE80FF91FEE0FE1
:10B02000FF1FEE0FFF1FEE0FFF1FE156FA4E859137
:10B030009491888784E08F8380E0DF91CF91089599
:10B04000CF93DF93EC018C819D810E940448209175
:10B05000593230915A322B55324369F4E82FF0E0DF
:10B06000EE0FFF1FEE0FFF1FEB54FD4C608171814F
:10B070008281938102C00E94749669877A878B8748
:10B080009C878C819D81FC01EE0FFF1FE80FF91F4B
:10B09000EE0FFF1FEE0FFF1FEE0FFF1FE156FA4EE0
:10B0A00085919491888784E08F8380E0DF91CF91B0
:10B0B0000895CF93DF93EC018C819D810E94044819
:10B0C000E0915932F0915A3294E0899FE00DF11DE0
:10B0D0001124458D568D678D70A149875A876B87DE
:10B0E0007C878C819D81FC01EE0FFF1FE80FF91F0B
:10B0F000EE0FFF1FEE0FFF1FEE0FFF1FE156FA4E80
:10B1000085919491888784E08F8380E0DF91CF914F
:10B110000895CF93DF93EC010E941C5D69857A85C9
:10B120008B859C850E9424D6462F60EE73E1CE016C
:10B13000DF91CF910C949756CF93DF93EC018C81E4
:10B140009D810E940448833054F48F3FA9F407C0C6
:10B15000CE010E94C65D80E01CC08DE61AC020E0D2
:10B1600030E040E450E469857A858B859C850E94B7
:10B17000B3D7181694F3ECCF20E030E040E050E471
:10B1800069857A858B859C850E94B3D718162CF328
:10B19000DFCFDF91CF91089595E3899FF0011124CE
:10B1A000E350FF4C60817181828193810895CF9239
:10B1B000DF92EF92FF92CF93DF936A017B0125E349
:10B1C000829FC0011124885D9F4CFC01EB52FF4F10
:10B1D0004083518362837383EC01C352DF4F20E0CD
:10B1E00034E244E759E4C701B6010E9455D89B01F7
:10B1F000AC0160E070E080E89FE30E94B7D568830F
:10B2000079838A839B83DF91CF91FF90EF90DF90CA
:10B21000CF900895CF92DF92EF92FF92CF93DF937A
:10B22000EC01C984DA84EB84FC8420E034E244E756
:10B2300059E4C701B6010E94B3D7181664F420E0A0
:10B2400034E244E759E4C701B6010E94B7D56987E3
:10B250007A878B879C87CE010E94C362C984DA8477
:10B26000EB84FC848C819D810E94044825E3829FAD
:10B27000C0011124885D9F4CFC01EB52FF4FC0823E
:10B28000D182E282F382EC01C352DF4F20E034E24C
:10B2900044E759E4C701B6010E9455D89B01AC01AF
:10B2A00060E070E080E89FE30E94B7D5688379830F
:10B2B0008A839B8380E0DF91CF91FF90EF90DF90B6
:10B2C000CF900895CF92DF92EF92FF92CF93DF93CA
:10B2D000EC01C984DA84EB84FC8420E034E244E7A6
:10B2E00059E4C701B6010E94B3D7181664F420E0F0
:10B2F00034E244E759E4C701B6010E94B7D5698733
:10B300007A878B879C87CE010E94C36280E0DF91A1
:10B31000CF91FF90EF90DF90CF90089581E08093E0
:10B32000533280E008952CEA35EC47E257E3FC0104
:10B3300061857285838594850E94B3D7181614F4AD
:10B340000E94CC6A80E00895609155327091563227
:10B35000809157329091583208950E94D25E80E0D9
:10B360000E944F6D80E008950E94D25E81E00E94AD
:10B370004F6D80E008950E94D25E82E00E944F6D82
:10B3800080E008950E94D25E83E00E944F6D80E0CD
:10B390000895CF93DF93EC01E0915932F0915A3246
:10B3A000E55BFF4FE081F0E0EE0FFF1FED5EFB4E2F
:10B3B000659174914FE450E084ED9CE30E94C3E1F9
:10B3C000AC0162EE7FE0CE01DF91CF910C94F9C128
:10B3D000CF93DF93EC01E0915932F0915A32E55B63
:10B3E000FF4FE081F0E0EE0FFF1FED5EFB4E659139
:10B3F00074914FE450E084ED9CE30E94C3E1AC0102
:10B400006AEC7FE0CE01DF91CF910C94F9C1CF932C
:10B41000DF93EC0181EF90E20E9428E3CE010E94CD
:10B42000C959CE010E94E85966EB7FE0CE010E9427
:10B43000C0C16DE97FE0CE010E948BC164E87FE06E
:10B44000CE010E948BC16BE67FE0CE010E948BC1D2
:10B4500062E57FE0CE010E948BC169E37FE0CE010F
:10B460000E948BC160E27FE0CE010E948BC167E049
:10B470007FE0CE010E948BC16EEE7EE0CE010E9485
:10B480008BC165ED7EE0CE010E948BC16CEB7EE04E
:10B49000CE010E948BC163EA7EE0CE010E948BC187
:10B4A0006AE87EE0CE010E948BC161E77EE0CE01BA
:10B4B0000E948BC168E57EE0CE010E94C0C180E0A1
:10B4C000DF91CF91089566EB7FE00C94C0C16DE9E8
:10B4D0007FE00C948BC164E87FE00C948BC16BE639
:10B4E0007FE00C948BC162E57FE00C948BC169E333
:10B4F0007FE00C948BC160E27FE00C948BC167E02D
:10B500007FE00C948BC16EEE7EE00C948BC165EDF8
:10B510007EE00C948BC16CEB7EE00C948BC163EAF3
:10B520007EE00C948BC16AE87EE00C948BC161E7ED
:10B530007EE00C948BC168E57EE00C94C0C16CED9C
:10B540007DE00C94C0C16BEA7DE00C94C0C166E75D
:10B550007DE00C94C0C16BE37DE00C94C0C167E05A
:10B560007DE00C94C0C1CF93DF93EC01E0915932A0
:10B57000F0915A32E55BFF4FE081F0E0EE0FFF1FE4
:10B58000ED5EFB4E659174914FE450E084ED9CE3D9
:10B590000E94C3E1AC0163EE7CE0CE01DF91CF916C
:10B5A0000C94F9C1CF93DF93EC01E0915932F09103
:10B5B0005A32E55BFF4FE081F0E0EE0FFF1FED5EDA
:10B5C000FB4E659174914FE450E084ED9CE30E9442
:10B5D000C3E1AC0162EC7CE0CE01DF91CF910C9431
:10B5E000F9C165EA7CE00C94A1C1CF93DF93EC0133
:10B5F000E0915932F0915A32E55BFF4FE081F0E083
:10B60000EE0FFF1FED5EFB4E659174914FE450E02D
:10B6100084ED9CE30E94C3E1AC0166E87CE0CE01CE
:10B62000DF91CF910C94F9C10F931F93CF93DF93C8
:10B630008C01FC0161857285838594850E9424D6E6
:10B64000E62FF0E0EE0FFF1FE052FC4E6591749183
:10B650004FE450E084ED9CE30E94C3E1E8012D96A5
:10B660009F938F93F80161857285838594850E94ED
:10B6700024D61F926F93DF93CF930F5E1F4F1F93BC
:10B680000F93DF93CF938AE69CE09F938F93ECED2B
:10B69000F9E581818F9380818F930E948AE2EDB7D3
:10B6A000FEB73E96EDBFFEBFDF91CF911F910F9188
:10B6B000089562E47CE00C9476486AE17CE00C94A6
:10B6C000764868EF7BE00C94764866ED7BE00C945E
:10B6D000764864EA7BE00C94764863E77BE00C9460
:10B6E00076486AE37BE00C9476486AE17BE00C9450
:10B6F000764868ED7AE00C94444866E97AE00C9468
:10B7000044486FE67AE00C94764869E47AE00C9459
:10B71000764868E27AE00C94764868E07AE00C9427
:10B7200076486BEE79E00C94C9486CEC79E00C94A7
:10B73000C948BC01675F7F4F2091A63242E45EE0BA
:10B74000FC01848195810C942049BC01675F7F4F87
:10B7500021E048E25EE0FC01848195810C9420495F
:10B76000BC01675F7F4F21E04FE05EE0FC01848118
:10B7700095810C9420490F931F93CF93DF93EC0195
:10B780000C811D810E94766408171907C4F48C810E
:10B790009D81FC01EE0FFF1FE80FF91FEE0FFF1F49
:10B7A000EE0FFF1FEE0FFF1FEC55FA4E259134915F
:10B7B000CE01F901DF91CF911F910F91199485E18D
:10B7C000DF91CF911F910F9108950F931F93CF9306
:10B7D000DF93EC010C811D810E9476640817190724
:10B7E000C4F48C819D81FC01EE0FFF1FE80FF91F4F
:10B7F000EE0FFF1FEE0FFF1FEE0FFF1FEE55FA4E6D
:10B8000025913491CE01F901DF91CF911F910F91D4
:10B81000199485E1DF91CF911F910F9108950F93B6
:10B820001F93CF93DF93EC010C811D810E947664FE
:10B8300008171907C4F48C819D81FC01EE0FFF1FCE
:10B84000E80FF91FEE0FFF1FEE0FFF1FEE0FFF1F98
:10B85000E056FA4E25913491CE01F901DF91CF9156
:10B860001F910F911994DF91CF911F910F9108951E
:10B87000CF93DF93EC018C819D810E9489648823A2
:10B88000C9F08C819D81FC01EE0FFF1FE80FF91FAD
:10B89000EE0FFF1FEE0FFF1FEE0FFF1FE256FA4ED7
:10B8A000E491E1FF05C0CE01DF91CF910C94B68009
:10B8B00080E001C085E1DF91CF9108950F931F9340
:10B8C000CF93DF93EC0181E00E94834E1C821D82A6
:10B8D00080E090E08E010F5E1F4F47C08C819D81FC
:10B8E0009C01220F331FF901E80FF91FEE0FFF1F14
:10B8F000EE0FFF1FEE0FFF1FE256FA4EE491E0FF3E
:10B900002EC0280F391F220F331F220F331F220F83
:10B91000331F28553A4EF90145915591659174911F
:10B9200049875A876B877C87BC01660F771F680F32
:10B93000791F660F771F660F771F660F771F685690
:10B940007A4E45E050E0C8010E94C3E1CE010E945A
:10B95000BB5BCE010E94385C2C813D8101C09C0103
:10B960002F5F3F4F2C833D83C9010E947964811171
:10B97000B5CF81E00E9425A8DF91CF911F910F9153
:10B980000C940DA8CF93DF93EC012CEA35EC47E241
:10B9900057E369857A858B859C850E94B0D587FFA2
:10B9A00005C0CE01DF91CF910C94B079CE010E94F9
:10B9B0005E5C82E08F8340E050E060E87FE349878F
:10B9C0005A876B877C8780E0DF91CF9108958091C3
:10B9D0009639909197398F3E924111F08AE50895FA
:10B9E0008091D8399091D9398F3E9241B9F78091A1
:10B9F0006C3490916D348F3E924181F780918E37F7
:10BA000090918F378F3E924149F780919037909176
:10BA100091378F3E924111F78091943990919539E9
:10BA20008F3E9241D9F68091233D8111D7CF089561
:10BA3000FC01178289E60895CF93DF93EC018C8196
:10BA40009D81FC01EE0FFF1FE80FF91FEE0FFF1F96
:10BA5000EE0FFF1FEE0FFF1FEA55FA4EA591B491AE
:10BA60006C9170E080E090E00E9450D669877A8700
:10BA70008B879C8782E08F8380E0DF91CF91089550
:10BA8000CF93DF93EC018C819D81FC01EE0FFF1FB2
:10BA9000E80FF91FEE0FFF1FEE0FFF1FEE0FFF1F46
:10BAA000EA55FA4EA591B4916D917D918D919C913D
:10BAB0000E9450D669877A878B879C8782E08F8324
:10BAC00080E0DF91CF910895CF93DF93DC0114964E
:10BAD0008D919C911597FC01EE0FFF1FE80FF91F48
:10BAE000EE0FFF1FEE0FFF1FEE0FFF1FEA55FA4E7E
:10BAF000C591D491488159816A817B8119964D9372
:10BB00005D936D937C931C9783E017968C9380E0F4
:10BB1000DF91CF910895CF93DF93DC0114968D913F
:10BB20009C911597FC01EE0FFF1FE80FF91FEE0F18
:10BB3000FF1FEE0FFF1FEE0FFF1FEA55FA4EC591D4
:10BB4000D491488159816A817B8119964D935D9387
:10BB50006D937C931C97FC01EE0FFF1FE80FF91FFC
:10BB6000EE0FFF1FEE0FFF1FEE0FFF1FE156FA4E05
:10BB70008591949118968C93189784E017968C93DE
:10BB800080E0DF91CF91089588E608950F931F9389
:10BB9000CF93DF93EC018C819D81FC01EE0FFF1FA1
:10BBA000E80FF91FEE0FFF1FEE0FFF1FEE0FFF1F35
:10BBB000EA55FA4E0591149169857A858B859C85A5
:10BBC0000E9424D6F801608382E08F8380E0DF91B9
:10BBD000CF911F910F910895CF93DF93EC01698569
:10BBE0007A858B859C850E9424D66230B0F48C8146
:10BBF0009D81FC01EE0FFF1FE80FF91FEE0FFF1FE5
:10BC0000EE0FFF1FEE0FFF1FEA55FA4EA591B491FC
:10BC10006C9382E08F8380E001C08EE6DF91CF914C
:10BC20000895CF93DF93EC0169857A858B859C8598
:10BC30000E9424D66330B0F48C819D81FC01EE0F0C
:10BC4000FF1FE80FF91FEE0FFF1FEE0FFF1FEE0F94
:10BC5000FF1FEA55FA4EA591B4916C9382E08F8351
:10BC600080E001C08EE6DF91CF910895CF93DF93FE
:10BC7000EC0169857A858B859C850E9424D6643089
:10BC8000B0F48C819D81FC01EE0FFF1FE80FF91FBE
:10BC9000EE0FFF1FEE0FFF1FEE0FFF1FEA55FA4ECC
:10BCA000A591B4916C9382E08F8380E001C08EE611
:10BCB000DF91CF9108950F931F93CF93DF93EC0102
:10BCC0008C819D81FC01EE0FFF1FE80FF91FEE0F25
:10BCD000FF1FEE0FFF1FEE0FFF1FEA55FA4E0591F3
:10BCE000149169857A858B859C850E9424D6F801FC
:10BCF0006083718382E08F8380E0DF91CF911F9119
:10BD00000F9108950F931F93CF93DF93EC018C81D4
:10BD10009D81FC01EE0FFF1FE80FF91FEE0FFF1FC3
:10BD2000EE0FFF1FEE0FFF1FEA55FA4E059114911B
:10BD300069857A858B859C850E9424D6F80160836D
:10BD400071838283938382E08F8380E0DF91CF9140
:10BD50001F910F910895CF93DF93DC0114968D917D
:10BD60009C911597FC01EE0FFF1FE80FF91FEE0FD6
:10BD7000FF1FEE0FFF1FEE0FFF1FEA55FA4EC59192
:10BD8000D49119964D915D916D917C911C9748834A
:10BD900059836A837B8383E017968C9380E0DF91DD
:10BDA000CF910895CF93DF93DC0114968D919C91F0
:10BDB0001597FC01EE0FFF1FE80FF91FEE0FFF1F95
:10BDC000EE0FFF1FEE0FFF1FEA55FA4EC591D491FB
:10BDD00019964D915D916D917C911C974883598383
:10BDE0006A837B83FC01EE0FFF1FE80FF91FEE0F44
:10BDF000FF1FEE0FFF1FEE0FFF1FE156FA4E85915A
:10BE0000949118968C93189784E017968C9380E001
:10BE1000DF91CF9108951F93CF93DF93EC01809131
:10BE2000F8398823D1F01DE10A80DB81C02D2097ED
:10BE300011F480E013C08F818F3FD9F3811104C0CA
:10BE4000CE010E94E55B06C0CE010E94BB5BCE0125
:10BE50000E94385C115041F7ECCF85E6DF91CF911D
:10BE60001F910895CF93DF93EC01BC018FEF90E217
:10BE70000E94FCE1892B41F0BE0182E091E20E9428
:10BE8000FCE121E0892B09F420E0822FDF91CF91A2
:10BE900008950F931F93CF93DF93CDB7DEB7299704
:10BEA000CDBFDEBF8B0144E050E0BC01CE01019666
:10BEB0000E941CE246E050E0B801CE0101960E94CB
:10BEC0000CE20E947664181619060CF03FC07981C6
:10BED000AA81BB811C810D8128E935E140E050E059
:10BEE000F9016491671327C03196E491E11103C011
:10BEF000A11121C029C0EA131EC0F9013296E491B4
:10BF0000E11103C0B11117C01FC0EB1314C0F90138
:10BF10003396E491E11103C011110DC015C0E11376
:10BF20000AC0F9013496E491E11103C0011103C084
:10BF30000BC0E01749F04F5F5F4F285E3F4F481737
:10BF4000590709F0CDCF02C0CA0102C08FEF9FEFA1
:10BF50002996CDBFDEBFDF91CF911F910F9108953C
:10BF6000CF93DF93FC012189222371F1EC016196CB
:10BF7000BE0186E091E20E94FCE1892B39F1BE010D
:10BF80008FEF90E20E94FCE1892B11F1BE0189E064
:10BF900091E20E94FCE1892BD9F0BE018DEE90E286
:10BFA0000E94FCE1892BB1F0BE018CE091E20E947D
:10BFB000FCE1892B79F0BE0180EE91E20E94FCE168
:10BFC000892B51F485E009C080E007C082E005C0FC
:10BFD00083E003C084E001C081E0DF91CF91089548
:10BFE000FC018FEF878314821582118612861386D7
:10BFF00014861086118A1586178A108EA081B18149
:10C00000109711F416820DC017968C9117978730F0
:10C0100029F416968C918F5F868303C016968C91B7
:10C020008683CF010895EF92FF920F931F93CF93D2
:10C03000DF93EC010C811D810E94766408171907BB
:10C040000CF06FC00C811D81CE010E94F05F0C834B
:10C050001D837E0181E1E80EF11CB801660F771F98
:10C06000600F711F660F771F660F771F660F771FB0
:10C0700068567A4EC7010E94A4E18E01035F1F4FEC
:10C080002C813D81B901660F771F620F731F660F08
:10C09000771F660F771F660F771F6C567A4EC801A1
:10C0A0000E94A4E18D85882311F18C819D81FC0182
:10C0B000EE0FFF1FE80FF91FEE0FFF1FEE0FFF1F20
:10C0C000EE0FFF1FE256FA4EE491E2FF02C01D861A
:10C0D00010C0F80101900020E9F7BF01601B710B4F
:10C0E000605F7F4F6C0F7D1FC7010E9405E28C814E
:10C0F0009D81FC01EE0FFF1FE80FF91FEE0FFF1FE0
:10C10000EE0FFF1FEE0FFF1FEE55FA4E25913491F3
:10C11000CE01F901DF91CF911F910F91FF90EF9028
:10C120001994DF91CF911F910F91FF90EF90089597
:10C130008F929F92AF92BF92CF92DF92EF92FF9237
:10C140000F931F93CF93DF9300D01F92CDB7DEB72D
:10C150006C015C0181E1A80EB11C87E0F6018783C8
:10C16000A4E9EA2EA5E1FA2E00E010E01DC0B70117
:10C17000CE0101960E94A4E1BE016F5F7F4FC50111
:10C180000E94FCE1892B59F44601F9E18F0E911CC4
:10C19000F601058F168FC4010E94136064010F5FC2
:10C1A0001F4FF8E1EF0EF11CC8010E947964811164
:10C1B000DECF2496CDBFDEBFDF91CF911F910F91CF
:10C1C000FF90EF90DF90CF90BF90AF909F908F90B7
:10C1D0000895CF93DF931092923710929337A5E58D
:10C1E000B4E3EEE6F4E391E08FEFA083B1837996B8
:10C1F0005B96ED93FC935C975D961D921C925E9707
:10C20000EF016397988322961882219788832A9654
:10C210001882599627E3EE38F20739F710927737EC
:10C220001092783710926E3410926F3410927434EA
:10C2300087E08093753482E790E080937F34909319
:10C24000803487E894E3DF91CF9108950F931F9393
:10C25000CF93DF930E94E960EC018FEE92E180932F
:10C260009639909397398093D8399093D9398093A0
:10C270006C3490936D3480938E3790938F37809386
:10C28000903790939137809394399093953981E0CA
:10C290000E94834E1C821D82CE010E948D802091BF
:10C2A000E0393091E1394091E2395091E3396985C3
:10C2B0007A858B859C850E94B0D5882339F0CE0184
:10C2C000DF91CF911F910F910C945E5C0E9412A898
:10C2D0001C821D8280E090E08E010F5E1F4F2FC0F8
:10C2E0006C817D819B01220F331FF901E60FF71F3F
:10C2F000EE0FFF1FEE0FFF1FEE0FFF1FE256FA4E6D
:10C30000E491E0FF17C0620F731F660F771F660F7F
:10C31000771F660F771F68567A4E45E050E0C801D8
:10C320000E94C3E1CE010E948D80CE010E94BB5BC2
:10C330006C817D816F5F7F4F6C837D83CB010E9419
:10C3400079648111CDCFDF91CF911F910F910C9422
:10C3500025A8EF92FF920F931F93CF93DF938C0149
:10C360002091923730919337EB0109900020E9F743
:10C370002197C61BD70BAE01420F531F41305240CD
:10C38000D8F4F901EC56F84C7F01AE014F5F5F4FD6
:10C39000CF010E94DDE140919237509193374F5F7A
:10C3A0005F4F4C0F5D1F4093923750939337F801C6
:10C3B000E78AF08E80E001C08DE0DF91CF911F9180
:10C3C0000F91FF90EF900895CF93DF932EE1C7E890
:10C3D000D4E33F813F3F59F00A80DB81C02D209795
:10C3E00019F480E090E010C0215099F7FACFBC0119
:10C3F00084E493E20E94495F8C839D83019689F3D4
:10C40000CE010E941360CE01DF91CF910895EF928B
:10C41000FF920F931F93CF93DF938B012EE1C7E819
:10C42000D4E33F813F3F59F00A80DB81C02D209744
:10C4300019F480E090E01DC0215099F7FACF7E01F9
:10C4400021E1E20EF11C45E050E0BC01C7010E9471
:10C450001CE2B801CE010E94A9618111EACFB701A7
:10C4600084E493E20E94495F8C839D8385E08F83FF
:10C47000CE01DF91CF911F910F91FF90EF90089522
:10C480002091F839213021F42091D03C213029F439
:10C49000BC018DEE90E20C94076280E090E008957C
:10C4A0009091F839913019F4642F0C94097F0C9411
:10C4B0000BC1CF93DF93EC018091E52F811103C075
:10C4C0000E9446D202C00E9454C9682F70E080E0EA
:10C4D00090E00E9450D669877A878B879C8782E09C
:10C4E0008F8380E0DF91CF9108950F931F93CF93B7
:10C4F000DF93CDB7DEB7C058D109CDBFDEBFFC0199
:10C5000061857285838594850E9424D68FEF860F7E
:10C51000863030F080E491E20E9440628EE62AC0CC
:10C520006093E02F81E08093E12FE62FF0E0EE0FA3
:10C53000FF1FE15AFA4E659174914FE450E084ED8B
:10C540009CE30E94C3E19F938F9386E294E19F93C3
:10C550008F938E010F5F1F4F1F930F930E947EE3F7
:10C56000C8010E9440620F900F900F900F900F90A3
:10C570000F9080E0C058DF4FCDBFDEBFDF91CF917D
:10C580001F910F9108950F931F93CF93DF93EC01A9
:10C590008BE592E30E944E4A882329F009851A858B
:10C5A0008B859C8511C023E333E34BEC51E4698513
:10C5B0007A858B859C850E9455D88B01AB01BC0187
:10C5C00049875A876B877C872C813D81F901EE0F63
:10C5D000FF1FE20FF31FEE0FFF1FEE0FFF1FEE0F07
:10C5E000FF1FEA55FA4EA591B491A801BC014D93E5
:10C5F0005D936D937C931397F901EE0FFF1FE20F8C
:10C60000F31FEE0FFF1FEE0FFF1FEE0FFF1FE15690
:10C61000FA4E85919491888784E08F8380E0DF9142
:10C62000CF911F910F91089560E375E10C94A1C122
:10C630006CE075E10C94A1C160ED74E10C94A1C1B2
:10C640006CE974E10C94A1C16FE474E10C94A1C194
:10C650001F93CF93DF93EC0110E08881882301F1D1
:10C660000E94E96045E050E0BE0188E994E30E9441
:10C670001CE268E974E384E493E20E94495F8093DA
:10C680008B3490938C3487E894E30E94136042E0EB
:10C6900063E080E00E9450621F5F26961D31E9F63C
:10C6A00084E0DF91CF911F910895CF93DF93CDB7B1
:10C6B000DEB7EC97CDBFDEBF8CE3E8E1F0E2DE0150
:10C6C000119601900D928A95E1F7CE0101960E9494
:10C6D0002863EC96CDBFDEBFDF91CF910895CF9355
:10C6E000DF93CDB7DEB7AA97CDBFDEBF8AE2E4E520
:10C6F000F0E2DE01119601900D928A95E1F7CE01EC
:10C7000001960E942863AA96CDBFDEBFDF91CF912C
:10C710000895CF93DF93CDB7DEB76E97CDBFDEBF61
:10C720008EE1EEE7F0E2DE01119601900D928A951E
:10C73000E1F7CE0101960E9428636E96CDBFDEBF61
:10C74000DF91CF910895CF93DF93EC0143E759E751
:10C7500063E770E0498B5A8B6B8B7C8B0E949860EF
:10C7600042E063E080E00E945062CE010E94896353
:10C77000CE010E946F6320E731E340E0298B3A8BC2
:10C780004B8BCE010E94986042E063E080E00E9403
:10C790005062CE01DF91CF910C945563CF92DF921E
:10C7A000EF92FF92FC01C184D284E384F48420E000
:10C7B00030E040E85FE3C701B6010E94B3D7181626
:10C7C000FCF0C701B6010E9424D66093E22FC70196
:10C7D000B6019F772CEA35EC47E257E30E94B3D7C6
:10C7E00018163CF460E470E080E00E9432C780E0FC
:10C7F00008C060E870E080E00E9432C780E001C0BD
:10C800008EE6FF90EF90DF90CF900895CF92DF9269
:10C81000EF92FF92FC01C184D284E384F48420E08F
:10C8200030E040E050E4C701B6010E94B3D71816CB
:10C83000FCF0C701B6010E9424D66093E42FC70123
:10C84000B6019F772CEA35EC47E257E30E94B3D755
:10C8500018163CF464E070E080E00E9432C780E08B
:10C8600008C068E070E080E00E9432C780E001C04C
:10C870008EE6FF90EF90DF90CF900895CF92DF92F9
:10C88000EF92FF92FC01C184D284E384F48420E01F
:10C8900030E040E85FE3C701B6010E94B3D7181645
:10C8A000FCF0C701B6010E9424D66093E32FC701B4
:10C8B000B6019F772CEA35EC47E257E30E94B3D7E5
:10C8C00018163CF460E170E080E00E9432C780E01E
:10C8D00008C060E270E080E00E9432C780E001C0E2
:10C8E0008EE6FF90EF90DF90CF9008958CE891E076
:10C8F000089521E08334914008F020E0822F0895CC
:10C900009C012F55314081E02932310508F080E04B
:10C91000089521E08036914008F020E0822F0895AC
:10C92000CF92DF92EF92FF92CF93DF93EC01C98415
:10C93000DA84EB84FC84A7019601C701B6010E944A
:10C9400076D981113CC0E894F7F82FEF3FEF4FE71D
:10C950005FE7C701B6010E9476D981110AC02FEFA7
:10C960003FEF4FE75FE7C701B6010E94B0D5181649
:10C9700034F18C819D81FC01EE0FFF1FE80FF91F40
:10C98000EE0FFF1FEE0FFF1FEE0FFF1FE256FA4ED6
:10C99000E491E3FF14C08BE592E30E944E4A8111BB
:10C9A0000EC025E832E441E25DE369857A858B8536
:10C9B0009C850E9455D869877A878B879C87DF91F1
:10C9C000CF91FF90EF90DF90CF9008958091E12F6D
:10C9D000882349F01092E12F6091E02F80E00E94BF
:10C9E0003AC780E0089583E00895CF93DF93E09104
:10C9F000163AF091173A04C0E093163AF093173ABA
:10CA0000EF018191982F9D7F9032B1F38930A1F38E
:10CA10004FE750E0BE018AE19CE30E941CE268817E
:10CA2000611105C08091F83981116DC039C0613242
:10CA300021F4DF91CF910C942A55653221F4DF91D6
:10CA4000CF910C942E556E3721F4DF91CF910C9439
:10CA500032556F3379F4FE0101900020E9F73197E8
:10CA6000EC1BFD0B329780F02196C093163AD093C1
:10CA7000173A49C06B3741F481E08093F839CE0111
:10CA8000DF91CF910C94067A70E080E791E20E94EA
:10CA9000F1E1892B59F01092F839CE010E9463BD63
:10CAA0006AE17CE3DF91CF910C94A3BE8091F839C9
:10CAB000811109C0CE010E9419706AE17CE3DF9107
:10CAC000CF910C94A3BE0E94E960EC0127E633E607
:10CAD00040E0298B3A8B4B8B6091163A7091173A54
:10CAE0000E94A96185E08F838091163A9091173A50
:10CAF0000E94197042E060E00E94506280E0DF9185
:10CB0000CF910C9476AADF91CF910895FF920F9365
:10CB10001F93CF93DF931F921F92CDB7DEB7F82EEE
:10CB2000EAEDF9E322EC32E0DF01C9011D92019741
:10CB3000E9F72FEE32E12083318320939A3C309342
:10CB40009B3C07ED13E22CED33E40093E0391093A6
:10CB5000E1392093E2393093E3390CEE11E528E70F
:10CB60003FE30093E4391093E5392093E63930939D
:10CB7000E73900E010E020EA30E40093E839109350
:10CB8000E9392093EA393093EB3900E010E020E8EE
:10CB90003FE30093EC391093ED392093EE39309355
:10CBA000EF3983E08093F9398F2D4A8369830E949E
:10CBB0004AC76981862F0E9455C74A81842F0E94E7
:10CBC00060C7F092DF2FF092DD2F0F900F90DF9172
:10CBD000CF911F910F91FF900895CF93DF931F92F4
:10CBE0001F92CDB7DEB780E6F82E01E010E00E947C
:10CBF0006E788230E1F30E9475788230C1F30E9432
:10CC00002D4A863009F0D9C00E942DC58090FF3989
:10CC10009090003AA090013AB090023A861697069A
:10CC2000A806B90620F70E942DC56C597F4F8F4F7B
:10CC30009F4F6093FF397093003A8093013A90932D
:10CC4000023A0E94E477D3CF0E943EBC882329F0A9
:10CC50008CEC0E946F4E823051F20E9483558230DC
:10CC600031F20E94689D823011F20E94E75C80934D
:10CC7000243D81112EC08091DA399091DB398F3EAD
:10CC8000924109F0AAC080919A3C90919B3C8F3EC2
:10CC9000924109F0A2C097C00E9462818093243D16
:10CCA000811117C00E94CBB28093243D811111C025
:10CCB0000E94E46F8093243D81110BC00E9459C6ED
:10CCC0008093243D811105C00E949FB3823031F4CE
:10CCD0008ECF0E946F4E8230B9F789CF0E94A8AAEA
:10CCE000823009F484CF0E9414AC823009F47FCFE3
:10CCF0000E94D0AC823009F47ACF09831A8368E1AC
:10CD00007AE3CE0101960E946FC78093163A909302
:10CD1000173A8F3F2FEF920739F48DE00E94584E5B
:10CD2000823009F464CF04C0892B11F00E94F564AD
:10CD30000E94C78B823009F45ACF0E941B6B82304D
:10CD400009F455CF0E94DA6D823009F450CF0E9469
:10CD5000BF6F823009F449CF0E94FC4B823009F446
:10CD600044CF0E9417828430F0F53FCF8091F9398B
:10CD7000843038F484E08093F9390E942E550E9463
:10CD800017A883E090E089839A8368E17AE3CE0173
:10CD900001960E946FC78093163A9093173A8F3F7F
:10CDA0002FEF920721F48DE00E94584E1ECF892B61
:10CDB00009F41BCF0E94F56418CF0E942D4A8230DF
:10CDC00009F44BCF41CF1092243D0E942A4E80930C
:10CDD000243D882309F460CF7CCFF092243D80E687
:10CDE0000E946F4E78CF8091222A9091232A0E9430
:10CDF000BAD0682F70E080E090E00E9452D620E028
:10CE000030E048E451E40E94B3D787FFEECE0E94A1
:10CE1000E664823009F0AACFE8CE8091DF2F8093BC
:10CE2000DD2F08958093DD2F08958093DE2F0895E0
:10CE3000CF93C82F80918F23882379F040E050E072
:10CE4000BA018C2F0E94D44FEC2FFF27E7FDF095FD
:10CE5000E05DFD4C81E080830AC06C2F83E296E5A3
:10CE60000E94734BAB01BC018C2F0E94D44F4091A8
:10CE7000B6235091B7236091B8237091B9238C2FBA
:10CE80000E94D75881EE98E6809390239093912347
:10CE900082E0CF910895CF92DF92EF92FF920F93AD
:10CEA0001F93CF93DF93CDB7DEB7E097CDBFDEBF43
:10CEB00098E17E01A9E1EA0EF11CF701A92F119278
:10CEC000AA95E9F7FE0131966F0111929A95E9F75B
:10CED000F60194E08902E00DF11D1124408F518F7D
:10CEE000628F738F80E090E0A0E8BFE3808391833E
:10CEF000A283B383009398321093993220939A328D
:10CF000030939B320E949A820E943255B601C7012B
:10CF10000E94FC528093243D811101C082E0E09682
:10CF2000CDBFDEBFDF91CF911F910F91FF90EF90AA
:10CF3000DF90CF9008950F931F93E0918923FF27EF
:10CF4000E7FDF095EB5FFF4C9381913099F40091F0
:10CF50009A2310919B2320919C2330919D234091F3
:10CF6000A2235091A3236091A4237091A5230E9432
:10CF70004B671DC0E0918A23FF27E7FDF095EB5F2B
:10CF8000FF4C9381913099F400919A2310919B2347
:10CF900020919C2330919D234091A2235091A32363
:10CFA0006091A4237091A52370580E944B6781EE75
:10CFB00097E6809390239093912382E01F910F91A5
:10CFC00008950F931F93CF93C82F85E3C802F001F4
:10CFD0001124EF5FFE4C40815181628173818C2F5F
:10CFE0000E94D75800919A2310919B2320919C2353
:10CFF00030919D23409196235091972360919823DF
:10D00000709199238C2F0E944B6780E798E680935C
:10D0100090239093912382E0CF911F910F910895D7
:10D020000F931F9300919A2310919B2320919C238F
:10D0300030919D234091A6235091A7236091A8236E
:10D040007091A9230E944B6788E197E68093902313
:10D050009093912382E01F910F9108950E949A82EC
:10D060008091AF230E943D4F8091AE230E94834E5A
:10D070008091B0230E94874E8091B1230E94E85294
:10D080008091B2239091B323A091B423B091B523A2
:10D090008093983290939932A0939A32B0939B32B6
:10D0A00064E08BE592E30E946B4A0E94DF55109288
:10D0B0002C3280E00895CF93C82F4091B623509131
:10D0C000B7236091B8237091B9230E94D7588C2F51
:10D0D0000E942E6880E00E9476AA80EFCF9108958A
:10D0E0000F931F93E0918923FF27E7FDF095EB5FF6
:10D0F000FF4C9381913039F08BE598E68093902333
:10D100009093912318C000919E2310919F2320910A
:10D11000A0233091A1234091A2235091A323609199
:10D12000A4237091A5230E944B6780E198E6809329
:10D1300090239093912382E01F910F910895FF9285
:10D140000F931F93CF93DF93CDB7DEB7C058D109AC
:10D15000CDBFDEBFF82E0E94E9608EEFF81205C049
:10D1600085E791E20E94406219C08F2D0E9474569B
:10D170001F928F9324EB3AE33F932F938E010F5F1F
:10D180001F4F1F930F930E947EE3C8010E944062CD
:10D190000F900F900F900F900F900F9042E062E071
:10D1A00080EF0E9450628F2D0E942E6880EFC05841
:10D1B000DF4FCDBFDEBFDF91CF911F910F91FF9069
:10D1C00008954F925F926F927F929F92AF92BF921B
:10D1D000CF92DF92EF92FF920F931F93CF93DF9343
:10D1E0008F3F09F045C02CEA35EC47E257E36091E8
:10D1F00093337091943380919533909196330E943C
:10D20000B3D718160CF469C12CEA35EC47E257E3A2
:10D2100060918B3370918C3380918D3390918E33EC
:10D220000E94B3D718160CF45DC12CEA35EC47E226
:10D2300057E360918F337091903380919133909147
:10D2400092330E94B3D718160CF455C12CEA35EC72
:10D2500047E257E360919733709198338091993307
:10D2600090919A330E94B3D718160CF43FC171C144
:10D270008230A1F52CEA35EC47E257E360918B331D
:10D2800070918C3380918D3390918E330E94B3D7FF
:10D2900018160CF427C12CEA35EC47E257E36091ED
:10D2A0008F337091903380919133909192330E949B
:10D2B000B3D718160CF41FC12CEA35EC47E257E33C
:10D2C00060919733709198338091993390919A330C
:10D2D0000E94B3D718160CF409C131C18823D9F2C2
:10D2E000813051F32CC17E018DEEE80EF11CF70167
:10D2F00080819181A281B381BC01CD019F772CEA0D
:10D3000035EC47E257E30E94B0D587FD46C06E0179
:10D31000F1EFCF0ED11CF601408051806280738006
:10D3200020E030E0A901C301B2010E94B0D587FD21
:10D3300034C0FE01EF52FF4F208131814281538181
:10D34000349760817181828193810E9407D49B010F
:10D35000AC015F77C301B2010E9408D42B013C01EC
:10D360009F772CEA35EC47E257E30E94B0D587FD62
:10D3700014C0AB2CAA0C8A2D0E9438BC8093872342
:10D38000992493949A0C892D0E9438BC8093882309
:10D3900020918723822780FD02C08B2DDBC0B092B5
:10D3A0008623F80180819181A281B381BF77809328
:10D3B0009A2390939B23A0939C23B0939D23F701E2
:10D3C00040815181628173817F7740939E23509386
:10D3D0009F236093A0237093A12320FF2DC0A092D0
:10D3E000892390928A2377FA709477F87094409208
:10D3F0009623509297236092982370929923F60176
:10D4000080819181A281B3818093A2239093A323F1
:10D41000A093A423B093A523CB50DF4F888199819B
:10D42000AA81BB818093A6239093A723A093A823CE
:10D43000B093A9238A2D2AC090928923A0928A238F
:10D44000409296235092972360929823709299234A
:10D45000F60180819181A281B381B0588093A2238B
:10D460009093A323A093A423B093A523CB50DF4F85
:10D4700088819981AA81BB81B0588093A62390931B
:10D48000A723A093A823B093A923892D0E9438BC79
:10D490008D7F813039F081EE98E6809390239093D0
:10D4A000912369C080918A230E9438BC811103C0F6
:10D4B0008FEF80938A238B2D0E94CC586093B623E4
:10D4C0007093B7238093B8239093B9238BE997E6A1
:10D4D00080939023909391234EC082E090E032E0BD
:10D4E000B32E0DC080E090E0B12C09C083E090E045
:10D4F00023E0B22E04C081E090E0BB24B394FC0191
:10D50000E05DFD4C108225E3289FE001299FD00DAE
:10D510001124C85DDF4C8E0107511F4FF801808137
:10D520009181A281B381BC01CD019F772CEA35ECBA
:10D5300047E257E30E94B0D587FFD5CE2ECF81E0DA
:10D5400080932F328EE298E68093902390939123DC
:10D5500012C08EEFDF91CF911F910F91FF90EF904E
:10D56000DF90CF90BF90AF909F907F906F905F9033
:10D570004F900C949F6882E0DF91CF911F910F91A3
:10D58000FF90EF90DF90CF90BF90AF909F907F90F3
:10D590006F905F904F900895CF93DF93C9E5D2E3EA
:10D5A000888199810E944E4A8093AE238881998117
:10D5B0000E94494A8093AF23888199810E94584AEA
:10D5C0008093B023888199810E945D4A8093B12322
:10D5D000888199810E94644A6093B2237093B32337
:10D5E0008093B4239093B52381E00E94834E81E021
:10D5F0000E94874E80E00E943D4F81E00E94E852E9
:10D6000081E080938F238FEF8093862381EE98E6CD
:10D61000809390239093912383E080932C321092F7
:10D620002F3280E0DF91CF9108950E94CC6A109252
:10D630008F2380E0089580912C32833059F40E942A
:10D64000624A813049F0E0919023F09191238091DA
:10D650008623199483E0089582E0089586E39BE68B
:10D660008093CB239093CC2382E008952F923F9216
:10D670004F925F926F927F928F929F92AF92BF92E2
:10D68000CF92DF92EF92FF920F931F93CF93DF938E
:10D69000CDB7DEB7CA54D109CDBFDEBF98E19E0138
:10D6A000275E3F4F29AB3AABD901E92F1D92EA958E
:10D6B000E9F7285131091901D9011D929A95E9F725
:10D6C00024E08202F00111242B96EEAFFFAF2B97DE
:10D6D000E20DF31D80E090E0A0E8BFE3808391833A
:10D6E000A283B383C090C323D090C423E090C5230A
:10D6F000F090C6234090BF235090C0236090C12378
:10D700007090C2238090BB239090BC23A090BD2337
:10D71000B090BE23A5019401C301B2010E94B0D50F
:10D7200018165CF080E090E0A0E8BFE329968CAF8B
:10D730009DAFAEAFBFAF29970AC080E090E0A0E8F0
:10D74000BFEB29968CAF9DAFAEAFBFAF2997A301BA
:10D750009201C501B4010E9407D40E941FD69B010B
:10D7600077FF04C022273327261B370BB9018827F0
:10D7700077FD8095982F0E9452D625966CAF7DAF8D
:10D780008EAF9FAF2597C0929832D0929932E09297
:10D790009A32F0929B320E949A820E94325520E087
:10D7A00030E040E050E425966CAD7DAD8EAD9FAD90
:10D7B00025970E94B3D718166CF08091C7239091DB
:10D7C000C823A091C923B091CA238BAF9CAFADAF42
:10D7D000BEAFDBC02AE037ED43E25CE325966CADDB
:10D7E0007DAD8EAD9FAD25970E94B3D718162CF74F
:10D7F00009E110E08AE0882E87ED982E83E2A82EBA
:10D800008CE3B82E412C512C32012B96AEADBFAD1E
:10D810002B97A20DB31D58962196AEAFBFAF21979F
:10D820004BAA5CAA6DAA7EAA8FAA98AEA9AEBAAE80
:10D8300029962CAD3DAD4EAD5FAD29976FA978AD62
:10D8400089AD9AAD0E9455D89B01AC016091BF2370
:10D850007091C0238091C1239091C2230E9408D46B
:10D860002196EEADFFAD2197608371838283938310
:10D87000C0929832D0929932E0929A32F0929B32D2
:10D88000B101CE0149960E94FC528093243D811142
:10D89000AAC020E030E040E85FE36BA97CA98DA935
:10D8A0009EA90E9408D46BAB7CAB8DAB9EAB20E0F5
:10D8B00030E048EC51E40E94B7D59B01AC0160E038
:10D8C00070E080E291E40E94B8D82B013C01809185
:10D8D000C7239091C823A091C923B091CA238BAFCD
:10D8E0009CAFADAFBEAFC090C323D090C423E09037
:10D8F000C523F090C623A7019601BC01CD010E946B
:10D9000007D44B015C0120E030E040E251E4C30168
:10D91000B2010E94B7D59B01AC01C501B4010E94C0
:10D9200055D89B01AC01C701B6010E9408D46B0118
:10D930007C012BA93CA94DA95EA9CA01B9010E948D
:10D9400008D420E030E048EC51E40E94B7D59B01B8
:10D95000AC016FA978AD89AD9AAD0E9408D46FABC8
:10D9600078AF89AF9AAF9B01AC0125966CAD7DADC8
:10D970008EAD9FAD25970E94B3D7181634F4015091
:10D9800011090115110509F053CF8BAD9CADADAD5B
:10D99000BEAD8093983290939932A0939A32B0930F
:10D9A0009B322B96EEADFFAD2B97E20DF31D8091D0
:10D9B000BB239091BC23A091BD23B091BE23808F47
:10D9C000918FA28FB38FB101CE0149960E94FC5274
:10D9D0008093243D811107C08AE09DE68093CB238C
:10D9E0009093CC2382E0C65BDF4FCDBFDEBFDF91DB
:10D9F000CF911F910F91FF90EF90DF90CF90BF904C
:10DA0000AF909F908F907F906F905F904F903F90DE
:10DA10002F900895CF93DF931F92CDB7DEB7898300
:10DA20000E949A824091D5235091D6236091D723AA
:10DA30007091D82389810E94D7588091D2230E9467
:10DA40003D4F8091D1230E94834E8091D3230E9429
:10DA5000874E8091D4230E94E8528091CD239091EB
:10DA6000CE23A091CF23B091D0238093983290936E
:10DA70009932A0939A32B0939B3264E08BE592E3A3
:10DA80000E946B4A0E94DF5510922C3281EA91E28B
:10DA90000E9428E380E00F90DF91CF9108950F93CB
:10DAA0001F93CF93C82F09E512E3F801808191817C
:10DAB0000E944E4A8093D123F801808191810E9477
:10DAC000494A8093D223F801808191810E94584A6B
:10DAD0008093D323F801808191810E945D4A8093D5
:10DAE000D423F801808191810E94644A6093CD2300
:10DAF0007093CE238093CF239093D0238C2F0E94BA
:10DB0000CC586093D5237093D6238093D7239093DA
:10DB1000D82381E00E94834E80E00E94874E80E0FF
:10DB20000E943D4F81E00E94E85240E050E060E2F8
:10DB300071E44093C3235093C4236093C52370932F
:10DB4000C62385E3C89FF0011124EF50FF4C4081AC
:10DB50005181628173814093C7235093C82360939E
:10DB6000C9237093CA236C2F83E296E50E94604B11
:10DB70006093BF237093C0238093C1239093C223EB
:10DB80000E94A4596093BB237093BC238093BD2350
:10DB90009093BE23C093BA238EE29BE68093CB235F
:10DBA0009093CC2384E080932C3280E0CF911F911E
:10DBB0000F91089580912C32843059F40E94624A6A
:10DBC000813049F0E091CB23F091CC238091BA23AE
:10DBD000199483E0089582E00895E091DB23F0E05A
:10DBE000EB5FFF4C8381882341F088E09EE68093C1
:10DBF000D9239093DA2382E0089568E274E280E109
:10DC000094E20E94FC528093243D882371F308958E
:10DC10001F93CF93DF93E091DB23F0E0EB5FFF4CAA
:10DC200081E09381913009F080E080933632C7E340
:10DC3000D2E310E0812F0E948896AB01BC01812FB6
:10DC40000E94D44F612F8091593290915A320E9494
:10DC5000604B69937993899399931F5F163051F7BD
:10DC60008BEA91E20E94067A84E79EE68093D923AC
:10DC70009093DA2382E0DF91CF911F9108951F9353
:10DC8000CF93DF930E949A828091DC2380930530AA
:10DC9000E091DB23F0E08091DD23EB5FFF4C838795
:10DCA0000E9455BCC0EED3E210E0499159916991B0
:10DCB0007991812F0E94D7581F5F1630B1F780915C
:10DCC000DF230E943D4F8091DE230E94874E64E057
:10DCD0008BE592E30E946B4A0E94DF5510922C3232
:10DCE000DF91CF911F9108950E943F6E80E00895CB
:10DCF0000F931F93CF93DF93CDB7DEB7C058D109F1
:10DD0000CDBFDEBF182F0E94E9601E3F29F488EBCB
:10DD100091E20E94406219C0812F0E9474561F92A6
:10DD20008F9382EE9AE39F938F938E010F5F1F4F25
:10DD30001F930F930E947EE3C8010E9440620F90E0
:10DD40000F900F900F900F900F9042E062E08AEFDB
:10DD50000E9450620E943F6E8AEFC058DF4FCDBFD5
:10DD6000DEBFDF91CF911F910F910895FF920F9326
:10DD70001F93CF93DF931092363282E080932C3240
:10DD800000EE13E2C1E0D1E3F12C8F2D0E94CC58BC
:10DD9000F80161937193819391938F014881598127
:10DDA0006A817B818F2D0E94D7586F2D80915932C7
:10DDB00090915A320E94604BF801648B758B868B70
:10DDC000978BF394E596F6E0FF12DFCF60E174E203
:10DDD00088EF93E20E9430C22AE43CE042E85EE32E
:10DDE0000E94B0D587FF03C08EEF0E94786EC4E01A
:10DDF000D4E213E069917991899199912C893D89B7
:10DE00004E895F890E9407D49F772CEA35EC47E260
:10DE100057E30E94B3D718161CF4812F0E94786E26
:10DE20001F5F163039F784E08093DB238091143034
:10DE30008093DD2381E080931430809105308093BE
:10DE4000DC23109205300E9455BC8091593290918C
:10DE50005A320E94494A8093DF238091593290912F
:10DE60005A320E94584A8093DE2380E00E94874EF7
:10DE700080E00E943D4F80E00E94B1AE8DEE9DE6B5
:10DE80008093D9239093DA2382E0DF91CF911F9181
:10DE90000F91FF9008950F931F93CF93DF938C0101
:10DEA000EB018091A432882399F08091983290916F
:10DEB0009932A0919A32B0919B32BC01CD019F77EB
:10DEC0002CEA35EC47E257E30E94B0D587FD4FC0FE
:10DED00088819981AA81BB81BC01CD019F772CEA01
:10DEE00035EC47E257E30E94B3D71816F4F48C815F
:10DEF0009D81AE81BF81BC01CD019F772CEA35ECBD
:10DF000047E257E30E94B3D718167CF488859985B9
:10DF1000AA85BB85BC01CD019F772CEA35EC47E291
:10DF200057E30E94B3D7181624F188E1F801A0E165
:10DF3000B4E201900D928A95E1F788E1FE01A8E232
:10DF4000B4E201900D928A95E1F788E1E7E3F2E30C
:10DF5000DF011D928A95E9F782E08093363286EBE5
:10DF60009EE68093D9239093DA2380E003C08EE865
:10DF700001C086E8DF91CF911F910F9108958091A4
:10DF80002C32823021F080913632823049F40E9466
:10DF9000624A813039F0E091D923F091DA23199463
:10DFA00083E0089582E00895ECE9FCE380E2DF017C
:10DFB0001D928A95E9F78FEE92E18093BA3C909397
:10DFC000BB3C8083918308958091BA3C9091BB3C87
:10DFD0008F3E924111F08CE5089580919C3C909188
:10DFE0009D3C8F3E9241B9F780E00895CF93DF9337
:10DFF000C82FCB01BA010E9404D927E0C29FE001DB
:10E000001124C456D34C0E941FD66D837E838F8308
:10E010009887DF91CF91089597E0899FF0011124AF
:10E02000E456F34C65817681878190850E9452D6B3
:10E0300008952F923F924F925F926F927F928F92AC
:10E040009F92AF92BF92CF92DF92EF92FF920F9387
:10E050001F93CF93DF93CDB7DEB72797CDBFDEBF3A
:10E060008C011B8280912B32823009F40EC7D801BB
:10E07000BC90B11037C780E06E01B3E0CB0ED11C6D
:10E080003DC0F6018081811108C0B72CD7011C92D8
:10E090006E01B3E0CB0ED11C22C7883239F4B72C05
:10E0A000F7011082FFEFCF1ADF0A19C78B33B9F3DC
:10E0B000A82EB12CC5010E9478E1892B39F4B50155
:10E0C00082EE91E20E94F1E1892B51F047018FEF3E
:10E0D000881A980AC5010E949CE1D7018C937401AB
:10E0E000BFEFCB1ADB0AF70180818111CACFB72CB1
:10E0F000D8018C916E01B3E0CB0ED11CF8011CC08D
:10E100008E32E1F090E0C0970A9790F081818033E1
:10E1100091F4828190E0C0970A9760F4DF01119634
:10E1200011968C9111978D938111FACF808104C043
:10E13000818101C080E331968111E2CFF601A08098
:10E14000A11007C036C0D6011196AC90BFEFCB1A14
:10E15000DB0A76018A2C912CC4010E948CE1892B68
:10E1600091F7C4010E9494E18D369105A1F4F60166
:10E17000818190E00E9494E18337910561F4D6019A
:10E1800012968C9190E00E9494E18736910519F4E3
:10E19000F601339602C0FE013396AA2061F08A2D63
:10E1A000D701893209F41C9211968C918111F9CF13
:10E1B00002C0FE013396BFE2BB1609F468C6808137
:10E1C000882319F0CF010E94255580E1ECEBFCE398
:10E1D000DF011D928A95E9F78BE5E4E8F3E3DF01BF
:10E1E000982F1D929A95E9F7E9E2F3E3DF011D927A
:10E1F0008A95E9F78BE592E30E94464A80932A3399
:10E20000812C912C80E8A82E8FE3B82E55245394AE
:10E2100092E0492E24E0322E23C4C701B6010E94A9
:10E2200024D6862F90E08F35910508F034C6FC0186
:10E23000EC50FF4F0C94FBDD10922A335092853343
:10E240008091BD3C8F5F8093BD3C0AC450922A33BD
:10E25000509285338091BD3C8F5F8093BD3C00C45C
:10E2600040922A33509285338091BD3C8F5F8093DA
:10E27000BD3CF6C383E080932A335092853380916E
:10E28000BD3C8F5F8093BD3CEBC38DE08093293311
:10E2900050928433E5C388E0B2C010925933509253
:10E2A000B4338091BE3C8F5F8093BE3CD9C3509203
:10E2B00059335092B4338091BE3C8F5F8093BE3C03
:10E2C000CFC3409259335092B4338091BE3C8F5F9C
:10E2D0008093BE3CC5C310925A335092B53380919F
:10E2E000C13C8F5F8093C13CBBC350925A33509264
:10E2F000B5338091C13C8F5F8093C13CB1C3C701EE
:10E30000B6010E946FD96C837D838E839F8320E04A
:10E3100030E040E251E4C701B6010E9455D86B01DC
:10E320007C0120E030E040E251E46C817D818E810F
:10E330009F810E9455D89B01AC01C701B6010E9484
:10E3400007D40E9424D6623001F128F4662341F0FC
:10E35000613089F0A0C56330E9F0643001F19BC5FC
:10E36000B5E0B0932933509284338091BC3C8F5FE9
:10E370008093BC3C75C33092293360938433809181
:10E38000BC3C8F5F8093BC3C6BC35092293350924E
:10E39000843366C3409229335092843361C383E04F
:10E3A00080932933509284335BC3C701B6010E9426
:10E3B0006FD96C837D838E839F8320E030E040E2C1
:10E3C00051E4C701B6010E9455D86B017C0120E0E1
:10E3D00030E040E251E46C817D818E819F810E941A
:10E3E00055D89B01AC01C701B6010E9407D40E9419
:10E3F00024D6662319F0613061F04DC587E0809323
:10E400002933509284338091BC3C8F5F8093BC3C15
:10E4100027C3E6E0E0932933609384338091BC3CCA
:10E420008F5F8093BC3C1CC3C701B6010E946FD9AB
:10E430006C837D838E839F8320E030E040E251E453
:10E44000C701B6010E9455D86B017C0120E030E085
:10E4500040E251E46C817D818E819F810E9455D87C
:10E460009B01AC01C701B6010E9407D40E9424D6CB
:10E47000623009F010C58EE08093293350928433C6
:10E48000EFC250925C335092B733EAC250925B3382
:10E490005092B6338091C53C8F5F8093C53CE0C2FB
:10E4A00040925B335092B6338091C53C8F5F80932E
:10E4B000C53CD6C283E016C030925B335092B6336F
:10E4C0008091C53C8F5F8093C53CCAC2F5E0F09354
:10E4D0005B335092B6338091C53C8F5F8093C53CCF
:10E4E000BFC286E080935B335092B6338091C53CC7
:10E4F0008F5F8093C53CB4C2C701B6010E946FD93B
:10E500006C837D838E839F8320E030E040E251E482
:10E51000C701B6010E9455D86B017C0120E030E0B4
:10E5200040E251E46C817D818E819F810E9455D8AB
:10E530009B01AC01C701B6010E9407D40E9424D6FA
:10E54000662319F0613059F0A6C410925E335092E0
:10E55000B9338091C63C8F5F8093C63C81C2609383
:10E560005E336093B9338091C63C8F5F8093C63C25
:10E5700077C240925E335092B9338091C63C8F5F30
:10E580008093C63C6DC230922A335092853380917D
:10E59000BD3C8F5F8093BD3C63C2C701B6010E9442
:10E5A0006FD96C837D838E839F8320E030E040E2CF
:10E5B00051E4C701B6010E9455D86B017C0120E0EF
:10E5C00030E040E251E46C817D818E819F810E9428
:10E5D00055D89B01AC01C701B6010E9407D40E9427
:10E5E00024D6662319F0613059F055C410925F3378
:10E5F0005092BA338091BF3C8F5F8093BF3C30C252
:10E60000109260336093BB338091BF3C8F5F8093E7
:10E61000BF3C26C2C701B6010E946FD96C837D83BF
:10E620008E839F8320E030E040E251E4C701B601D1
:10E630000E9455D86B017C0120E030E040E251E4BB
:10E640006C817D818E819F810E9455D89B01AC0198
:10E65000C701B6010E9407D40E9424D6662319F090
:10E66000613059F018C450925F335092BA338091A0
:10E67000BF3C8F5F8093BF3CF3C160936033609376
:10E68000BB338091BF3C8F5F8093BF3CE9C1C70122
:10E69000B6010E946FD96C837D838E839F8320E0B7
:10E6A00030E040E251E4C701B6010E9455D86B0149
:10E6B0007C0120E030E040E251E46C817D818E817C
:10E6C0009F810E9455D89B01AC01C701B6010E94F1
:10E6D00007D40E9424D6613089F028F06230A1F07E
:10E6E0006330C1F0D8C399E09093293350928433BA
:10E6F0008091BC3C8F5F8093BC3CB2C1AAE0A093E8
:10E70000293360938433ACC1BBE0B093293350927A
:10E710008433A6C1ECE0E093293350928433A0C146
:10E72000109254335092AF338091C03C8F5F8093EE
:10E73000C03C96C1509254335092AF338091C03C4C
:10E740008F5F8093C03C8CC1C701B6010E9424D664
:10E75000862F90E08D33910508F09BC3FC01ED5AA4
:10E76000FE4F0C94FBDD10922B3350928633809138
:10E77000C73C8F5F8093C73C73C150922B3350923C
:10E7800086338091C73C8F5F8093C73C69C15092AC
:10E7900066335092C1338091C93C8F5F8093C93CEE
:10E7A0005FC1409266335092C1338091C93C8F5F04
:10E7B0008093C93C55C1109266335092C133809109
:10E7C000C93C8F5F8093C93C4BC1509263335092D8
:10E7D000BE3346C1509264335092BF338091CA3CDD
:10E7E0008F5F8093CA3C3CC1509265335092C033D6
:10E7F0008091CA3C8F5F8093CA3C32C110926533CE
:10E800005092C0338091CA3C8F5F8093CA3C28C12C
:10E81000509257335092B2338091CB3C8F5F8093AC
:10E82000CB3C1EC1109257335092B2338091CB3CF7
:10E830008F5F8093CB3C14C1509255335092B033CC
:10E840008091CB3C8F5F8093CB3C0AC150926F3359
:10E850005092CA338091CB3C8F5F8093CB3C00C1F8
:10E86000C701B6010E946FD90E9424D6609362331B
:10E870005092BD33F5C0C0924833D0924933E092F4
:10E880004A33F0924B338092A3339092A433A092F8
:10E89000A533B092A633E4C0C0927033D0927133E6
:10E8A000E0927233F09273338092CB339092CC33F8
:10E8B000A092CD33B092CE33D3C0C0926733D09202
:10E8C0006833E0926933F0926A338092C233909257
:10E8D000C333A092C433B092C533C2C0C0923033A8
:10E8E000D0923133E0923233F092333380928B33D3
:10E8F00090928C33A0928D33B0928E33B1C0C0927F
:10E900003433D0923533E0923633F09237338092FD
:10E910008F3390929033A0929133B0929233A0C0F3
:10E92000C0923833D0923933E0923A33F0923B338D
:10E930008092933390929433A0929533B092963311
:10E940008FC0C0923C33D0923D33E0923E33F09280
:10E950003F338092973390929833A0929933B0923C
:10E960009A337EC0C0924033D0924133E09242331A
:10E97000F092433380929B3390929C33A0929D33CC
:10E98000B0929E336DC0C0924433D0924533E09232
:10E990004633F092473380929F339092A033A092F7
:10E9A000A133B092A2335CC0C0927833D092793355
:10E9B000E0927A33F0927B338092D3339092D433C7
:10E9C000A092D533B092D6334BC0C0927C33D09254
:10E9D0007D33E0927E33F0927F338092D7339092F2
:10E9E000D833A092D933B092DA333AC0C092803390
:10E9F000D0928133E0928233F09283338092DB3382
:10EA00009092DC33A092DD33B092DE3329C0C09205
:10EA10007433D0927533E0927633F09277338092EC
:10EA2000CF339092D033A092D133B092D23318C06A
:10EA3000C701B6010E9424D660932C3370932D3306
:10EA400080932E3390932F3381E090E0A0E0B0E0EC
:10EA50008093873390938833A0938933B0938A331C
:10EA6000D8012C90222009F424C2822D90E00E942B
:10EA700083E1892B09F42FC23801BFEF6B1A7B0A9F
:10EA8000F8018181803349F48281883531F40E5F49
:10EA90001F4FC12CD12C760100C2BE016F5F7F4F8A
:10EAA000C3010E941BDE6B017C0109811A81601683
:10EAB000710609F0F2C111C2809154330E94E852EC
:10EAC000182F01C010E06091A3337091A43380919E
:10EAD000A5339091A6330E9424D6662359F0609105
:10EAE00048337091493380914A3390914B330E945F
:10EAF000B752182F6091A7337091A8338091A93332
:10EB00009091AA330E9424D6662371F060914C3311
:10EB100070914D3380914E3390914F330E9424D6A3
:10EB2000862F0E949354182F6091AB337091AC33B1
:10EB30008091AD339091AE330E9424D6662371F05C
:10EB4000609150337091513380915233909153338F
:10EB50000E9424D6862F0E94D254182F6091C2336F
:10EB60007091C3338091C4339091C5330E9424D6F1
:10EB7000662359F0609167337091683380916933EF
:10EB800090916A330E94E5AE182F6091C633709160
:10EB9000C7338091C8339091C9330E9424D666232D
:10EBA00071F060916B3370916C3380916D33909103
:10EBB0006E330E9424D6862F0E941155182F809103
:10EBC000BD33882329F0809162330E945053182F5F
:10EBD0008091BE33882329F0809163330E9484534F
:10EBE000182F8091C133882329F0809166330E94C9
:10EBF000B1AE182F8091BF33882329F08091643300
:10EC00000E94B953182F8091C033882329F0809136
:10EC100065330E94ED53182F8091B033882329F07B
:10EC2000809155330E946854182F8091B133882306
:10EC300029F0809156330E94A754182F8091CA332F
:10EC4000882329F080916F330E94E654182F809119
:10EC5000B233882329F0809157330E946054182FD3
:10EC6000809129338D3029F08091B4338823A9F025
:10EC70000FC06091703370917133809172339091B5
:10EC800073330E94F0528093243D882369F32FC18F
:10EC9000809159330E947F4E182F8091B53388237D
:10ECA00029F080915A330E94834E182F8091B633F9
:10ECB000882329F080915B330E943D4F182F80916B
:10ECC000B933882329F080915E330E94EC52182FCB
:10ECD0008091BA33882329F080915F330E94874E58
:10ECE000182F4091293350E04F30510508F0B6C03D
:10ECF000FA01E057FE4F0C94FBDD0E943952182FA9
:10ED0000ADC06BE873E380E393E30E944452182F95
:10ED1000A5C00E947852182FA1C06BE873E380E36E
:10ED200093E30E948352182F99C00E94CC6A182F37
:10ED300095C06BE873E380E393E30E940350182FC0
:10ED40008DC00E94156B182F89C06BE873E380E3B8
:10ED500093E30E944B6F182F81C0609170337091C4
:10ED6000713380917233909173330E9424D6862F31
:10ED70002BE833E340E353E3609158330E948B4E1A
:10ED8000182F6CC06BE873E380E393E30E9480501C
:10ED9000182F64C00E943351182F60C00E949A51EE
:10EDA000182F5CC00E94D151182F58C060915C335D
:10EDB0008BE592E30E94E14A80912A33843038F453
:10EDC0008230D8F4882349F0813079F047C084300C
:10EDD00009F044C080935F3241C06BE873E380E385
:10EDE00093E30E940952182F39C06BE873E380E364
:10EDF00093E30E94FC52182F31C0A0908033B09052
:10EE00008133C0908233D0908333E0907C33F09094
:10EE10007D3300917E3310917F3320917833309190
:10EE2000793340917A3350917B338F93809177334C
:10EE30008F93809176338F93809175338F938091E8
:10EE400074338F936BE873E380E393E30E942A8427
:10EE5000182F0F900F900F900F900F9060E08BE5A0
:10EE600092E30E94E14A80918633813061F480917F
:10EE70002B33811104C00E941256812F38C00E948A
:10EE80004356812F34C0812F32C08BEC30C083E0D9
:10EE90002EC084E82CC083E82AC0822D90E0FC01BB
:10EEA000E154F109EA31F105B0F7E156FE4F0C9457
:10EEB000FBDD1092243D60912C3370912D338091B5
:10EEC0002E3390912F330E947B4A8091AF33882359
:10EED00009F4F8CDF1CD85E60AC086E608C0D80170
:10EEE0008C910CC968018B2D78017B2CD6C8279694
:10EEF000CDBFDEBFDF91CF911F910F91FF90EF90BB
:10EF0000DF90CF90BF90AF909F908F907F906F9049
:10EF10005F904F903F902F900895CF93DF93EC0137
:10EF20006AE17CE30E94A9618093243D811102C0C3
:10EF300095E09F83DF91CF910895FC018789908DA3
:10EF40000C94197083FF06C0E091FD2FF091FE2F05
:10EF500090E2958382FF06C0E091FF2FF091003090
:10EF600090E2958381FF06C0E0910130F09102307C
:10EF700090E2958380FF06C0E0910330F091043069
:10EF800080E28583089583FF06C0E091FD2FF09114
:10EF9000FE2F90E2968382FF06C0E091FF2FF09152
:10EFA000003090E2968381FF06C0E0910130F0913D
:10EFB000023090E2968380FF06C0E0910330F0912A
:10EFC000043080E2868308958091FA39811107C068
:10EFD00084E00E94A27781E08093FA39089584E06A
:10EFE0000E94C3771092FA390895CF92DF92EF9280
:10EFF000FF920F931F93CF93DF93C12C26E0D22E65
:10F00000C092ED2FD092EE2F30EAE32E36E0F32EB1
:10F01000E092EF2FF092F02F00E816E00093F12F2E
:10F020001093F22FC0E6D6E0C093F32FD093F42FC5
:10F03000C092F52FD092F62FC093F72FD093F82FD0
:10F040000093F92F1093FA2FE092FB2FF092FC2FF0
:10F050002DEC3CEC4CED50E40E94B3D7C092FD2F58
:10F06000D092FE2FE092FF2FF092003018164CF451
:10F07000C0930130D09302300093033010930430DA
:10F0800008C00093013010930230C0930330D09336
:10F090000430DF91CF911F910F91FF90EF90DF909F
:10F0A000CF9008950E945AD360E070E080E091E430
:10F0B0000E94F5770C9479D381E08093033A089508
:10F0C00020E093E088ED08B618BE84BF90938000DE
:10F0D0002091820021FDFCCF08BEFFCF8091033A32
:10F0E00081110E94607883E008958091043A88231A
:10F0F00041F0F89461E089E790E00E945CD382E0FF
:10F10000089583E00895CF93DF93CDB7DEB7AD9731
:10F11000CDBFDEBF21E2E5EEF1E2DE011196019006
:10F120000D922A95E1F722E02093CA01DE01929622
:10F13000E8E0F0E024912D933196EE30F105D1F71F
:10F140002DE228A7E0E1F0E0E491EF7121E030E06A
:10F150002C0F3D1F2E0F311DF901208129A7E2E15F
:10F16000F0E0E491EF719E012E0F311DF901218134
:10F170002AA7E4E1F0E0E491EF719E012E0F311D2A
:10F18000F90121812BA71CA61092CA0125E0FC01E0
:10F190002783BE016E5D7F4F0E94A9618093243D4D
:10F1A000AD96CDBFDEBFDF91CF91089581E0809312
:10F1B000043A80E00895CF93DF93EC0120E030E043
:10F1C00040E051E469857A858B859C850E94B3D7A0
:10F1D00018166CF0CE010E94D25E69857A858B8507
:10F1E0009C850E94F5770E9455BC80E001C08DE6A9
:10F1F000DF91CF91089564E87BE30C94E0C166E66B
:10F200007BE30C94E0C167E47BE30C94E0C169E22A
:10F210007BE30C94E0C165E17BE30C948BC1CF935D
:10F22000DF938AEC96E49F938F93CCEDD9E58981A7
:10F230008F9388818F930E948AE284E994E49F935C
:10F240008F9389818F9388818F930E948AE28CE0CB
:10F2500094E49F938F9389818F9388818F930E94E9
:10F260008AE282E493E49F938F9389818F938881CC
:10F270008F930E948AE20E9417A88DB79EB740968E
:10F280008DBF9EBF80E0DF91CF910895CF93DF9334
:10F290008DE193E49F938F93CCEDD9E589818F9392
:10F2A00088818F930E948AE28FEA91E49F938F93E3
:10F2B00089818F9388818F930E948AE284E290E40F
:10F2C0009F938F9389818F9388818F930E948AE285
:10F2D0008CE094E49F938F9389818F9388818F939F
:10F2E0000E948AE282E493E49F938F9389818F93B3
:10F2F00088818F930E948AE28DB79EB744968DBF16
:10F300009EBF80E0DF91CF910895CF93DF9383E09C
:10F3100090E49F938F93CCEDD9E589818F93888179
:10F320008F930E948AE285E89CE39F938F93898163
:10F330008F9388818F930E948AE282E493E49F9363
:10F340008F9389818F9388818F930E948AE28DB7F2
:10F350009EB70C968DBF9EBF80E0DF91CF91089540
:10F36000CF93DF938DE59CE39F938F93CCEDD9E50D
:10F3700089818F9388818F930E948AE28CEE9BE330
:10F380009F938F9389818F9388818F930E948AE2C4
:10F3900082E493E49F938F9389818F9388818F93E5
:10F3A0000E948AE28DB79EB70C968DBF9EBF80E00B
:10F3B000DF91CF910895CF93DF9389EC9BE39F93E7
:10F3C0008F93CCEDD9E589818F9388818F930E94AB
:10F3D0008AE280EA9BE39F938F9389818F93888150
:10F3E0008F930E948AE282E493E49F938F938981B2
:10F3F0008F9388818F930E948AE28DB79EB70C9677
:10F400008DBF9EBF80E0DF91CF9108952F923F92F4
:10F410004F925F926F927F928F929F92AF92BF9224
:10F42000CF92DF92EF92FF920F931F93CF93DF93D0
:10F43000CDB7DEB76A97CDBFDEBF5C010E94E96041
:10F440002C011F86188A198A1A8AF501019000205A
:10F45000E9F73197EA19FB09E130F24008F002C2FE
:10F46000D5018C91882359F17501BFEFEB1AFB0A86
:10F47000850120E0211115C0883229F08132C8F0C1
:10F480008F37B9F001C021E06801EFEFCE1ADE0A34
:10F4900090E02A8F0E9494E1D8018C9386012A8DF6
:10F4A00008C021E0893209F420E0F80180830F5F71
:10F4B0001F4FD7018D917D018111DCCF01C08501E6
:10F4C000F80110821092243DFDE19F2EAAE36A2EDE
:10F4D000A2E27A2E812CB6E02B2E03C09A9409F476
:10F4E0009CC18BE79CE2A2E2B0E08B879C87AD8752
:10F4F000BE876B8A7C8A8D8A8DE79CE2A2E2B0E0AF
:10F500008F839887A987BA87E6E0F2E2DE01119639
:10F51000822D01900D928A95E1F7C2010E94F05F61
:10F520008501075F1F4F75019FEFA91AB90AD7011F
:10F530006C9170E0CE010B960E94F1E1892B21F4D1
:10F5400087010E5D1F4F04C0A016B10661F793C17D
:10F550006501BFEFAB1ABB0AF601608170E0CE0116
:10F5600043960E94F1E1892B91F0D6011D928D0105
:10F5700092012F5E3F4F288F398F46E050E0B70150
:10F58000C9010E941CE23AE0C30ED11C04C0A016BF
:10F59000B106F1F670C15801D8013D908D01E32C00
:10F5A000F12CC7010E9478E1892B59F4B701CE01F3
:10F5B00001960E94F1E1892B21F40C151D0559F7E4
:10F5C0005AC18501BEE63B1641F0E2E23E120CC094
:10F5D000D50111968C918232A9F5F201178211861C
:10F5E000128613861486A3C0B0E3EB1AF108EAE092
:10F5F000EE16F10418F0FDE23F1217C0BE016A5E7C
:10F600007F4FC5010E941BDED20119966D937D9339
:10F610008D939C931C978E899F898A159B0509F46D
:10F620002DC1E4E01796EC9382C0FBE73F124FC078
:10F63000E7E0D2011796EC93FFEFAF1ABF0AE2E0C2
:10F64000FE2E95C02FEFA21AB20AE5E0D20117965E
:10F65000EC9362E270E0C5010E94F1E18E8B9F8B1A
:10F66000009709F408C1DC011C92F501019000200B
:10F67000E9F73197EA19FB093397C8F0F80181815E
:10F680008033A9F48281883791F440E050E060E053
:10F6900070E0C5010E948CDFD20119966D937D93B5
:10F6A0008D939C931C9783E017968C9308C0B501AB
:10F6B000C2010E94A9618093243D811153C0AE888C
:10F6C000BF88BFEFAB1ABB0AAE8ABF8A30C0E4E77F
:10F6D0003E120EC0E1E0D2011796EC9380E090E07C
:10F6E000A0E8BFE3F20181879287A387B4871FC098
:10F6F000F6E63F120CC0E1E0D2011796EC931797A3
:10F7000019961D921D921D921C921C9710C0BBE56C
:10F710003B12B1C0F2012782B501C2010E94A9616A
:10F720008093243D81111EC077E6F72E7DC0BE0177
:10F73000695F7F4FC5010E9436E25C01009709F4C2
:10F740009AC0DC018C918D3729F411968C91F501CA
:10F7500031965F018C3209F48BC0FFEFAF1ABF0AFC
:10F76000F12C05C0F82E22E0281708F45DC08F8523
:10F770008201035F1F4F882341F043E050E0BE0148
:10F78000615F7F4FC8010E941CE2688D798DC801BE
:10F790000E94495FD20114968D939C9315978F3FD9
:10F7A000BFEF9B07B9F10E948064882371F0888DB8
:10F7B000998D0E94325F882341F043E050E0688DCC
:10F7C000798DCE010F960E941CE2F2014280538097
:10F7D0004114510411F1F11081CE80918E348111C8
:10F7E00008C087E894E30E94E55B8093243DF82EEF
:10F7F0001BC080912B32823099F087E894E30E94FD
:10F80000BB5B8093243D81110EC087E894E30E9486
:10F81000385C0AC064E6F62E07C050E7F52E04C037
:10F820004BECF42E01C0F82E42E060E08F2D0E94D8
:10F83000506281E00E9476AA6A96CDBFDEBFDF915A
:10F84000CF911F910F91FF90EF90DF90CF90BF90DD
:10F85000AF909F908F907F906F905F904F903F9070
:10F860002F9008958BE68093243D3BE6F32EDCCF6A
:10F8700022E0F22E7CCF9FE6F92ED6CF86E6F82E38
:10F88000D3CF2F923F924F925F926F927F928F923F
:10F890009F92AF92BF92CF92DF92EF92FF920F931F
:10F8A0001F93CF93DF9300D000D0CDB7DEB78C018C
:10F8B00069837A834B835C835A0128E0A21AB108DA
:10F8C000A60EB71EDC0116967C907B01BFEFEB1AEB
:10F8D000FB0A8BE7FB01808380E0912C95E0692E89
:10F8E00020E1422E22E2522E3CE0232E32E2332E41
:10F8F0004DE7842EED82FE82D80117969C919F3FA2
:10F9000009F429C1882339F02CE2ED81FE8120839E
:10F910003196ED83FE838091CE3C811119C0C801E0
:10F9200041969F938F933F922F923E813F938D817B
:10F930008F930E9455E3AD81BE81A80FB91FAD839F
:10F94000BE830F900F900F900F900F900F9018C0E4
:10F95000C80141969F938F935F924F92BE81BF9350
:10F96000ED81EF930E9455E32D813E81280F391FD1
:10F970002D833E830F900F900F900F900F900F905C
:10F98000D80117968C911797843059F51996CD9018
:10F99000DD90ED90FC901C97A7019601C701B60180
:10F9A0000E9476D9811117C0E894F7F82FEF3FEF46
:10F9B0004FE75FE7C701B6010E9476D9811121C1E7
:10F9C0002FEF3FEF4FE75FE7C701B6010E94B0D5C9
:10F9D00018160CF016C1F8011186128613861486CB
:10F9E00010C1811113C0E6E1F2E2AD81BE81862D26
:10F9F00001900D928A95E1F72D813E812C5F3F4F5A
:10FA00002D833E83D80117968C9199C0823061F482
:10FA1000F80184858F9383858F9382858F93818569
:10FA20008F93ABE1B2E214C0833029F5D8011C9664
:10FA30008C911C978F931B968C911B978F931A9682
:10FA40008C911A978F9319968C918F93A1E2B2E2C1
:10FA5000BF93AF93FE81FF932D812F930E9455E3B7
:10FA6000AD81BE81A80FB11DAD83BE83F801878132
:10FA7000CDBFDEBF64C0853059F4D80158968C9153
:10FA800058978F9357968C918F93A9E2B2E20CC04E
:10FA9000863009F5D80158968C9158978F935796D0
:10FAA0008C918F93AEE2B2E2BF93AF93FE81FF934E
:10FAB0002D812F930E9455E3AD81BE81A80FB11D0A
:10FAC000AD83BE83F80187810F900F900F900F9048
:10FAD0000F900F9034C0813091F52CEA35EC47E25D
:10FAE00057E3D80119966D917D918D919C911C974A
:10FAF0000E94B0D587FF12C0E3E3F2E2AD81BE8180
:10FB000086E001900D928A95E1F7ED81FE813596B0
:10FB1000ED83FE83D80117968C9111C0E9E3F2E2E0
:10FB2000AD81BE81862D01900D928A95E1F7ED8120
:10FB3000FE813496ED83FE83D80117968C91873031
:10FB400049F42BE7ED81FE8120833196ED83FE831E
:10FB500080E001C081E0AD81BE81AA15BB0518F02F
:10FB60008FEF9FEF65C0F801028113810115110528
:10FB700049F0D80116969C912FEF290D99153CF06C
:10FB8000992EBACEED80FE807914B4F020C0ED81BC
:10FB9000FE81D801CF010196808216969C9016971F
:10FBA0003FEF320F92161CF4232FFC01F3CF8D830D
:10FBB0009E838D0181E0A0CEF7012DE7CF01019654
:10FBC00020839A94791414F4FC01F8CF7C018DE71A
:10FBD0009AE0A0E0F70180839183A283F2E0EF0E28
:10FBE000F11C89819A812B813C81820F931F8E1594
:10FBF0009F0508F4B5CFC701A981BA818A1B9B0B69
:10FC000017C0C8010E949064F80141855285638540
:10FC1000748520858D819E810E9424C42D813E8122
:10FC2000280F311D2D833E83D80117968C9187CFE5
:10FC30002696CDBFDEBFDF91CF911F910F91FF9030
:10FC4000EF90DF90CF90BF90AF909F908F907F907C
:10FC50006F905F904F903F902F90089540E052E05A
:10FC60006AE17AE30E94417C6091DC597091DD5930
:10FC70008AE19AE30C94D9E2EF92FF920F931F93DB
:10FC8000CF93DF93CDB7DEB76297CDBFDEBFF82E3F
:10FC90009091CC3C992309F4B2C08FE6F81212C0BF
:10FCA0000E94E9606AE17CE38091163A9091173AEC
:10FCB0000E9404C4BC018CE091E20E94076207E844
:10FCC00014E34AC080912B3207E814E3882309F437
:10FCD00043C0EE24EA94C8010E94B05F8823E1F19A
:10FCE000823029F48091D33C811120C01DC0843022
:10FCF00029F48091D03C811119C016C08530B1F42F
:10FD00008091D23C882381F0F80181859285A3857A
:10FD1000B485BC01CD019F772CEA35EC47E257E36F
:10FD20000E94B0D587FF02C0F801E782F801028186
:10FD300013810115110579F60FC0F80102811381B5
:10FD40000115110549F440E052E06AE17AE38EE6DC
:10FD500094E30E94417C53C0F80197819F3F69F76B
:10FD60008091E52F81111AC08091193A8F9380916B
:10FD7000183A8F931F92FF928EE392E29F938F9394
:10FD8000CE0101967C01FF928F930E9455E3109261
:10FD9000183A1092193ACDBFDEBF13C00E9454C961
:10FDA0001F928F931F92FF9286E492E29F938F930C
:10FDB000CE0101967C01FF928F930E9455E3CDBF47
:10FDC000DEBFB701C8010E94A961F801168286E072
:10FDD000878386E690E0818B928B1282138240E0CB
:10FDE00052E06AE17AE38EE694E30E94417C6091FE
:10FDF000DC597091DD598AE19AE30E94D9E262965A
:10FE0000CDBFDEBFDF91CF911F910F91FF90EF909B
:10FE10000895613019F0623029F0089587E894E37D
:10FE20000C942E7E0C943C7ECF92DF92EF92FF9248
:10FE3000FC01C184D284E384F48420E030E040EA11
:10FE400050E4C701B6010E94B3D718160CF453C092
:10FE5000C701B6010E9424D66093CC3C1092CF3CDF
:10FE60001092D03C1092D13C1092D23C1092D33CD4
:10FE700020E030E040E85FE3C701B6010E94B3D75D
:10FE800087FD03C081E08093CF3C20E030E040E07C
:10FE900050E4C701B6010E94B3D787FD03C081E0DB
:10FEA0008093D03C20E030E040E450E4C701B6014C
:10FEB0000E94B3D787FD03C081E08093D13C20E04E
:10FEC00030E040E850E4C701B6010E94B3D787FD97
:10FED00003C081E08093D23C20E030E040EA50E46F
:10FEE000C701B6010E94B3D787FD07C081E08093A8
:10FEF000D33C80E003C08EE601C080E0FF90EF902D
:10FF0000DF90CF9008956CE677E40C94A1C165E191
:10FF100077E40C94A1C161EE76E40C94A1C1BF9288
:10FF2000CF92DF92EF92FF920F931F93CF93DF93C5
:10FF3000CDB7DEB76897CDBFDEBF6B0128E1FC010E
:10FF4000DE01119601900D922A95E1F78CEEE82ED4
:10FF500080E3F82E8E010F5F1F4FB12CF7018081D7
:10FF6000823029F4F801108211821282138280916A
:10FF70005E588B1114C02091715830917258409185
:10FF8000735850917458F801608171818281938116
:10FF90000E9455D8F6016083718382839383809198
:10FFA0007D588B1114C020919058309191584091F8
:10FFB000925850919358F8016081718182819381A8
:10FFC0000E9455D8F6016483758386839783809158
:10FFD0009C588B1114C02091AF583091B05840916B
:10FFE000B1585091B258F80160817181828193813A
:10FFF0000E9455D8F6016087718782879387809128
:020000021000EC
:10000000BB588B1114C02091CE583091CF584091DD
:10001000D0585091D158F8016081718182819381CB
:100020000E9455D8F6016487758786879787B394B1
:10003000F5E3EF0EF11C0C5F1F4F86E0B8128ECF78
:100040006896CDBFDEBFDF91CF911F910F91FF90DA
:10005000EF90DF90CF90BF900895F8940E9452786F
:100060000E9484800E9479D30E9417C60E9410B318
:100070000E94D46F0E9455BC0E946CA540E060E0D5
:1000800080E00E9486650E9426610E9472800E9424
:1000900076820E94734F0E9471D38091A200846087
:1000A0008093A2008091A20082608093A200809140
:1000B000A20081608093A20078940E9417A80E94F9
:1000C00062BD0E94ED65FDCFE82FF0E0EE0FFF1F4F
:1000D000E856F84B659174914FE450E084ED9CE351
:1000E0000C94C3E18091F739823041F440E060E044
:1000F00081E00E94866580E00E9415670C944DCADD
:10010000682F81E00C94F4C61092253D1092263D94
:100110001092273D1092283D0895CF93DF93EC0174
:100120008C819D81880F991F880F991F2091273DF1
:100130003091283D820F931F8093293D90932A3D53
:1001400044E050E06FE27DE30E9471D240912F3D88
:100150005091303D6091313D7091323D49875A87D1
:100160006B877C8780E0DF91CF9108958F929F927B
:10017000AF92BF92CF92DF92EF92FF92CF93DF9335
:10018000EC0180912C32882369F089E0DF91CF91D6
:10019000FF90EF90DF90CF90BF90AF909F908F90A7
:1001A0000C949FA789859A85AB85BC8580932B3D50
:1001B00090932C3DA0932D3DB0932E3DCE010E94F7
:1001C0008D808093243D81116EC0C984DA84EB84D4
:1001D000FC84A7019601C701B6010E9476D981115E
:1001E0002FC046015701E894B7F82FEF3FEF4FE7D4
:1001F0005FE7C501B4010E9476D981110AC02FEFD3
:100200003FEF4FE75FE7C501B4010E94B0D5181674
:10021000BCF080902B3D90902C3DA0902D3DB09057
:100220002E3DA5019401C701B6010E9407D49F7716
:100230002CEA35EC47E257E30E94B3D7181674F561
:1002400080912B3D90912C3DA0912D3DB0912E3D64
:1002500080932F3D9093303DA093313DB093323D3C
:100260008C819D81880F991F880F991F2091273DB0
:100270003091283D820F931F8093293D90932A3D12
:1002800044E050E06FE27DE30E9402D380902B3D7A
:1002900090902C3DA0902D3DB0902E3D89869A8661
:1002A000AB86BC8680E0DF91CF91FF90EF90DF902E
:1002B000CF90BF90AF909F908F9008950E946BB8A1
:1002C00080E008958091333D9091343D8F3E92417E
:1002D00011F08EE508958091593D90915A3D8F3EE1
:1002E0009241B9F780915B3D90915C3D8F3E924188
:1002F00081F78091E4549091E5548F3E924149F703
:100300008091E6549091E7548F3E924111F780918D
:10031000795690917A568F3E9241D9F680E00895B1
:1003200094E0899FF0011124ED5CF24C42835383E9
:1003300064837583089594E0899FF0011124EA5144
:10034000FB4A45AB56AB67AB70AF08955F926F92B7
:100350007F928F929F92AF92BF92CF92DF92EF9255
:10036000FF920F931F93CF93DF93CDB7DEB76097C4
:10037000CDBFDEBFBE016F5F7F4F8BE195E50E9471
:100380008F7FCE0101964C0183E9A82E85E5B82E1A
:1003900093EAC92E95E5D92E23EBE22E25E5F22E20
:1003A00003ED15E535EF632E38E5732E512CF4017E
:1003B00041915191619171914F01F5014193519397
:1003C000619371935F01F60141935193619371932E
:1003D0006F01F70141935193619371937F01852DD3
:1003E0000E94F66FF80111921192119211928F01F1
:1003F000F30110821182128213825394F8E16F0E7E
:10040000711C84E05812D3CF6096CDBFDEBFDF9160
:10041000CF911F910F91FF90EF90DF90CF90BF9001
:10042000AF909F908F907F906F905F900895809194
:100430005D3D08951F93CF93DF938BE897E1EBE544
:10044000FDE3DF019C011D9221503040E1F78FEE6A
:1004500092E180935B3D90935C3D8093E454909354
:10046000E554C4E6DDE3C0935E3DD0935F3DC093A9
:10047000603DD093613DC093623DD093633D81E088
:1004800090E068E274E520E030E01CEB129FA001F0
:10049000139F500D1124FA01E55AF24CD90111961F
:1004A0001A9F90011B9F300D11242C59324C238729
:1004B000348761877287BA016C59724C9C0101962E
:1004C0008032910519F78CEB829FF001839FF00D2C
:1004D0001124E55AF24CC387D4876187728780E282
:1004E00080935D3DDF91CF911F910895CF93DF936E
:1004F000E6EEF4E585E991E0DF01EC011D9221973C
:10050000E9F7A3E3BDE388E2ED0119928A95E9F7E3
:100510008FEE92E18D939C938093593D90935A3D39
:10052000808391838093795690937A56DF91CF910F
:100530000C941A820E94938C0E941A8280E00C9480
:10054000304AE0915E3DF0915F3D848581111BC092
:1005500022813381808191814CEBDF011D924A958C
:10056000E9F7228333838083918381E084878091BC
:100570005D3D815080935D3D8281938180935E3D9E
:1005800090935F3D05C08CE10E949FA7E0E0F0E002
:10059000CF010895A0E6BDE3ED91FC911197858709
:1005A00081E0878782E08487828193818D939C9309
:1005B00081E00E94C7AB0C94B1B5EF92FF920F930C
:1005C0001F93CF93DF9300D01F92CDB7DEB78C017E
:1005D0004B835C8369837A830E94A182FC014B81F7
:1005E0005C8169817A81009761F48EE02496CDBFA9
:1005F000DEBFDF91CF911F910F91FF90EF900C9490
:100600006F4E83E085878EE591E88483958306832A
:1006100017838B017A0126E0D8014D915D916D9190
:100620007D918D01CF0185599F4FDC014D935D93E5
:100630006D937C931397D7014D915D916D917D9151
:100640007D01418B528B638B748B21503496211129
:10065000E3CF83E02496CDBFDEBFDF91CF911F9122
:100660000F91FF90EF900C94CA82CF92DF92EF929D
:10067000FF926B017C010E94A182009739F48EE009
:10068000FF90EF90DF90CF900C946F4E28EB33E803
:10069000FC0124833583E556FF4FC082D182E2827C
:1006A000F38221E0FC01278782E00E94CA8280E079
:1006B000FF90EF90DF90CF9008958091623D9091F0
:1006C000633DFC0124853EEF320F323018F424E004
:1006D00024870895243011F080E090E00895E0919F
:1006E000623DF091633D22813381808191814CEBA9
:1006F000DF011D924A95E9F722833383808391833A
:10070000E091623DF091633D0280F381E02DE09342
:10071000623DF093633D8485823011F483E08487E9
:1007200080915D3D8F5F80935D3D8FEF0E94C7ABF1
:1007300081E040915E3D50915F3D2091623D30915E
:10074000633D4217530709F080E00895BC016F5ED6
:100750007F4FDC011696ED91FC91179785599F4FBD
:1007600019950E946F8381110E94DF5580E00895E2
:1007700085569F4F20E034E244E759E4FC01608154
:100780007181828193810E9455D80E9424D60E9453
:1007900050D60E9475B80E946F8381110E94DF5568
:1007A00080E008958091623D9091633DFC01248535
:1007B0003EEF320F323018F424E0248708952430BD
:1007C00011F080E090E00895CF93DF93C091623DF7
:1007D000D091633D8C859EEF980F923018F484E0A1
:1007E0008C8705C0843019F080E090E010C020971D
:1007F000D9F3DE011296ED91FC911397878588233A
:1008000029F0EC17FD0711F0DF01F4CFCD01DF91E6
:10081000CF910895CF93DF93EC012A813B818881AA
:1008200099814CEBFB01DE0101900D924A95E1F7B5
:100830002A833B8388839983DF91CF9108958FEE3C
:1008400092E180937B5690937C5680933857909397
:10085000395708952F923F924F925F926F927F92F5
:100860008F929F92AF92BF92CF92DF92EF92FF92C0
:100870000F931F93CF93DF93CDB7DEB76A97CDBFAA
:10088000DEBF4C011B0129013A01E986FA860B877C
:100890001C871A2D0B2DE8A8B9A8AAA82BA9298373
:1008A0008091A432882399F0809198329091993266
:1008B000A0919A32B0919B32BC01CD019F772CEA76
:1008C00035EC47E257E30E94B0D587FD11C7809110
:1008D000CF339091D033A091D133B091D233BC01BA
:1008E000CD019F7731E03D832CEA35EC47E257E3B9
:1008F0000E94B3D7181614F01D8210C02DEC3CECEA
:100900004CEC5DE360917433709175338091763374
:10091000909177330E94B0D587FDECC6F1018081BC
:100920009181A281B381BC01CD019F77F1E0FD8768
:100930002CEA35EC47E257E30E94B3D718160CF0C7
:100940001D86F10184819581A681B781BC01CD010D
:100950009F77F1E0F98B2CEA35EC47E257E30E94F0
:10096000B3D718160CF0198AF10180859185A285FC
:10097000B3852091D3333091D4334091D533509106
:10098000D6332E8B3F8B488F598F2091D7333091A0
:10099000D8334091D9335091DA332A8B3B8B4C8B2F
:1009A0005D8B4091DB335091DC336091DD3370918E
:1009B000DE33F090A532F11021C01092C35681E0D1
:1009C0008093C45682E08093C5563D81332341F025
:1009D0004D85411195C65989511192C68CE9C1C600
:1009E000CB01BA019F772CEA35EC47E257E30E942E
:1009F000B3D718160CF089C68BE9B3C6BC01CD017C
:100A00009F77A1E0AA8F2CEA35EC47E257E30E94DA
:100A1000B3D718160CF01A8EB1E0FB1216C0109264
:100A2000C35682E08093C456F092C556ED81EE2302
:100A300039F0FD85F11164C62A8D222379F260C652
:100A40006A897B898C899D89CDCF32E0F31217C0EA
:100A500081E08093C356F092C4561092C5564D81E2
:100A6000442341F0598951114BC68A8D882309F4DA
:100A7000B5CF46C66E897F89888D998DB3CFB10178
:100A8000C4010E947F4C9D81992309F451C020919B
:100A900060323091613240916232509163326091A4
:100AA000B5327091B6328091B7329091B8320E94CF
:100AB00007D49F772CEA35EC47E257E30E94B0D584
:100AC00087FF36C0209164323091653240916632A2
:100AD000509167326091B9327091BA328091BB32D5
:100AE0009091BC320E9407D49F772CEA35EC47E204
:100AF00057E30E94B0D587FF1BC020916832309128
:100B0000693240916A3250916B326091BD3270917E
:100B1000BE328091BF329091C0320E9407D49F773D
:100B20002CEA35EC47E257E30E94B0D587FDE4C5D7
:100B30008CA980935F328BE592E30E94874A86E519
:100B4000EBE5F2E3A2EEB6E501900D928A95E1F7AE
:100B500088E1E5EBF2E3AEE7B6E501900D928A9508
:100B6000E1F78091A6328111D5C523E333E34BEC45
:100B700051E46E2D7B2D8A2D99810E9455D84B0111
:100B80005C016093AE567093AF568093B0569093CD
:100B9000B15623E333E34BEC51E4C301B2010E94AD
:100BA00055D8609396567093975680939856909325
:100BB000995623E333E34BEC51E469857A858B85C1
:100BC0009C850E9455D860939A5670939B5680934B
:100BD0009C5690939D5623E333E34BEC51E4612FF5
:100BE000702FC6010E9455D8162F072F412F502F66
:100BF000BC0140939E5650939F566093A0567093AD
:100C0000A1568091703390917133A0917233B0915D
:100C10007333BC01CD019F770E948DD60E9424D6EC
:100C20006093BF567093C0568093C1569093C2563E
:100C3000A091C356A98BB091C456BA8BEB2FF0E0AC
:100C4000ED83FE837F01EE0CFF1CEE0CFF1CF10117
:100C5000EE0DFF1D80819181A281B381BC01CD0188
:100C60009F772CEA35EC47E257E30E94B0D5D82EA7
:100C7000DD1CDD24DD1C3989232F30E029833A83F4
:100C80008901000F111F000F111FF101E00FF11F6B
:100C900080819181A281B381BC01CD019F772CEA33
:100CA00035EC47E257E30E94B0D5881F8827881F9C
:100CB0008D218093BE562CEA35EC47E257E3C501FF
:100CC000B4019F770E94B3D718160CF0F9C0F80151
:100CD000E05AFD4CD801AB54BD4C2D913D914D9146
:100CE0005C9160817181828193810E9407D46B0144
:100CF0007C01ED81FE81EE0FFF1FEE0FFF1FE05A1A
:100D0000FD4CAD81BE81AA0FBB1FAA0FBB1FAB5408
:100D1000BD4C2D913D914D915C916081718182819D
:100D200093810E9407D469877A878B879C87A50166
:100D30009401C501B4010E9455D820E030E040E89C
:100D400050E40E9455D86D877E878F87988BA701C6
:100D50009601C701B6010E9455D82B013C01298597
:100D60003A854B855C85CA01B9010E9455D89B0123
:100D7000AC01C301B2010E9408D49B01AC016D8596
:100D80007E858F8598890E9407D42B013C0120E045
:100D900030E0A9010E94B3D71816C4F4C301B20110
:100DA0000E942ED92B013C0129853A854B855C8513
:100DB000C701B6010E94C0D79B01AC01C301B201BB
:100DC00090580E94B7D52B013C0103C0412C512CF7
:100DD000320180915F32833021F477FA709477F892
:100DE000709420E030E0A901C501B4010E94B0D5A3
:100DF00087FF04C077FA709477F8709409811A819C
:100E0000000F111F000F111FA8014558594A5A0120
:100E1000A301920169857A858B859C850E9455D8AE
:100E20009B01AC01C701B6010E9407D420E030E06D
:100E300040E05FE30E9455D8D5015B966D937D93AA
:100E40008D939C935E97AD80BE80AA0CBB1CAA0CB0
:100E5000BB1CF501E558F94A4F01A3019201C701F6
:100E6000B6010E9455D89B01AC0169857A858B85B6
:100E70009C850E9408D420E030E040E05FE30E94BF
:100E800055D8D4015B966D937D938D939C935E971B
:100E9000E091C556F0E0EE0FFF1FEE0FFF1FE55883
:100EA000F94A138E148E158E168EB091AE56B987F0
:100EB000E091AF56ED872090B0563090B15625C0E6
:100EC0005701F701E558F94A838D948DA58DB68DAC
:100ED0009C01AD015058F801E558F94A838D948D75
:100EE000A58DB68DBC01CD0190580E94C0D79B0145
:100EF000AB01BC014093AE565093AF566093B056D1
:100F00007093B15629873D871C01D801A558B94A6D
:100F10005B96CD90DD90ED90FC905E97E981FA8133
:100F2000EE0FFF1FEE0FFF1FE951F94A13962D91A7
:100F30003D914D915C911697608171818281938181
:100F40000E9407D4A70196010E9407D469837A837F
:100F50008B839C83D501A558B94A5B964D905D90D3
:100F60006D907C905E97ED81FE81EE0FFF1FEE0F7E
:100F7000FF1FE951F94A13962D913D914D915C91D6
:100F8000169760817181828193810E9407D4A301A9
:100F900092010E9407D46D837E838F8398879B0183
:100FA000AC0169817A818B819C810E94C0D729859F
:100FB0003D85A1010E9407D44B015C01E894B7F87C
:100FC00020E030E040E85FE3C501B4010E94B3D700
:100FD00018160CF4C3C32AE037ED43EA5BE3C501FE
:100FE000B4010E94B3D7181694F42FE632E143E817
:100FF0005AE369857D85C1010E9455D89B01AC01EA
:10100000C501B4010E94B3D718160CF4A7C3A301FD
:1010100092015058C701B60190580E947BD44B01F1
:101020005C016093A6567093A7568093A856909340
:10103000A9568091A532813039F4412C512C30E8E9
:10104000632E3FEB732E06C0412C512C20E8622EFC
:101050002FE3722E8091BE568823D1F16091BF5646
:101060007091C0568091C1569091C2560E9450D640
:101070006B017C012CEA35EC47E257E30E94B0D5C6
:1010800087FD10C010915F322BED3FE049EC50E43A
:10109000C701B6010E9455D89B01AC01C12CD12CCF
:1010A0007601B9C081E090E0A0E0B0E08093BF5647
:1010B0009093C056A093C156B093C25610915F3220
:1010C0002BED3FE049EC50E4C12CD12C7601A3C0BC
:1010D0002D813E814F81588569817A818B819C81E8
:1010E0000E947BD469837A838B839C836093AA5606
:1010F0007093AB568093AC569093AD56A501940176
:101100000E9407D46B017C019F772CEA35EC47E203
:1011100057E30E94B0D587FF18C010915F326091ED
:10112000BF567091C0568091C1569091C2560E9490
:1011300050D62BED3FE049EC50E40E9455D89B017E
:10114000AC01C12CD12C760166C029813A814B813A
:101150005C81C501B4010E94B3D71816F4F42BEDDD
:101160003FE049EC50E4C301B2010E9455D89B0115
:10117000AC0169817A818B819C810E9408D4609343
:10118000AA567093AB568093AC569093AD56A5017A
:1011900094010E9407D46B017C0110915F321330DF
:1011A00099F06091BF567091C0568091C156909150
:1011B000C2560E9450D62BED3FE049EC50E40E940D
:1011C00055D89B01AC0127C02BED3FE049EC50E422
:1011D000C301B2010E9455D89B01AC01C701B60101
:1011E0000E9407D47B018C016091BF567091C0565C
:1011F0008091C1569091C2560E9450D62BED3FE08F
:1012000049EC50E40E9455D89B01AC01C701D801BC
:101210006C017D010BC0123049F4C301B2010E9480
:1012200055D8A70196010E9408D40AC0C301B20193
:101230000E9455D89B01AC01C701B6010E9407D49A
:101240007B01AB01BC014093B2565093B3566093FF
:10125000B4567093B5568C015090C556A52DB0E08C
:10126000FD01EE0FFF1FEE0FFF1FE951F94AAA0F14
:10127000BB1FAA0FBB1FA558B94A13962D913D91CC
:101280004D915C91169760817181828193810E945A
:1012900007D44B015C016093B6567093B7568093A8
:1012A000B8569093B9569701A80169857D85C1010B
:1012B0000E9455D86B017C016093BA567093BB565F
:1012C0008093BC569093BD56A50194010E94C0D74F
:1012D00069837A838B839C836093A2567093A35611
:1012E0008093A4569093A5568091A432811117C083
:1012F000F0919832FD834090993220919A322E8B52
:1013000030919B323A8F109298321092993210920B
:101310009A3210929B3281E08093A43212C02091C5
:1013200098323091993240919A3250919B32698132
:101330007A818B819C810E94B7D56D83472E8E8BDD
:101340009A8F598945E3549FF0011124E351FF4CD2
:101350002081318142815381C701B6010E94B7D5F6
:10136000662E072F182F792E2D81342D4E895A8DF8
:101370000E94B0D587FF04C06D80042D1E897A8C31
:101380009A8985E3989FF0011124E351FF4C208155
:10139000318142815381C701B6010E94B7D56B01EB
:1013A0007C019B01AC01662D702F812F972D0E942F
:1013B000B3D7181624F06C2C0D2D1E2D7F2C862DE6
:1013C000902FA12FB72D8093C6569093C756A09308
:1013D000C856B093C95620E030E0A901C501B40158
:1013E0009F770E94B3D7181684F5A5E35A9EF001A3
:1013F0001124E351FF4C2081318142815381C50189
:10140000B4010E94B7D54B015C01E894B7F8A5017F
:101410009401662D702F812F972D0E94B3D7181637
:1014200014F4A72C04C0682C092D1A2DAB2C862D82
:10143000902FA12FBA2D8093C6569093C756A09394
:10144000C856B093C956B62C02C0B62CA72CC09073
:101450002E30D0902F30E0903030F090313020E0BE
:1014600030E040E850E4C701B6010E9455D82B0196
:101470003C0129853D85A10169857D85C1010E94C9
:1014800008D4A70196010E9407D49B01AC01C301B7
:10149000B2010E9455D80E942ED92B013C0120ECAC
:1014A00031EE44E65CE46B2D702F812F9A2D0E9463
:1014B00055D820E030E44CE156E40E94B7D56B01EA
:1014C0007C01209137303091383040913930509143
:1014D0003A3069817A818B819C810E94B7D54B011A
:1014E0005C01A301920169817A818B819C810E94B8
:1014F000B7D587017601A50194010E940CC30E9413
:101500008DD67B018C0120E030E040E85FE30E9453
:10151000B3D718163CF4B701C8010E941FD64B017F
:101520005C0108C0812C912C54018394E12CF12C96
:1015300000E81FE3C701D8018093CA569093CB56A9
:10154000A093CC56B093CD569701A8016091C65692
:101550007091C7568091C8569091C9560E94B7D5D0
:1015600060931757709318578093195790931A5791
:101570008092CE569092CF56A092D056B092D1562D
:101580009701A8016091B2567091B3568091B456FC
:101590009091B5560E94B7D56093D2567093D356AA
:1015A0008093D4569093D5569701A8016091B65672
:1015B0007091B7568091B8569091B9560E94B7D5A0
:1015C0006093D6567093D7568093D8569093D95639
:1015D0008090A6569090A756A090A856B090A95675
:1015E000C501B4010E9424D9C090AE56D090AF5628
:1015F000E090B056F090B1560091C35610E0000F45
:10160000111F000F111F0558194AA70196010E94CA
:1016100055D89B01AC01F801638174818581968165
:101620000E9407D46093DA567093DB568093DC56A1
:101630009093DD56C501B4010E94B4D59B01AC0165
:101640000091C45610E0000F111F000F111F055824
:10165000194AC701B6010E9455D89B01AC01D801B7
:1016600013966D917D918D919C9116970E9407D450
:101670006093DE567093DF568093E0569093E15668
:10168000A091C556B0E0FD01EE0FFF1FEE0FFF1F4A
:10169000E951F94AAA0FBB1FAA0FBB1FA558B94AA7
:1016A00013968D919D910D90BC91A02D8083918377
:1016B000A283B3831092243D8091A2569091A356A9
:1016C000A091A456B091A556BC01CD019F772CEAFC
:1016D00035EC47E257E30E94B0D587FD0FC00E946A
:1016E000D25582E080937D560E94E24B80E039C063
:1016F0008EE837C08EE935C08FE933C089EC31C040
:10170000B101C4010E947F4CC2C9B101C4010E9451
:101710007F4C0ECA8E2D9B2DAA2DB9818093AE567B
:101720009093AF56A093B056B093B1564092965650
:1017300050929756609298567092995629853A859C
:101740004B855C8520939A5630939B5640939C56CC
:1017500050939D564C015D01C60148CA8BE98093A8
:10176000243D6A96CDBFDEBFDF91CF911F910F91CF
:10177000FF90EF90DF90CF90BF90AF909F908F90B1
:101780007F906F905F904F903F902F9008958F9231
:101790009F92AF92BF92CF92DF92EF92FF92CF9340
:1017A000DF9380917D56882309F4B1C00E9417828F
:1017B000843010F482E0ACC02091D2563091D356E0
:1017C0004091D4565091D5566091A6567091A75627
:1017D0008091A8569091A9560E9408D46B017C0173
:1017E0006093A6567093A7568093A8569093A956D7
:1017F0000E9424D98090AE569090AF56A090B056DB
:10180000B090B156C091C356D0E0CC0FDD1FCC0FC5
:10181000DD1FC951D94AA50194010E9455D89B01E9
:10182000AC016091DA567091DB568091DC56909154
:10183000DD560E9408D4688379838A839B83C7011D
:10184000B6010E94B4D59B01AC01C091C456D0E052
:10185000CC0FDD1FCC0FDD1FC951D94AC501B40122
:101860000E9455D89B01AC016091DE567091DF5605
:101870008091E0569091E1560E9408D46883798364
:101880008A839B83C091C556D0E0CC0FDD1FCC0F5F
:10189000DD1FC951D94A2091D6563091D756409173
:1018A000D8565091D956688179818A819B810E944E
:1018B00008D4688379838A839B8382EE96E50E94AD
:1018C000A99688E1E7EEF6E5AEE7B6E501900D9260
:1018D0008A95E1F78091CE569091CF56A091D0563F
:1018E000B091D1560197A109B1098093CE5690933A
:1018F000CF56A093D056B093D156181619061A0693
:101900001B060CF457CF10927D5680E001C083E097
:10191000DF91CF91FF90EF90DF90CF90BF90AF908D
:101920009F908F90089510927D5608954F925F92E8
:101930006F927F928F929F92AF92BF92CF92DF92DF
:10194000EF92FF92CF93DF93CDB7DEB76497CDBF11
:10195000DEBF69837A838B839C8369017A0120E0EF
:1019600030E040E751E40E9455D84B015C0120E093
:1019700030E040E751E4C701B6010E9455D89B0111
:10198000AC01C501B4010E9407D46D877E878F87A3
:10199000988B20E030E040E251EC69817A818B81C4
:1019A0009C810E9455D84B015C0120E030E040E270
:1019B00051E4C701B6010E9455D89B01AC01C50195
:1019C000B4010E9408D4698B7A8B8B8B9C8B2091FD
:1019D000FB553091FC554091FD555091FE5560E00E
:1019E00070E080E89FE30E94B7D54B015C0120E0E6
:1019F00030E040EC50EC69817A818B819C810E94BF
:101A000055D82B013C0120E030E040EC50E4C70108
:101A1000B6010E9455D89B01AC01C301B2010E94DE
:101A200008D4A50194010E9455D8A50194010E94F3
:101A300055D8A50194010E9455D8A50194010E9492
:101A400055D8A50194010E9455D86B017C01A501D0
:101A500094016D857E858F8598890E9455D8A50152
:101A600094010E9455D8A50194010E9455D8A50162
:101A700094010E9455D86D837E838F839887A5013A
:101A8000940169897A898B899C890E9455D8A5011E
:101A900094010E9455D8A50194010E9455D86987E8
:101AA0007A878B879C8720E030E042EF50E4C701C3
:101AB000B6010E9455D82B013C0120E030E040EAFD
:101AC00050E46D817E818F8198850E9455D89B015D
:101AD000AC01C301B2010E9408D42B013C0120E0FB
:101AE00030E040E550E469857A858B859C850E94CD
:101AF00055D89B01AC01C301B2010E9408D4609388
:101B00001F5670932056809321569093225620E0C2
:101B100030E045EA52E4C701B6010E9455D82B01D6
:101B20003C0120E030E048EE51E46D817E818F8100
:101B300098850E9455D89B01AC01C301B2010E9457
:101B400008D42B013C0120E030E040E151E46985FC
:101B50007A858B859C850E9455D89B01AC01C30179
:101B6000B2010E9408D460931B5670931C56809358
:101B70001D5690931E5620E030E04FE753E4C70116
:101B8000B6010E9455D82B013C0120E030E040E432
:101B900052E46D817E818F8198850E9455D89B018A
:101BA000AC01C301B2010E9408D42B013C0120E02A
:101BB00030E040EC50E469857A858B859C850E94F5
:101BC00055D89B01AC01C301B2010E9408D46093B7
:101BD0001756709318568093195690931A5620E012
:101BE00030E046E953E4C701B6010E9455D82B0105
:101BF0003C0120E030E040EC51E46D817E818F813A
:101C000098850E9455D89B01AC01C301B2010E9486
